:1000000090F70020913200006F4F01007D32000018
:100010007D3200007D3200007D3200007D32000024
:100020000000000000000000000000006D33000030
:100030007D32000000000000693500007D320000C4
:10004000E1350000E1350000E1350000E135000058
:10005000E1350000E1350000E1350000E135000048
:10006000E1350000E1350000E1350000E135000038
:10007000E1350000E1350000E1350000E135000028
:10008000E1350000E1350000E1350000E135000018
:10009000E1350000E1350000E1350000E135000008
:1000A000E1350000E1350000E1350000E1350000F8
:1000B000E1350000E1350000E1350000E1350000E8
:1000C000E1350000E1350000E1350000E1350000D8
:1000D000E1350000E1350000E1350000E1350000C8
:1000E000E1350000E1350000E1350000E1350000B8
:1000F000E1350000E1350000E1350000E1350000A8
:10010000E1350000E1350000E1350000E135000097
:10011000E1350000E1350000E1350000E135000087
:10012000E1350000E1350000E1350000E135000077
:10013000E1350000E1350000E1350000E135000067
:10014000E1350000E1350000E1350000E135000057
:04015000E135000095
:1001540053B94AB9002908BF00281CBF4FF0FF312A
:100164004FF0FF3000F00CB8ADF1080C6DE904CE8F
:1001740000F010F8DDF804E0DDE9022304B0704774
:10018400704700BF034613F8012B002AFBD1181A4D
:10019400013870472DE9F0478C468E46089E154677
:1001A40004461946002B40F0D080724547D9B2FA74
:1001B40082F74FB1C7F120030EFA07FCBD40BC40E3
:1001C40020FA03F343EA0C0C4FEA154EA8B2230CB1
:1001D400BCFBFEF80EFB18CC08FB00F943EA0C4309
:1001E400994528D9EB1808F1FF3204D2994502D970
:1001F400A8F102022B44A3EB0903A4B2B3FBFEFC57
:100204000EFB1C330CFB00F044EA0344A04214D957
:100214002C190CF1FF3304D2A04202D9ACF1020331
:100224002C44241A43EA02401EB1FC4000233460EB
:100234007360BDE8F0874246DDE76346F1E7002AD4
:1002440079D0B2FA82F3002B3FD01946C1F12003D2
:1002540002FA01F500FA01F42EFA03F20EFA01FE95
:1002640020FA03F3AFB243EA0E034FEA154EB2FB92
:10027400FEFC0EFB1C201A0C0CFB07F842EA0042A1
:1002840090455AD9AA180CF1FF3004D2904502D9EE
:10029400ACF102002A44A2EB08029BB2B2FBFEFCC2
:1002A4000EFB1C220CFB07F743EA02439F4246D98C
:1002B400EB180CF1FF3204D29F4202D9ACF10202D6
:1002C4002B44DB1B42EA004202E0AEEB02030122B4
:1002D4004FEA154EAFB2200CB3FBFEFC0EFB1C33F1
:1002E4000CFB07F840EA034398452AD9EB180CF1B4
:1002F400FF3004D2984502D9ACF102002B44A3EBA1
:100304000803A4B2B3FBFEFC0EFB1C330CFB07F783
:1003140044EA0344A74216D92C190CF1FF3304D242
:10032400A74202D9ACF102032C44E41B43EA004087
:100334000F46114678E71F2188E76046ABE762461F
:10034400BFE76046DBE76346EFE7734506D916B9B6
:10035400002108466DE7C6E9000EF9E7B3FA83F712
:1003640087B9734501D3824207D8841A6EEB03031D
:1003740001209C461EB900215BE73846FAE7C6E92E
:10038400004CF8E7C7F1200CBB4000FA07F422FA4E
:100394000CF520FA0CF1BA401D432EFA0CF30EFAB8
:1003A40007FE4FEA154941EA0E011FFA85FEB3FB29
:1003B400F9F809FB18300B0C08FB0EFA43EA00436A
:1003C4009A4540D9EB1808F1FF3004D29A4502D976
:1003D400A8F102002B44A3EB0A0389B2B3FBF9F89A
:1003E40009FB183308FB0EFE41EA03418E452CD964
:1003F400691808F1FF3304D28E4502D9A8F102032B
:10040400294443EA0040A1EB0E01A0FB02984145B8
:10041400CE46434602D306D14C4504D20138B9EB4B
:10042400020E68EB0503002EA5D0B4EB0E0261EBBF
:10043400030101FA0CFC22FA07F3F9404CEA030326
:10044400C6E9003197E74046C5E74346D9E70000CF
:1004540031492DE9F0438B4208BF012A93B006D0FD
:100464008B4208BF022A42D013B0BDE8F0832B4D63
:1004740084682B680133012B2B600DD1284B294A4A
:100484000393294B29490293294B2A4801932A4B68
:1004940000932A4B14F086FA2022214609A816F06C
:1004A40074FA002394F824002E688DF8443094F8EC
:1004B400217094F8238094F9279004F08FFA94F82B
:1004C4002E3005468BB11223062104AA04F128001C
:1004D40004F050FDCDE902503B463146CDE9008998
:1004E400174809AA14F05EFABEE71648F2E78368D3
:1004F4001B686BB10121144A144814F089FC0022D2
:10050400064B1A60124813B0BDE8F0430BF0B0BCC0
:10051400104814F047FAF2E70000D0D0C0110020D0
:10052400DF750100E0750100E5750100AE7501009D
:10053400EE750100B2750100F3750100A8750100A4
:10054400F8750100C58E010025760100AC6E01002E
:10055400B80400203E7601000022B0B55B4B8EB09B
:100564001A6083225A495B4B02AF4B605A4B0846D0
:10057400C1E9042304F080FE00214FF400400DF093
:1005840063FA564B56491A68564B5748B2FBF3F276
:1005940014F008FA04F018FB70B1036863B15A7CD4
:1005A400062A09D1D3F812003860DB8A3846BB80AA
:1005B40014F059F800285BD14C4814F054F850B9A1
:1005C40001214B4A4B4814F01AFC6FF015042046E5
:1005D4003037BD46B0BD04F0F7FA0546A0B1036854
:1005E40093B10C33D3E8AF3FDB070DD504F052FBD6
:1005F400041E09DA14F1780F06D023463E4A01217D
:100604003C4814F005FCE2E700233B60BB80302348
:100614002A463A49009301203B4604F08DF82846C7
:1006240004F0E4FA041E05DA14F1780F02D0344A17
:100634002346E4E7002D45D02868002842D0417CB9
:100644001823304A123004F095FC6C4688B002AA94
:100654002D4BC2E905304FF4007393832B4B42F8C2
:10066400103F00234FF4E651224801F0B3FEA546A3
:1006740004F0AAFA182504462A460021384616F042
:100684006CF98223BB80322322467B8001203B46C7
:100694001F49009504F0AEF950B101211D4A1548D7
:1006A40014F0ADFB00214FF4A0200DF0CDF9DFE7ED
:1006B400194814F077F94FF4A022002317480BF0DF
:1006C4005BFCEFE700235B78FFDE00BFC011002076
:1006D400D0050020550400000000D0D010020020F6
:1006E4005176010040420F005B7601005DCF0100AE
:1006F40083760100AC6E0100D276010000009050B8
:10070400EF760100342A00200A770100030000017B
:100714000000D0503577010049770100B80400206B
:100724002DE9F04104460D4613F0F3FF80460028FE
:100734004BD12946204613F0BDFF0146204614F054
:1007440000F804EB80010E6996B90122E368824047
:100754001343E36002220D612B462946204613F021
:100764009EFF032229462046BDE8F04113F097BFBF
:1007740002223146204613F087FF03220146074632
:10078400204613F081FF86420BD00121104A114804
:1007940014F035FB88F31188BFF36F8F04231846D8
:1007A40002DF3B4602222946204613F078FF03224B
:1007B40033462946204613F072FF39462B4620461D
:1007C40013F06DFF02223146CDE7BDE8F08100BF92
:1007D4005E770100A46E01002DE9F0411746032263
:1007E4000E46044613F050FF8642054607F10408FE
:1007F4000AD10122E368BA4023EA0203E36000233A
:1008040044F82830BDE8F08102223146204613F036
:100814003BFF032201460746204613F035FF86427C
:1008240006D102222946204613F02EFF86420CD020
:1008340001210E4A0E4814F0E2FA002383F31188D2
:10084400BFF36F8F0423184602DF2B463946204638
:10085400032244F8285013F022FF3B462946204641
:10086400BDE8F041022213F01ABF00BF5E77010019
:10087400A46E010038B5012205460C4613F004FFAE
:10088400C30713D42146284613F03DFF01462846EA
:1008940013F032FF844209D12146284613F02CFF7D
:1008A4000146284613F02FFF84420CD00121064A4A
:1008B400064814F0A4FA002383F31188BFF36F8F62
:1008C4000423184602DF38BD82770100A46E0100BC
:1008D4002DE9F8430E4600AF002900F0A380046818
:1008E4000122204613F023FF01460546204613F05B
:1008F400CBFE10EA020816D1E94688B06A464B4B93
:10090400CDE90536032342F8103F4FF4C251434664
:10091400474801F05FFDCD4688F31188BFF36F8F20
:100924000423184602DF2946204613F0ECFE014654
:10093400204613F0E1FEA84217D0E84688B06A4684
:100944003C4BCDE90536032342F8103F00234FF416
:10095400C251374801F03EFD0023C54683F3118898
:10096400BFF36F8F0423184602DF2946204613F095
:10097400C3FE0146204613F0C6FEA84217D0E8463F
:1009840088B06A462C4BCDE90536032342F8103F64
:1009940000234FF4C251264801F01CFD0023C54634
:1009A40083F31188BFF36F8F0423184602DF0022FC
:1009B4002946204613F084FE294613F0A4FE0122A2
:1009C40001460646204613F05FFEC2070CD43146AA
:1009D4002046FFF74FFF3146204613F001FF324611
:1009E4002946204613F0B7FE2946204613F084FE1C
:1009F400012201460646204613F046FEC3070DD4E5
:100A040031462046FFF736FF3146204613F0E8FE14
:100A14002A463146204613F09EFE35462946204696
:100A2400FFF77EFEBD46BDE8F88300BF1B780100DA
:100A3400A46E0100CB770100F47701002DE9F047A3
:100A44004B42066803EA010731EA03031446B2681D
:100A54001DD0B2F5004F2CBF08230423BB4228BF8E
:100A64003B46B946CF1B07F1FF3A1AEA070F1DD0E0
:100A74003C4940F2E9133C4A3C4813F0A9FF3C4886
:100A840013F0A6FF40F2E911374813F098FFB2F5CE
:100A9400004F34BF04230823994204D82146BDE8FB
:100AA400F04713F0F1BE4FF00009DCE71CB9002554
:100AB4002846BDE8F087B2F5004F34BF0425082569
:100AC400FB1AE10804F0070001EBD301073003F03F
:100AD400070303442B4401EBD301914228BF114681
:100AE400304613F093FE80460028E0D0B36809EB4B
:100AF400C005B3F5004F34BF042308231D44354417
:100B04005544B5FBF7F57D43A5EB09052946304669
:100B140013F00DFE2C44073424F00704A41B804575
:100B240007464FEAE40408D202464146304613F031
:100B340030FE41463046FFF7F3FD3946304613F0A8
:100B4400E2FDA04208D939463046224613F021FE80
:100B540021463046FFF7E4FD01223946304613F0C2
:100B6400AFFDA5E763780100407801007E780100BD
:100B74009B780100B2F5802FF8B510D2042A28D84A
:100B84003F4940F2E3233F4A3F4813F021FF3F48E7
:100B940013F01EFF40F2E3213A4813F010FF08233C
:100BA400D21ACC1D114424F0070421F00701091BBB
:100BB40017294FEAD1060ED835494FF43B73314A11
:100BC400314813F005FF314813F002FF4FF43B7135
:100BD400E2E70423E4E70023046031462046A660EC
:100BE400E36013F0AEFD820002F11B05B6F5004F81
:100BF4004FEAD5050FD26B1C9E420CD2254940F218
:100C04000233204A204813F0E3FE204813F0E0FEAC
:100C140040F20231C0E70021043204F1100015F063
:100C24009CFE2A462046002113F062FD0023204644
:100C34001A46194613F033FD771B19462046012244
:100C440013F03EFD3A46294613F052FD2B4600228E
:100C54002946204613F023FD3146204613F048FD73
:100C64003B4631462046002213F019FD314620460A
:100C7400012213F025FD2946BDE8F840FFF750BDD9
:100C8400B8780100407801007E780100D97801002D
:100C9400F27801001B7901002DE9F04F95B000AF07
:100CA4008A460546C7E9083258B99A4940F2993349
:100CB400994A9A4813F08CFE40F29931964813F001
:100CC4007EFE49B903784678807800EB8300284497
:100CD400564521D8A0EB050ABB6F95F8028003F0B6
:100CE4000103BC6F3B61EB78B8F1000F0CBF00242B
:100CF40004F00104FB6113B1BB6F9A0715D4A4B9C6
:100D04007B6A1BB1514628463A6A98475646304694
:100D14005437BD46BDE8F08F441C2046FFF732FA35
:100D2400013020440AF1010AD2E7BB6FC3F3C003C8
:100D34007B612B78FB609B007B606B68BB60FB680E
:100D440005EB830B7B6A002B71D15646D844ACB1BA
:100D54001C461BF8013B55F82300FFF713FAFB6F01
:100D640001303BB1D7F88030A34282BFFB6F23F838
:100D740014000134C3450644EBD1D846BB6F4FF091
:100D8400000913F0050F0CBF4FF0020B4FF0010BDD
:100D9400FB699945BBD298F8013008F1020855F86F
:100DA40023A05F4B9A45C0F080815E4B7A699A45D7
:100DB4002CBF002301230AB318F8021CB8687B6215
:100DC40013F0D1FD7B6AC8B1EA468AB06A46564B35
:100DD4000593BB68CDE906314FF40073ADF82030BC
:100DE400524B42F8103F00234FF41251504801F087
:100DF400F1FAD546023E09F10109C9E723B13B697D
:100E04002BB9A6EB0B06F6E7BB6F9B07F3D5504651
:100E1400FFF7B8F9FB6F43B1D7F880309C423FBF6E
:100E2400FA6F431C22F8143001340644E3E7002C23
:100E340065D1B8F1000F68D0BB6F580768D5C146BB
:100E440007F140004246594615F061FD0BEB0803DB
:100E5400BB610023334AF9698B426BD3BA6F95F8AF
:100E640001B03969920704EB0B0348BF0022DBB2DF
:100E740058BF4FEA5902002940F0E180B96F11F0E0
:100E8400040F14BF494600216B70A970EA7028460C
:100E94003A6A79687B6A9847061EFFF638AFFB68A2
:100EA40049462B70FB693A6AEB7085F801B07B6A9E
:100EB40085F8028007F140009847B0F10009C0F2BC
:100EC400F0807B68FA69B86903EB420141443A6AED
:100ED4007B6AAAEB010198470028C0F2E4804FF036
:100EE400000BB14409EB000607F1300AA345C0F03A
:100EF400A88000213A6A08467B6A984707E7444677
:100F04004FF0000907F130009CE74446C1469DE7D5
:100F1400A1469BE7CE7901004E7901007E7801005D
:100F2400906A0100E46B0200E97901000400000109
:100F3400546E0100B869DFF88CC110F8021B10F878
:100F4400016CB86155F826006045C0F0B480904249
:100F540078692CBF4FF0000B4FF0010B30B1B8682B
:100F64003B6013F000FD3B68574A60BBBBF1000FC8
:100F74002BD0396959B10F2C36D9544940F2434327
:100F8400534A544813F024FD40F2434196E6B96FA6
:100F9400490718D5B9F10F0F09D94F4940F2464313
:100FA4004B4A4C4813F014FD40F2464186E609F1E1
:100FB400280007F1280C09F1010100EB0C0909F8DC
:100FC400106C5FFA81F9013345E7B86F800715D5D6
:100FD4000F2C09D93D4940F24D433D4A3D4813F099
:100FE400F7FC40F24D4169E6611C04F1280007F169
:100FF4002804041904F8206CCCB2E4E7B9F10F0F0B
:1010040009D935494FF48A63314A324813F0E0FC78
:101014004FF48A6152E609F1280C07F1280EF444D2
:1010240009F101000CF8101C07F1500109F1020943
:1010340051FA80F05FFA89F900F8106CC3E70021D7
:1010440022E71BF80A3055F8239087F82F30FB6FFE
:1010540023B3D7F880309B4520D2FB6F33F81B8035
:1010640001213A6A7B6A07F12F00984700281ADBAE
:101074000644B8F1000F06D14846FFF783F800F1A3
:1010840001081FFA88F8414648463A6A7B6A98473D
:10109400002808DB06440BF1010B27E74FF000089A
:1010A400DEE74E4633E6064631E67B69002B3FF425
:1010B400ABAE002380E67869002886D04FF0000BA1
:1010C4004DE700BF906A0100E46B02008C7A0100D6
:1010D4004E7901007E780100AB7A0100014B1B6858
:1010E400184700BF00000020014B1860704700BF84
:1010F4000000002030B5044685B00D4610220021C2
:10110400684615F02AFC02238DF80230044B2A4667
:1011140021466846019313F03DF805B030BD00BF89
:10112400E110000080B505460E46174698460CF0BF
:1011340033FD034602F0A2FADFF83C90044649F876
:101144000030424639463046A8470C4B1B7873B9E9
:101154000B4940F246330B4A0B4813F039FC0B4859
:1011640013F036FC40F24631064813F028FC54F8DC
:10117400090002F0E1F900BF080000009B2C0020E8
:10118400077B0100DC7A01007E7801001A7B0100F4
:1011940038B50D4604462022002115F0DEFB00225E
:1011A400EB68E361AB68A3612B6823626B68A2629E
:1011B40063622A6923B1591E194208BF42F0010231
:1011C40022610122002104F12C0015F00BF848B132
:1011D400054906482F23064A13F0FAFB2F21044839
:1011E40013F0EDFB38BD00BF627B01007E78010087
:1011F4003C7B01002DE9F04F002789B0CDE90123A4
:10120400436A04468B428846BA460597079754D3E7
:1012140000F11406EFF31185202383F31288BFF342
:101224006F8F3046A9460CF035FF58B984234D4AD8
:101234004D494E4813F0CCFB31464D4813F0C8FBE2
:10124400842163E030460CF049FF079A2AB13946FD
:10125400204613F0A3FC0023079306A9204613F0AD
:10126400C4FB06998346414530D32268236A20464D
:1012740013F8221003EB820A21F0030103F8221071
:101284002168424613F0D5FBE3682060984218D0E9
:101294004FF0000B30460CF00BFF50B389F311886C
:1012A400BFF36F8F059929B1A2690AB1204690470F
:1012B40000230593BBF1000FACD1504609B0BDE843
:1012C400F08F236943F008032361E1E718B1204656
:1012D40013F0C9FBDEE7DDE90132134339D0039192
:1012E40014F0F4FF0399A0BB9DBB30460CF0E0FE64
:1012F40078B94FF499731B4A1E491C4813F068FBD4
:1013040031461D4813F064FB4FF49971154813F0EE
:1013140056FB85F31188BFF36F8F04F12C00DDE9D0
:1013240001230AF029FE8346EFF31189202383F376
:101334001288BFF36F8F30460CF0ACFE00283FF4E8
:1013440075AFBBFA8BFB30460CF0C8FE4FEA5B1B53
:10135400A0E7204607AB05AA276813F0A3FB834642
:1013640098E700BF6B7B0100987B01007E78010049
:10137400AD7B0100C37B0100DA7B01002DE9F04164
:101384000446C36908460E46984704F11405074607
:10139400EFF31188202383F31288BFF36F8F28465D
:1013A4000CF078FE68B984231A4A1B491B4813F0D1
:1013B4000FFB29461A4813F00BFB8421154813F040
:1013C400FEFA28460CF08AFE33783A4643F00103CD
:1013D40033706168204613F02CFB6060204613F0E4
:1013E400F8FB28460CF064FE68B94FF49973094A77
:1013F4000C490A4813F0ECFA29460B4813F0E8FAB2
:101404004FF49971DAE788F31188BFF36F8FBDE861
:10141400F08100BF6B7B0100987B01007E780100A6
:10142400AD7B0100C37B0100DA7B01002DE9F047AD
:101434000446002700F11406EFF31188202383F3F8
:101444001288BFF36F8F30460CF024FE054668B94E
:101454008423394A39493A4813F0BAFA31463948AB
:1014640013F0B6FA8421344813F0A9FA30460CF08C
:1014740035FE2369A168180702D463688B4200D241
:10148400636A5B1A002B41D0206A10F8213000EB0C
:10149400810913F003023CD0022A04D150F8212020
:1014A4005FEA920A05D1DA0720D44846E3699847EF
:1014B4008246A1685246204613F0BBFA5146A0600A
:1014C400204613F0C4FA2F4630460CF0F1FD10BB51
:1014D4004FF49973184A1C49194813F079FA3146A4
:1014E4001A4813F075FA4FF49971BCE743F00203FC
:1014F40000F82130E3694846A56898472946024622
:10150400204613F096FA0025A060DDE71D46A946A3
:10151400DAE71546FBE788F31188BFF36F8F002DD8
:101524008AD137B1B9F1000F03D104F12C000AF0CC
:101534009FFC4846BDE8F0876B7B0100987B010067
:101544007E780100AD7B0100C37B0100DA7B0100E2
:101554002DE9F0410446C36908460D46984704F155
:1015640014060746EFF31188202383F31288BFF390
:101574006F8F30460CF08EFD68B98423274A2849C2
:10158400284813F025FA3146274813F021FA84211C
:10159400224813F014FA30460CF0A0FD2B7823F007
:1015A40001032B7023699B0705D5E268236A03EBCB
:1015B40082039D4222D12B7823F002032B70D4E9BD
:1015C4000231994204D13A46204613F032FAA0601F
:1015D4003946204613F03BFA30460CF069FD90B9C9
:1015E4004FF499730D4A11490E4813F0F1F931463D
:1015F4000F4813F0EDF94FF49971C9E72B6867F3BD
:101604009F032B60E8E788F31188BFF36F8F04F121
:101614002C00BDE8F0410AF02BBC00BF6B7B01003D
:10162400987B01007E780100AD7B0100C37B010043
:10163400DA7B010070B5044600F11405EFF311865E
:10164400202383F31288BFF36F8F28460CF022FD0A
:1016540068B984231A4A1B491B4813F0B9F929466F
:101664001A4813F0B5F98421154813F0A8F928464F
:101674000CF034FD2369A0681B0702D4636883421D
:1016840013D2646A241A28460CF012FD78B94FF478
:1016940099730B4A0E490C4813F09AF929460D48E0
:1016A40013F096F94FF49971DEE71C1AEBE786F311
:1016B4001188BFF36F8F201E18BF012070BD00BFBB
:1016C4006B7B0100987B01007E780100AD7B0100FB
:1016D400C37B0100DA7B01002DE9F84F0546AB8B93
:1016E40008461907904616D501280CBF43F010038D
:1016F40043F02003AB83143528460CF0D9FC0028B2
:1017040040F0B181AE494FF49973AE4AAE4813F03C
:101714005FF929469DE0022803F0070140F07D812E
:10172400284613F070FA052800F2FA8001A353F852
:1017340020F000BFFB1600001F1A0000251900004E
:10174400C917000063180000C318000002F0070264
:10175400531F012B1AD80023062A2E68A4B2C5E908
:10176400003309D1334603E0EA8B0132EA831B6874
:10177400002BF9D144F002042846AC8313F043FA59
:10178400002800F05A8144F0200455E1042A0DD1C8
:10179400A4B22846AC8313F036FA0646002800F0BB
:1017A4004C8144F020040026AC8346E1874940F292
:1017B4001B13874A844813F00BF940F21B11844829
:1017C40013F0FDF849B183494FF4AB73804A7E4866
:1017D40013F0FEF84FF4AB71F1E72B684BB97E4977
:1017E40040F257137A4A784813F0F2F840F257114E
:1017F400E5E72B691F684FB978494FF4AD73744A14
:10180400714813F0E5F84FF4AD71D8E70E468A46F7
:101814004FF00609AC8B24F0070444F00604A4B28C
:10182400AC83AB68002B00F00F814FF0010B44F048
:101834000804AC8305F1140420460CF039FC00289C
:1018440078D15F494FF499735E4A5F4813F0C0F84A
:101854002146634813F0BCF84FF499718EE00229D5
:1018640009D0604940F25D13594A574813F0B0F863
:1018740040F25D11A3E7EE8B4EB15B494FF4AF73B9
:10188400534A514813F0A4F84FF4AF7197E72B690A
:101894005F684FB9514940F261134D4A4A4813F009
:1018A40097F840F261118AE7AC8BB24624F0070442
:1018B40044F00404A4B24FF00409AC83B1E7012955
:1018C40009D04A494FF4B273414A3F4813F080F8B3
:1018D4004FF4B27173E72B684BB93F4940F265137B
:1018E4003B4A394813F074F840F2651167E72B69F5
:1018F4009F684FB939494FF4B473354A324813F0ED
:1019040067F84FF4B4715AE70026AC8BB24624F062
:10191400070444F00504A4B24FF00509AC8380E742
:101924002A4940F26B132A4A274813F051F840F22F
:101934006B1144E788F31188BFF36F8FBBF1000F7D
:101944001ED1002E33D117B128462949B847EFF3E9
:101954001188202383F31288BFF36F8F20460CF085
:1019640099FB00284AD18423164A2249164813F0C9
:101974002FF82146204813F02BF8842111481FE743
:10198400A9680029DDD0D1F800800029D9D05346B8
:101994004A462846D1F804B0D847B8F1000F04D01D
:1019A400D8F8003041469846EFE74346FAE7314617
:1019B40053464A462846366813F051F9C1E700BF3A
:1019C400C37B01006B7B01007E7801003DA4010014
:1019D400FA7B01001F7C01002B7C01004E7C01007E
:1019E400DA7B0100657C01007B7C01008A7C0100BC
:1019F400791A0000987B0100AD7B010020460CF0B1
:101A04006DFBAC8B24F00804A4B2AC83E20621D5B0
:101A140024F01003AB8304F00701D5F818A0AA8BB7
:101A2400BAF1000F22F00704BFF690AE00232E682F
:101A3400C5E9003344F00104AC8304F00709894587
:101A44004FF000077FF4EDAE0EB9002FDED04FF05B
:101A5400000BECE6A3067FF54EAE24F02003AB8327
:101A640004F007015CE688F31188BFF36F8FBDE8CB
:101A7400F88F00BFF8B504460D4600F11406EFF3E5
:101A84001187202383F31288BFF36F8F30460CF045
:101A940001FB68B984230C4A0C490D4812F098FFE5
:101AA40031460C4812F094FF8421074812F087FF56
:101AB40030460CF013FBA5613A462046BDE8F840D9
:101AC4000121FFF709BE00BF6B7B0100987B010079
:101AD4007E780100AD7B01002DE9F04704460E46F7
:101AE40013F0ADF8051E66DB04F11409EFF3118A57
:101AF400202383F31288BFF36F8F48460CF0CAFA91
:101B0400804660B98423374A3749384812F060FF69
:101B14004946374812F05CFF8421324843E0484686
:101B24000CF0DCFA4FF6FF72E38BA78B934207F0BD
:101B3400070743D0062F2CD8DFE807F01F43092BF3
:101B44001F041F006FF085054FF0000802E0022516
:101B54000133E38348460CF0ABFA002834D14FF448
:101B64009973204A2349214812F032FF49462248FA
:101B740012F02EFF4FF49971CFE7002333606368AE
:101B840023B9C4E9006687B13D46DDE71E6066609F
:101B9400F9E71A4915484FF4E473194A12F018FF8B
:101BA4004FF4E471164812F00AFF5246022120460F
:101BB400FFF792FD3D462846BDE8F0876FF00A0521
:101BC400C2E76FF00405BFE78AF31188BFF36F8F94
:101BD400B8F1000FEFD000233A463146204613F007
:101BE4003EF8E8E76B7B0100987B01007E780100FA
:101BF400AD7B0100C37B0100DA7B01008A7C01001C
:101C0400FA7B010010B54268034602F00302022A7F
:101C1400816016D0032A0BD0012A15D00C490D4837
:101C240045230D4A12F0D4FE45210B4812F0C7FE9D
:101C34000468002000225A6008B10CF0E3FE20463C
:101C440010BD00240068F5E700242046F2E700BF39
:101C54003DA401007E780100A07C010008B558B9BC
:101C64000749084840F23513074A12F0B1FE40F222
:101C74003511054812F0A3FE4368587908BD00BF2A
:101C8400FE7C01007E780100C67C010010B548B9D5
:101C940008490948A023094A12F09AFEA0210748DE
:101CA40012F08DFE03681B6913B1BDE8104018479C
:101CB400184610BDFE7C01007E780100C67C010040
:101CC4002DE9F843044606460127DFF8408094FADC
:101CD400A4F5B5FA85F507FA05F308EB05156FEADF
:101CE400030924EA03042B7B5BB12846FFF7CEFFEC
:101CF40038B96B6804222846196806EA090613F005
:101D04000EF8002CE3D13046BDE8F883DC6E010008
:101D140010B5002288B00E490E4814F0AAFB002228
:101D240000230024CDE906230E234FF40062CDE9FD
:101D34000334CDE90144084B0849009408480AF0EB
:101D4400B9FF0849064814F0C7FA204608B010BD88
:101D54004D1E0000700A002095210000A02C0020D8
:101D6400E8050020157D01002DE9F047DFF8B89063
:101D74002E4C8046A9EB04038F2B0F460BD92C491C
:101D840040F253132B4A2C4812F022FE40F2531116
:101D9400284812F014FE294812F0B3FF064660B337
:101DA40000252846BDE8F087237B8BB12368DB68D8
:101DB4000BB1204698476368204683F806A0FFF7D6
:101DC40065FFB0B9636804222046196812F0A7FFC2
:101DD400013610344C4514D9194940F25F13154AA1
:101DE400154812F0F5FD174812F0F2FD40F25F11AC
:101DF400CEE70AFA06F31D43EAE705464FF0010A67
:101E0400E8E7D1D3B8F1000FCBD0002DC8D02846D5
:101E1400FFF756FF0546002FF7D000214FF4A470BA
:101E24000BF012FEF1E700BFEC6E0100DC6E010066
:101E34004A7D01001D7D01007E780100D81100203B
:101E44007A7D01009B7D010001480AF011B800BFB2
:101E5400A0040020014B53F8200070475C6F010080
:101E640008B5034608462BB1044A136000F022FD6E
:101E7400002008BD6FF01500FBE700BF0400002040
:101E840010B5044C237813B9034809F0F1FF01237A
:101E9400237010BD4C2A0020A004002010B5044675
:101EA400094812F02EFF3CB1084BD3E8EF1F01396B
:101EB400C3E8E21F002AF8D105480CF0D9FCBDE8BC
:101EC4001040044809F0D4BFD0110020D4110020E0
:101ED400700A0020A00400200022044BD3E8EF0F76
:101EE400C3E8E12F0029F9D1704700BFD0110020C9
:101EF40070B5FFF7F1FF0546104C114EB4421AD9E4
:101F0400104940F21623104A104812F061FD10489F
:101F140012F05EFD40F216210B4812F050FD2046EF
:101F2400FFF79CFE28B123685B6813B1294620465D
:101F340098471034E2E7F2D370BD00BFDC6E0100B5
:101F4400EC6E01007A7D01001D7D01007E780100A8
:101F54009B7D010010B5044C04492046FFF718F995
:101F6400034B1C6010BD00BF18030020486F010024
:101F7400C41100200023154A10B51370144A4FF4FD
:101F840000411360134A14481360FFF769FFFFF719
:101F9400E1FF124B124918468B4215D9114940F200
:101FA4002B13114A114812F013FD114812F010FDC1
:101FB40040F22B110C4812F002FD1A1A5C6812113F
:101FC400013222711033E7E7F7D310BD4D2A002008
:101FD400D0110020D4110020034D0100DC6E01005B
:101FE400EC6E01007A7D01001D7D01007E78010008
:101FF4009B7D01000146002200230148FFF7FAB847
:10200400180300200148FFF711BA00BF180300208D
:10201400024B01461868FFF79BBA00BFC4110020A9
:102024000148FFF707BB00BF1803002070B5314B10
:102034001B78002B5BD0FFF7E5FF0446002846D150
:102044002D4B2E4D1B68002B19DD14F0CAF94FF4EB
:102054007A76A0FB063206FB0121D5E90020DB0BD2
:1020640043EA41439B1A40F2E9324FEAD13161EB32
:102074000001934271F1000101D3FFF739FFD5E963
:10208400003213F57A7342F10002C5E9003274B3E9
:10209400BDE87040FFF7C4BF2846FFF7DFFD20B15D
:1020A4002B68214628461B6898471035B54211D93C
:1020B400134940F20A23134A134812F089FC1348C7
:1020C40012F086FC40F20A210E4812F078FC104D02
:1020D400104EEBE7E0D32046FFF79AFF0E4BD3E810
:1020E400EF1F0139C3E8E21F002AA9D0F7E7002057
:1020F40070BD00BF4C2A0020D0110020680A0020C7
:102104007A7D01001D7D01007E7801009B7D010028
:10211400DC6E0100EC6E0100D411002070B5154D89
:10212400297831BB0120FFF71FFE134C134EB44234
:1021340018D9134940F2CF13124A134812F048FC3D
:10214400124812F045FC40F2CF110E4812F037FC51
:102154002046FFF783FD18B1236820469B68984703
:102164001034E4E7F4D3FFF761FF0028FBD1012327
:102174002B7070BD4D2A0020DC6E0100EC6E010056
:102184007A7D01001D7D01007E7801009B7D0100A8
:102194002DE9F843374F384BFB1A1B090AD137494D
:1021A4004FF46F73364A374812F012FC4FF46F71D4
:1021B400334819E000210846FFF7D6FD0446A8B1CC
:1021C40040F267684FF000092F4B1B789BB92F49E9
:1021D40040F246332E4A2B4812F0FAFB2D4812F0F7
:1021E400F7FB40F246312A4812F0E9FB4FF0FF3882
:1021F4004FF0FF39E8E701F041FA274B274A1B5813
:10220400136033B1264B1B68092B02DD254809F006
:102214002FFE002544B12046FFF752FD044618B9AD
:102224004FF0FF384FF0FF39FFF700FF064628B99B
:1022340035B91C4842464B4609F09EFE3546E9E74F
:102244000D4D08E0F5D22B689B691BB1002228468E
:10225400114698471035BD42F4D913494FF46C73B5
:10226400074A084812F0B4FB104812F0B1FB4FF4CF
:102274006C719DE7EC6E0100DC6E0100BA7D01001B
:102284001D7D01007E7801009B2C0020077B01004E
:10229400DC7A01001A7B010008000000CC11002048
:1022A400D4110020A00400207A7D01009B7D010050
:1022B40013B52C4812F025FD2B4B1B78002B35D081
:1022C400EFF31184202383F31288BFF36F8F274821
:1022D4000BF0E0FE68B98423254A2649264812F00B
:1022E40077FB2249254812F073FB8421204812F021
:1022F40066FB1E480BF0F2FEFFF798FE1B480BF03E
:10230400D7FE68B94FF49973194A1D491A4812F057
:102314005FFB16491B4812F05BFB4FF49971E5E72C
:1023240084F31188BFF36F8F02B010BD164B1B6886
:10233400002BF9D050B9002200231448CDE9002322
:102344004FF4004200230CF025FAEDE70928EBD105
:102354000E480CF08DFA0E4802B0BDE8104009F0AA
:1023640087BD00BFD41100204D2A0020C8110020D1
:102374006B7B0100987B01007E780100AD7B01003E
:10238400C37B0100DA7B0100CC110020700A00201D
:10239400A004002010B5064B04461B68984721464C
:1023A400A0600448FEF7EAFFBDE81040FFF780BFD5
:1023B4000400002018030020044A054B9B1AB1EBCB
:1023C400D30F34BF52F8310000207047546E01001F
:1023D400DC6E01002DE9F04F8FB0C1F34A2604AF43
:1023E4000D469046B8607B600C0D002E66D04FF011
:1023F40000090A234FF0040B07F1140AFE60C7E931
:102404000799C7F824900093CDF808B0CDF804A03C
:1024140007F11C034A464046F968FEF73DFCB0F557
:10242400006F03461CD36C468AB0D8F8041004AB82
:102434002B481A46C3E9050140F2FF71D9614FF4F4
:1024440000711984274B42F8103F4FF412514B4648
:102454002548FFF7BFFFA5462C37BD46BDE8F08FE2
:10246400C0F30A0604F11700184420F0070080089E
:102474003B60FFF7BFFD66F35325044630B33B686A
:1024840000F11001C7E908390A23F961CDE901AB6C
:1024940000934046154AF96807F11C03FEF7FCFB5C
:1024A400002813DA1249134840F24913124A12F071
:1024B4008FFA40F24911104812F081FA04F1170022
:1024C40020F007008008FFF795FD044666F35325C6
:1024D4002A4620467B68B96812F041FCBCE700BF7D
:1024E400E37D0100040000016C6E0100354D010024
:1024F4004E7E01007E780100227E0100406820B1FA
:10250400034BC01A40F3CF0070474FF0FF307047C1
:10251400546E01000EB403B503AB53F8042B01460B
:102524000448019301F050FB02B05DF804EB03B0E2
:10253400704700BF59250000CA0605D48B064CBF5E
:1025440002490349FFF7E6BF704700BFC48E01008C
:10255400577E010038B54B6805461A68CB680C46AF
:102564009A4202D1084612F077FC6368D3E8EF2F51
:10257400511CC3E8E01F0028F8D1A3689D54636888
:102584001A68E3689A4209D9054906487223064A3B
:1025940012F01EFA7221044812F011FA002038BD1C
:1025A400897E01007E7801005A7E01002DE9F04FFA
:1025B40089B099469DF85080159B044606930D46B4
:1025C400DDE916A3189F05920493B8F1000F00F0FB
:1025D400A180B8F1040F0BD988494FF41573884AC8
:1025E400884812F0F5F94FF41571854812F0E7F9AF
:1025F40007F48073079312F090FB07F0020B024676
:10260400002856D020468049FFF784FF0646BBF1D8
:10261400000F08D017F0440F4DD12A4620467B49BD
:10262400FFF778FF064407F0010353B1784B2046C7
:1026340053F82820774B7849002A08BF1A46FFF739
:1026440069FF07F48073002B07F0080318BF4FF0ED
:102654000009002B5BD0714B204653F828207049A9
:10266400FFF758FF0546059B2BB11A4620466D49D6
:10267400FFF750FF0544B9F1000F05D04A46204644
:102684006949FFF747FF054468483544069B002B1A
:1026940047D02246664912F035F9002841DA6549E7
:1026A40040F2B123564A574812F092F940F2B12150
:1026B4009BE70646ABE7604B18680028B2D05F4B37
:1026C4004FF47A7B1B684FF03C0CB5FBF3F5B5FB7C
:1026D400F0F14FF4616300FB11550BFB05F5B1FB01
:1026E400F3F2B5FBF0FE03FB121100FB1E55B1FB28
:1026F400FCF30BFB05F5B5FBF0F50CFB13112046C1
:102704000091CDE901E54E49FFF704FF8AE707F0A0
:102714000805A8E7B9F1010F45460CBF43484948ED
:10272400B4E7049B002B54D0DDF810903946B9F17E
:10273400100F204628BF4FF010090026FFF7FCFEBB
:10274400B54218DC0026334620461AF803203E49D9
:10275400FFF7E0FE0136102E13D0710703D1204697
:102764003A49FFF7D7FE4E453346EDD32046384964
:10277400FFF7D0FEEEE720463449FFF7CBFE0136E3
:10278400DEE7002620463349FFF7C4FE33461AF835
:1027940003202046A2F120035F2B28BF2E222E49BE
:1027A400FFF7B8FE0136102E0DD0720703D1204674
:1027B4002649FFF7AFFE4E453346E8D3204623496A
:1027C400FFF7A8FEEEE7049BCA44B3EB09030493A6
:1027D400AAD1B8F1000F0AD0FB0704D520460D4A50
:1027E4000D49FFF797FE39462046FFF7A5FE204620
:1027F40009B0BDE8F04F12F02FBB00BFBE7E010050
:102804005A7E01007E780100C97E0100CD7E010060
:102814006C6F0100B97E010032770100806F010006
:10282400F27E0100F87E0100FC7E010059250000C3
:10283400CD3B0000017F0100E0110020DC110020ED
:10284400D67E0100774E01000A7F0100127F01004D
:10285400107F0100147F0100167F010042F20F7304
:1028640073B58B4228BF0B460568044605216846AC
:102874000D4A11F065FC0646636828460B225B6826
:102884000A4912F0DBFA63683246694628465B68F7
:1028940012F0D4FA63681B2228465B68044912F0DC
:1028A400CDFA02B070BD00BF50C001007FCF01005F
:1028B40063CF010000210123064A904206D8064A4C
:1028C40001B901231360054B1860704701214008CA
:1028D4005B00F2E740420F00DC110020E011002011
:1028E400F8B50D460446064F4618B44201D12846B1
:1028F400F8BD14F8011BBB6801485B689847F4E70E
:10290400986B010010B543681C68094813F0F1FB8B
:1029140048B9084908489923084A12F059F89921F6
:10292400064812F04CF823685B685C6010BD00BF79
:10293400986B0100777F01007E780100397F0100E8
:10294400014B036000207047C86F010008B50448BC
:1029540012F028F8034812F025F8002008BD00BF43
:10296400AB7F0100E07F0100F0B5054689B000AF00
:1029740020220021384613F0F0FF3B4648F6D2727D
:1029840028461B490CF03CFC04460646C0B16D4683
:1029940088B06A46174B0593174B06934FF40073A0
:1029A400ADF81C30154B42F8103F00234FF4E251B0
:1029B4001348FFF70FFDAD4620462437BD46F0BD52
:1029C400394628460CF0D2FC04460028F4D06D4663
:1029D40088B06A460B4B0593074B06934FF400737C
:1029E400ADF81C30054B42F8103F3346DEE700BF1C
:1029F4009CCF01000D8001008BCF0100030000017A
:102A0400CC6E01002F80010001480FF053BC00BFC1
:102A1400C86F010038B5044618B90F4B0F485B68FE
:102A240098476168B1F5683F10D0B1F5680F0DD0D3
:102A34000B4DA9420AD011F46861206807D0014601
:102A4400084808F031FC00232360656038BD142277
:102A540013F083FFF9E700BF7C02002050800100DF
:102A64002C5F5CA91017002008B560B34368B3F568
:102A7400683F0ED0B3F5680F18D0144A934220D0A3
:102A840000684FF0FF324FF0FF3308F0E3FE58B117
:102A940015E001220368D3E8EF1F002903D1C3E83E
:102AA400E02F0028F7D10AD1002008BD0368084AA6
:102AB4001B7803F5807352F82330002BF4D00548BB
:102AC400F3E70548F1E76FF4E040EEE72C5F5CA91B
:102AD40000000350E98FFFFFEA8FFFFF08B520B322
:102AE4004368B3F5683F09D0B3F5680F13D0114AB2
:102AF40093421DD0006808F075FF14E000220368BB
:102B0400D3E8EF1F012903D1C3E8E02F0028F7D150
:102B140009D0094808BD00210368084A1B7803F559
:102B2400807342F823100020F4E76FF4E040F1E7EB
:102B34000348EFE72C5F5CA9E98FFFFF0000035017
:102B4400EA8FFFFF10B5044618B91D4B1D485B689A
:102B540098476368B3F5683F2FD0B3F5680F2CD05E
:102B6400194A934219D1236803BB4FF0FF324FF047
:102B7400FF332146154808F00BFB08B923681BB93D
:102B84000F4B13485B68984714220021206813F008
:102B9400E4FE4FF46863636008E0B3F5680F0DD892
:102BA4003A2B03D040F6BA629342DED1206813F088
:102BB400FCFA636843F03A03636010BD054AF3E727
:102BC4007C020020508001002C5F5CA910170020BB
:102BD400768001003A00003A08B5064940231422E1
:102BE400054813F0C5FABDE80840044904480FF04D
:102BF400F1BD00BF1012002010170020D06F01009B
:102C0400E46F010008B50348034A0021121A12F0C8
:102C1400A8F908BDD0050020A02C0020074808B55D
:102C2400074A0849121A12F09EF9BDE808400648FE
:102C3400064A0749121A12F096B900BF0000002094
:102C4400D0050020E46B02000000002000000020FA
:102C5400E46B02002DE9F04706460C4600AF00295C
:102C640036D0D1E90012E9468AB06D46A3684FF028
:102C7400050AE8461F48CDE90723CDE9050148F8D0
:102C840010AF002342464FF421511B48FFF7A2FB2B
:102C9400D4E90312CD466369AD461848C5E9072354
:102CA400C5E90501C5F810A0002342464FF421519F
:102CB4001148FFF78FFBCD46E3690121104A0E4806
:102CC40012F0A6F8A36901210E4A0B4812F0A0F8ED
:102CD400012E07D1EFF305830B4A31460648103B1A
:102CE40012F096F82146304607F0D8FEBD46BDE8FE
:102CF400F08700BFA38001009C6E0100D280010018
:102D040001810100108101003E810100034601465A
:102D1400024A53F8200B1360FFF79CBF34170020BE
:102D240030BFFFF7FDBF00BF2DE9F04105460B4E54
:102D3400DFF82C80324606EB0807CC1B20460949F5
:102D440013F0E5FDA01942460021083C13F005FEEE
:102D54006C6707F10800BDE8F08100BF00000000C7
:102D640004000000EC6E010010B5244C24492548F1
:102D740012F002F9A36A99013ED52248224912F0C1
:102D8400FBF81E20A36ADA0104D51E481F4912F07D
:102D9400F3F81F20194CA36ADB0204D519481C4917
:102DA40012F0EAF80220A36A1C0304D51548194955
:102DB40012F0E2F82120114CA36A590304D51148FA
:102DC400154912F0D9F82220A36A9A0304D50D48B4
:102DD400124912F0D1F82320084CA36ADB0304D56E
:102DE40008480F4912F0C8F82420A36A6FEA034385
:102DF4006FEA1343A36210BD1D20C3E700ED00E09A
:102E0400518101009C6E0100698101007C810100F7
:102E140096810100C0810100DE810100038201006E
:102E24001D82010070B506460D46334C33493448C3
:102E340012F0A2F8A36AD9064DD53148314912F0EF
:102E44009BF81120A36A1A0704D52D482E4912F0C5
:102E540093F81220284CA36A9B0712D52B492848C3
:102E640012F08AF8636BA26A110609D50121284A77
:102E7400234811F0CDFF1EB1A36A23F08003A3629F
:102E840013201D4CA36ADA0704D51D48214912F00A
:102E940073F81420A36A9B0604D519481E4912F03E
:102EA4006BF81520144B9A6AD60602D49A6A9407D2
:102EB40013D59B6AD90610D5184940F22D13184A28
:102EC400184811F085FD184811F082FD40F22D11CB
:102ED400134811F074FD1020B4E7074B9A6A920668
:102EE40042BF5A6A22F400525A629A6A42F0FF02BE
:102EF4009A6200232B7070BD00ED00E0488201004F
:102F04009C6E01005E82010091820100A482010096
:102F1400BC820100D2820100F182010052830100CF
:102F2400208301007E7801009C83010070B5064671
:102F34000D46284C2849294812F01EF8A36AD904E2
:102F44003CD52648264912F017F81720A36A1A051B
:102F540004D52248234912F00FF818201D4CA36A07
:102F64009B0512D51D48204912F006F8A36BA26AEE
:102F7400100409D501211D4A184811F049FF1EB15A
:102F8400A36A23F40043A3621920124CA36A5905CF
:102F940004D51248164911F0EFFF1A20A36ADA0586
:102FA4000ED50E48134911F0E7FF1B20094A936A16
:102FB40043F47F43936200232B7070BD1620C5E752
:102FC400A36A9B04F2D505480B4911F0D5FF1C20D8
:102FD400ECE700BF00ED00E0008401009C6E0100FE
:102FE40016840100918201002784010040840100BD
:102FF4005584010070840100F18201002DE9F04143
:103004008AB0804B04465868002500AFC0F308031B
:1030140085F31188BFF36F8F02F07F46B6F17F4FBF
:1030240007D102F00C06082E12D17749774811F027
:10303400A3FF774940F21B43764A774811F0C8FC56
:10304400764811F0C5FC40F21B41724811F0B7FC00
:1030540016074CBF0C460125002CEAD0704A04F137
:10306400200616600022FA71DA1E092A00F2A980ED
:10307400DFE802F0059FA282A7A7A7A7A7A5694931
:10308400624811F079FF0023DFF87881FB71D8F8EA
:103094002C309A0705D564495C4811F06DFF002374
:1030A40033E0D8F82C30002B01DA6049F4E7D8F883
:1030B4002C305B0070D55E49544811F05DFFD8F8A0
:1030C4001430A26943F48073C8F81430BFF34F8FEF
:1030D400BFF36F8F32F8023CD8F8142022F48072C8
:1030E400C8F81420BFF34F8FBFF36F8F03F47F42F0
:1030F400B2F55F4F29D1DBB2022B26D1236801211F
:103104004C4A424811F084FE2368FA79CAB907F19F
:10311400080C624620686168083403C2B4429446CD
:10312400F7D17A6A002D69D0C2F3080121B96FEA98
:1031340052226FEA42227A62184607F10801FFF729
:1031440089FD2837BD46BDE8F0812E4B9A6AD2B27C
:103154002AB10120F91DFFF765FE0346D5E79A6AF7
:1031640012F47F4F04D00120F91DFFF7DFFEF4E7CE
:103174009B6AB3F5803F02D3FFF7F6FDEDE72E49D6
:1031840040F2ED23234A244811F022FC2B4811F08D
:103194001FFC40F2ED2158E727494FF43C731D4AC8
:1031A4001D4811F015FC264811F012FC4FF43C7137
:1031B4004BE70020F91DCEE70020F91DD5E7214992
:1031C4006AE7214AE84610F4F87F8AB01F4918BF1D
:1031D40011466A46103B07934FF400731C48ADF840
:1031E40020301C4BCDE9050142F8103F00234FF479
:1031F40011510648FFF7EEF8C54650E76FF3080291
:1032040099E700BF00ED00E0B68401009C6E010068
:10321400E1840100208301007E780100F484010030
:103224003417002032850100498501006A850100B8
:1032340078850100978501003DA40100B385010054
:10324400D7850100078601009D8401008884010060
:103254002B86010004000001064B5A6942F010025B
:103264005A615A6942F480625A615A6922F008022A
:103274005A61704700ED00E0EFF30880EFF3098135
:1032840001B57246FFF7BAFE01BD00BF002080F30E
:103294001488BFF36F8F002080F30A8880F30B88B3
:1032A400124880F3088805F02BFF002010490860BD
:1032B400BFF34F8F00F032F8202080F311880D48BF
:1032C4004FF0AA014FF4006211F04BFE09484FF48D
:1032D4000061401880F30988EFF314800221084349
:1032E40080F31488BFF36F8F00F0C0F890F70020CC
:1032F40094ED00E000DA0020002318460649D1F8D6
:103304009020C2F30722934200DB7047C1F8983043
:10331400C1F8A0000133F6E700ED00E010B572B685
:10332400002484F31388FFF7E7FF23464FF0FF30B0
:103334000C4A03F120010133102B42F82100F8D18B
:1033440000234FF0FF30074A03F160010133102BD3
:1033540042F82100F8D162B6BFF34F8FBFF36F8FED
:1033640010BD00BF00E100E01EF0040F0CBFEFF33E
:103374000880EFF30980816911F8021C0229FFD04B
:1033840001B57246FFF7C2FC01BD00BF40B2002880
:1033940007DB01234109034A00F01F00834042F880
:1033A4002130704700E100E040B200280CDB01222C
:1033B4000649430900F01F008240203341F82320CE
:1033C400BFF34F8FBFF36F8F704700BF00E100E082
:1033D400054B420953F82220012300F01F0003FA91
:1033E40000F01040704700BF00E100E038B54B1C0E
:1033F400072B04460D460FD96B23104A1049114878
:1034040011F0E6FA294610480723224611F0E0FAA3
:103414006B210A4811F0D3FA40B20028ACBF00F186
:1034240060400A4A4FEA4313DBB2ABBF00F5614088
:1034340000F00F0080F80033135438BD3E860100BD
:10344400758601007E7801009086010014ED00E08D
:10345400044B054A23F07F039360BFF34F8FBFF300
:103464006F8F70470000000000ED00E008B5FFF723
:10347400EFFF074AD2F8883023F47003C2F888308B
:10348400FFF7C0FBFFF7CAFB00F09CF807F07EFCD7
:1034940000ED00E042F8203C009B0B4942F81C3C44
:1034A400019B21F0010142F8183C029B42F8081CE0
:1034B40042F8143C4FF0807342F8043C0023203A55
:1034C40002658367704700BF2911000000B50D4BEA
:1034D40015469860426F0C4B0E461A60436E83F398
:1034E4000B882C4686F309880020044B9847204615
:1034F400002100220023024C204700009B4F0100C2
:103504002911000078260020301700201022014BDA
:103514001A61704700ED00E0054B5A699B689A42B6
:103524001FBF044A536843F08053536009F03ABB09
:103534007826002000ED00E0084B9B6883420BD105
:10354400EFF3058343B1064B5A6842F080525A6048
:103554005A6A22F400425A620AF024BB78260020F8
:1035640000ED00E014498A684FF030001044EFF396
:10357400098C80E8F01F202080F31288BFF36F8F3E
:103584000E4F4FF000664A698A603E60506F0C4CE3
:103594002060906F0023936780F3118802F130005C
:1035A40090E8F01F8CF3098802F1000004B511F0D3
:1035B400EBFCBDE8044070477826002004ED00E0F1
:1035C40030170020002320210348C2180133452B63
:1035D40082F80013F9D1704700E100E008B5EFF379
:1035E4000583064A103B02EBC30152F833004968D5
:1035F4008847BDE80840FFF78FBF00BFD06B0100CC
:1036040073B50546144B18681B7900908DF8043087
:1036140005B3124C4C220021204613F09EF92B686E
:10362400052123606B6868466360AB68A360EB6840
:10363400E3602B6923616B696361AB69A361EB6927
:10364400E361074B1B68236200F02AFE4C212046ED
:1036540000F026FE02B070BD386F01004F2A002032
:1036640034170020034B9B68834206BF024B186843
:10367400006D704778260020341700200148006848
:1036840070470000301700201FB50121094B0A4A7A
:103694000A4800F00FF90023064A0393084B01215E
:1036A400019301A8D31A029300F028F905B05DF83C
:1036B40004FB00BF0000072000000020F46F01009D
:1036C400D00500200A7A0B6810B562F304031C4687
:1036D400CB68520923F01F0343EA4203044A43F030
:1036E4000103C2F89800C2F89C40C2F8A03010BD93
:1036F40000ED00E010B50A4BD3F89030C3F3072374
:10370400013B984208D901210346064A064811F0B4
:103714007FFB6FF0150010BDFFF7D4FFFBE700BF80
:1037240000ED00E0D4860100846E01002DE9F04F25
:103734008946144606464FF000084F4D85B0C845EB
:1037440027DAD6F804A0BAF1000F44D0BAF11F0F5B
:1037540017D91AF01F0F14D1D6F800B01BF01F0FA1
:103764000FD1584611F055FC07460AEB0B000138FF
:1037740011F04FFC874210D06FF015073F4A3B46CB
:1037840001E043463E4A01213E4811F041FB6FF0FF
:103794001504204605B0BDE8F08F17F1160FEDD0E3
:1037A400BC42EBDDC5F89870D5F89C10C5F898704C
:1037B400D5F8A03021F01F0143F01F0BD6E90032E9
:1037C4001A44994202F1FF3A1AD1D34507D131463E
:1037D400F8B211F027FC08F101080C36AFE73146C6
:1037E400C5F89870D5F89C30E0B263F30402C5F8CC
:1037F4009C2011F017FC10F1160FC8D0441CEAE706
:10380400C5F89870D5F8A020013B23F01F0302F0FF
:103814001F021343D3453146E0B2C5F8A030E8D0C7
:1038240011F000FC10F1160FB1D0C5F89870D5F85E
:103834009C209DF808300BF1FF3B62F304038DF8E4
:103844000830D5F8A0309DF808205B0863F34712D0
:103854008DF80820D6E900321344009323F01F03A7
:103864005B44A3EB0A03013023F01F036946C0B293
:103874000393FFF73FFFBEE700ED00E02087010060
:10388400FA860100846E01000522044BC3F89420DB
:10389400BFF34F8FBFF36F8F704700BF00ED00E0A1
:1038A400BFF35F8F0022024BC3F89420704700BF20
:1038B40000ED00E038B50C4D0C462A78FFF736FFD2
:1038C400287016300FD140F28913084A0849094874
:1038D40011F07EF82146084811F07AF840F2891177
:1038E400024811F06CF838BD9B2A00204387010080
:1038F4003DA401007E780100728701002DE9F74F95
:10390400314D894606464FF00008AB462F4FC84557
:1039140002DB03B0BDE8F08FD6F804A0BAF1000FC3
:103924004CD031680846019111F073FB01990446AB
:103934000AEB0100013811F06CFB84424FF01402D1
:10394400234B15D002FB08F36FF015024BF803204C
:1039540040F299131F4A2049204811F039F849468A
:103964001F4811F035F840F299111A4811F027F860
:1039740014F1160F2C60EBD01978A142E8DD02FB9C
:1039840008B0C7F89840C7F89840D7F89C4000F1B1
:103994000801007B64F304000871D7F8A0000C79D7
:1039A400400860F347140C71D7F89C1021F01F01F4
:1039B4006960D7F8A01021F01F01296108F10108FE
:1039C40014350C36A3E700BF3817002000ED00E0E3
:1039D4009B2A0020438701003DA401007E7801005A
:1039E4009E8701002DE9F0416B4D6C4ED5F8903067
:1039F4003468C3F307239C4286B013D940F20223F0
:103A0400674A6849684810F0E3FFD5F890202146DA
:103A14006648C2F3072210F0DBFF40F2022160483F
:103A240010F0CDFF0020FFF73BFF614BC5F8C0301D
:103A340084421BD15F4D01A82C70FEF781FF002644
:103A440007464FF061085C4CB74216D100202B7832
:103A54005149D1F89020C2F307229342C0F29580D5
:103A64000020FFF711FF06B0BDE8F081716801EB9B
:103A74000011FFF727FE0130DAE7019A300102EB6B
:103A84000613D3F80CC00CEA0401B1F1807F57D0BF
:103A94000AD8B1F5001F29D0B1F5800F43D0B1F594
:103AA400801F14D00136CFE7B1F1006F48D0B1F1D7
:103AB400805FF7D159689B681258013B21F01F00C1
:103AC4000344CDE9021223F01F0301220BE05968DD
:103AD40012589B68CDE902122122013B21F01F00FC
:103AE400034423F01F038DF8102036E05968125860
:103AF4009B68CDE902124122013B21F01F000344DF
:103B040023F01F031CF0010F8DF81020059325D01E
:103B14002A498423224A244810F05AFF284810F0E6
:103B240057FF84217BE759689B681258013B21F0B9
:103B34001F000344CDE9021223F01F030622D2E73B
:103B4400596812589B6821F01F00013BCDE902120D
:103B5400034423F01F038DF810800593287802A9ED
:103B6400FFF7C8FD00280CDA0E4940F235230C4A51
:103B74000D4810F02DFF134810F02AFF40F23521B4
:103B84004DE72B7801332B708CE7C1F89830C1F8DE
:103B9400A00001335DE700BF00ED00E0007001000C
:103BA400438701003DA401007E780100CD87010018
:103BB400AAFF44009B2A00200000F0FF01880100B6
:103BC4002788010056880100F0B587B007460E46E5
:103BD40014460021102268461D4612F0BEFE022340
:103BE4008DF80230054B2A4621466846CDE9047615
:103BF400019310F0CFFA07B0F0BD00BF5B50010095
:103C040008B5024B1B689847002008BD4C170020DC
:103C1400034B044A1860937843F00203937070478F
:103C24004C1700203000002008B50649064821F052
:103C34000701C1F1005202F5E022FCF79BFF0020CE
:103C440008BD00BF1F13012050170020827A3420C2
:103C5400074B00FB0233DB6A0846DB68032B94BF87
:103C64006FF003035B42CA5C0132CA54704700BF61
:103C7400D004002010B40C463421827A0A4B01FB94
:103C84000233DB6A5868DB68032B94BF6FF00303CD
:103C94005B42E25CE118013AD2B2E25412B910BCC0
:103CA40007F0F8B910BC7047D0040020F7B5867A45
:103CB40034208E46164D944600FB0650C46AE168D3
:103CC4006068DEF8004079B9211D07F0AFF968B1EA
:103CD40001230370342303FB0655EB6ADB68042BD2
:103CE4002CBFC018043002E0A14202D9002003B066
:103CF400F0BD013C0C4404290A46B4FBF1F438BF7E
:103D04000422CDE900C301FB042207F09DF9DEE79C
:103D1400D004002070B541690446867A0A4D59B131
:103D2400437ADB0706D4342303FB0653DB6A1B68A0
:103D34009B689847002363613420214600FB0650AA
:103D4400BDE8704012F044BAD004002008B54368BE
:103D54004BB1074907485A23074A10F039FE5A2144
:103D6400054810F02CFE03824369C36008BD00BF00
:103D7400B48801007E7801008F8801002DE9FF4797
:103D84000546684617461C46039112F02CFBDDE9F4
:103D9400008955B95D4940F201135D4A5D4810F050
:103DA40017FE40F201115A4818E005F11C06EFF322
:103DB400118A202383F31288BFF36F8F30460AF0F1
:103DC40069F968B98423544A5449524810F000FEF2
:103DD4003146534810F0FCFD84214F4810F0EFFDAC
:103DE40030460AF07BF96B8C002B5CD02A8C9A420B
:103DF40039D900220023284607F0AEFF04460028E4
:103E040031D030460AF054F968B94FF49973424AF4
:103E14004449404810F0DCFD3146434810F0D8FDD9
:103E24004FF49971D9E78AF31188BFF36F8F039D1B
:103E3400002D5BD042464B46684612F0F9FA342115
:103E4400A27A3A4B204601FB0233DB6A03A91B68C2
:103E54001E68DDE90023B0476061002839D120469F
:103E6400FFF758FF30E06C8C3046631E6B840AF019
:103E74001FF90028C9D08AF31188BFF36F8F95F812
:103E840024302A8C1B33121B2C6B23F0030302FBFC
:103E94000344264B264AEB1A9B105343A37295F80E
:103EA4002430E372C3E730460AF002F90028ACD0AC
:103EB4008AF31188BFF36F8F23463A46284607F0EA
:103EC4004BFF04460028B2D10024204604B0BDE8CC
:103ED400F087039B9D420BD916494FF4AB730C4AF0
:103EE4000C4810F075FD4FF4AB715CE72B4665612F
:103EF40000210122616022816382E27A04F11800C8
:103F040012F02BFD2046FFF721FFDEE7CE880100EB
:103F14008F8801007E7801006B7B0100987B010093
:103F2400AD7B0100C37B0100DA7B0100D0040020DB
:103F3400C54EECC4D3880100F8B5054698B13427C2
:103F4400184E2C46237A6D68CBB940F2C113164A39
:103F54001649174810F03CFD2146164810F038FD6C
:103F640040F2C11108E0144940F2BB130E4A104854
:103F740010F02EFD40F2BB110B4810F020FD013B68
:103F8400DBB2237253B9E3606360A37A204607FB74
:103F940003639B6A1BB19847002DD2D1F8BDFFF78C
:103FA400B9FEF9E7D00400208F880100E4880100FD
:103FB4007E780100ED8801000689010008B50346FA
:103FC40058B90849084840F23123084A10F000FD66
:103FD40040F23121054810F0F2FC18465B68002BD2
:103FE400FBD108BD068901007E7801008F8801009D
:103FF400034670B505688288DC889E68A818A41AF0
:10400400AD1B641BA14209D9064907483E23074A50
:1040140010F0DEFC3E21054810F0D1FC0A449A80E1
:1040240070BD00BF458901007E7801000A89010046
:1040340008B5828803468A420BD20949094840F2EE
:10404400C313094A10F0C4FC40F2C311064810F02F
:10405400B6FC521A828000680844186008BD00BF8C
:10406400698901007E7801000A890100052370B581
:10407400144D154E2C780134B4FBF3F303EB830396
:10408400E41A11F068FB114A137823B156F824306E
:10409400C01A072814D94FF05023D3F8141141B192
:1040A4000021C3F81411D3F814312C700CB9012376
:1040B40013702C7811F04FFB46F82400012070BDDA
:1040C4000020FCE79D2A00205C1700209C2A002089
:1040D400054B03EB8000D0F8003223F0E04343F0BB
:1040E4004053C0F80032704700258450012208B5BF
:1040F400114B1249C3F8002502230020C1F8D03621
:10410400FFF7E6FF1046FFF7E3FFC1F80427C1F805
:104114000429C1F8002B00F0A1F858B10849094856
:1041240040F23D23084A10F053FC40F23D2106487A
:1041340010F045FC08BD00BF0010005000400050C6
:10414400627B01007E7801008889010007B50022A6
:10415400134B1449C3F8A821C3F8AC204FF4806270
:10416400C3F8B8254FF400620F48C3F83C250DF19D
:10417400070211F00AFE00280BDA0C490C4840F241
:1041840047230C4A10F024FC40F24721094810F060
:1041940016FC9DF8070005F0B1F803B05DF804FBC8
:1041A40000A002502CA0025028A10250627B010002
:1041B4007E7801008889010048B1054B054A1B68D7
:1041C400B3FBF2F35843044B43F001031847704721
:1041D4001002002040420F00406F0100002170B522
:1041E400184C194D000714F8013B5E0914D0012E38
:1041F40006D14FF6FF7203F01F03DA40D2070ED444
:10420400124913484FF48263124A10F0E1FB4FF451
:104214008261104810F0D3FB4FF0FF32EBE70E4AF7
:104224000131012E18BF2A4602EB8302D2F8003274
:10423400042923F0E04343EA0003C2F80032D2D158
:1042440070BD00BF6E5F020000258450E989010043
:104254007E780100B6890100002884500149024893
:1042640010F013BD347001007017002008B54FF032
:10427400FF33044A13603F231046536005F018F8D7
:10428400002008BD90170020014B1B68184700BF91
:10429400D0000020014B5B68184700BFD00000200D
:1042A40018B111B1014B9B6818477047D00000202A
:1042B40030B5044685B0C0B1884216D24D238DF87E
:1042C400043001238DF8053000238DF80630084BA7
:1042D4000D1ACDF80700CDF80B1001A80B219B682F
:1042E400984729462046FFF7DBFF05B030BD00BFE5
:1042F400D00000207FB50D4606461446FFF7C4FFE4
:1043040044F25A53ADF804300223ADF806304FF4AA
:10431400A0230396029310F07AFE124BADF8080026
:104324000C219B6801A8984715B12846FFF768F946
:104334009CB1204604F18001FFF7BAFFD4E9195675
:104344002046FFF78FF985422E4402D8864228BFC3
:10435400054631462846FFF7ABFF04B0BDE8704080
:10436400FFF798BFD000002010B9034B18687047BE
:104374006FF08500704700BF9817002010B9034BF9
:10438400186070476FF08500704700BF98170020D1
:104394002DE9F0470E46044600AF00B121B96FF095
:1043A40015020026214B1A60DFF88480DFF8849020
:1043B4006EB10025207808EB0501000910F016FC09
:1043C4000028A24606DA6FF01502184B1A60BD46A3
:1043D400BDE8F0879AF80000691C58FA81F100F0F2
:1043E4000F0010F003FC002804F10104EBDB02359C
:1043F400EDB2402D06F1FF3601D0002EDAD10023B4
:1044040008F805306D4688B06A464FF40071ADF87F
:104414001C100949CDE9059842F8101F4FF4E251E8
:104424000648FDF7D7FFAD46C2E700BF9817002046
:104434009E2A00200C8A010003000001646E010022
:10444400002208B5074B1A60FDF7F0FD0028FBD1E8
:10445400FDF764FEBDE808400121034A034810F05B
:10446400CEBC00BF98170020138A0100646E0100BF
:1044740008B5074B1B6823B10121064A064810F012
:10448400BEFCBDE808400121044A034810F0B7BC53
:10449400981700201E8A0100646E0100358A01000D
:1044A4002DE9F047074610F038FEB1F830A0D0F8F7
:1044B40008800C469AFA9AF9B8F1000F66D0D8F839
:1044C4001C30002B65D0BAF1000F62D091F829306E
:1044D4004BB9314B1A68C1F829209A889B79A1F805
:1044E4002D2081F82F3040F6CD4200230E212046A6
:1044F40000F080FD064620B96FF00B052846BDE8A4
:10450400F0870E2150F80C5FFFF772FD40F60603AA
:104514009A4531D094F83330C3F30213022B2BD1D4
:10452400A368DB681B7EFF2B26D11C4B1B882B80CA
:10453400A368DB685B6AC5F80230D4F822303146E0
:10454400C5F80630E38C20466B81A5F80C9010F07A
:10455400FEFF204611F005F8384610F0DEFD214636
:10456400D8F81C30984705460028C7D1A3684BB932
:10457400204610F0CCFFC1E7D4F82A302B60E38D3D
:10458400AB80DAE71A8A5B681544F0E76FF001053F
:10459400B4E76FF08505B1E7478A0100725F020056
:1045A4002DE9F843D1F808800546D8F80C300C46BC
:1045B40013B90220BDE8F883B8F810200D2AF8D901
:1045C400D3F806200320C1F822205A8981F820005C
:1045D400CA84062281F821201E682A31C4F82A6080
:1045E4009E8884F82800E68584F829209B8908465B
:1045F4009EB25BBA23869FB210F0B7FD81467DB3AD
:104604002B684BB15A7C062A2AD103F1120012F00E
:10461400ACF9B0FA80F35B09B9F1000F05D194F855
:104624002A20D20701D4002BC3D00E2108F10C009C
:10463400FFF7FEFCA368ABB92A4B2B4A2B499342E4
:1046440037D92B4940F27D132A4A2B4810F0C0F980
:104654002A4810F0BDF940F27D11264810F0AFF958
:104664000023D9E75B68E6E7224639462846C04777
:1046740000289FD002289CD048F688639E4299D097
:1046840094F83330C3F30213012B21D1A368DB6800
:104694005B885BBA9BB22D2B8CD8A268002A89D088
:1046A400118A994235BF5B1A13829BB20023526868
:1046B400F4E7BFF47EAF9889B84207D158688842BE
:1046C40004D1D3F80880B8F1000FCDD11033B6E788
:1046D400022B7FF46FAFA368DB689B885BBA283337
:1046E400D8E700BF446E0100546E0100A805002005
:1046F400848A01004F8A01007E7801009B7D0100BD
:1047040038B50123054610F003FD0A490376044633
:104714004561043007F094FE284610F003FD43057C
:1047240042BF237E43F004032376637E43F00203F7
:10473400637638BDE75101002DE9F04707468A4604
:104744001C4690468CB0002A00F00F811368002BA1
:1047540000F00B811E683022D6F8089000216846CC
:104764006D4612F0FAF8B9F1000F00F0FB80D9F8A9
:10477400103023B96FF085000CB0BDE8F08714B990
:104784006FF01500F8E7149B302BF9D1784B013FFB
:104794004AEB030A102F7AF1000AF1D20F2FEFD857
:1047A40001A353F827F000BFED4700001F480000A5
:1047B40059480000A5480000CD480000FB4800000F
:1047C40085470000854700008547000085470000B5
:1047D4008547000085470000154900003349000063
:1047E400854700004D4900000021404610F03CFD83
:1047F400002875D12068A3880090ADF804306A467B
:104804003046D9F8103098470028B5DB0323062238
:104814002146404610F0E4FDAEE74FF40071304607
:1048240010F014FD0028A5D023797BB1023B012BA5
:10483400A6D92B462068616803C30121A0681860CB
:104844002A463046D9F81030984795E7A368642B78
:10485400EFD995E74FF40031304610F0F7FC00280B
:1048640088D06379012B8BD02379032B0BD1414B57
:10487400226A9A4284D8D4E904128B424FF000038E
:104884009341FFF47DAF2A4604F1300713462068B4
:104894006168083403C3BC421A46F7D10221CFE74A
:1048A4004FF48021304610F0D1FC00283FF462AF71
:1048B4002379042B3FF464AF6B462068616803C31B
:1048C400A06803211860BBE74FF40021304610F0C4
:1048D400BDFC00283FF44EAF404610F0CFFC10B1B1
:1048E4006FF00C0048E76B462068616803C3A0685A
:1048F40004211860A4E74FF48061304610F0A6FC50
:1049040000283FF437AF237805218DF8003097E76E
:10491400404610F0B3FC0028E2D12068A288A379B5
:1049240009210090ADF804208DF8063088E74FF493
:104934008011304610F08AFC00283FF41BAF237826
:104944000A218DF800307BE74FF48051304610F097
:104954007DFC00283FF40EAF6B466168206803C3FA
:1049640007216DE76FF0010006E700239B68FFDE77
:10497400FFFF6FAFFFC99A3B002307B50246044906
:104984000120009300F0A0FC03B05DF804FB00BF1D
:10499400000090D0002307B502460449022000938A
:1049A40000F092FC03B05DF804FB00BF000090D05F
:1049B4001FB51346024640B153B9042302200093A5
:1049C400039103AB044900F07FFC05B05DF804FBE0
:1049D4002F2101200091F5E70000D0D016289ABFBE
:1049E400024B53F820000248704700BF407001009A
:1049F400A98A01002DE9F041104610F04EFC06464C
:104A0400104615461F4610F04DFC044660B103687D
:104A140053B1284610F058FC50B13946304623684B
:104A2400054ABDE8F04118476FF08500BDE8F08104
:104A34006FF07200FAE700BFB549000010B570B915
:104A44000B494FF443730B4A0B480FF0C1FF0B485B
:104A54000FF0BEFF4FF4437106480FF0B0FF4FF064
:104A6400FF32BDE810404FF0FF33183010F07DBC2A
:104A7400BD8E01008E8E01007E780100C38E010080
:104A840008B570B9094940F21333094A09480FF0CF
:104A94009FFF09480FF09CFF40F2133104480FF0C8
:104AA4008EFF1830BDE8084010F06DBCBD8E0100CB
:104AB4008E8E01007E780100C38E01002DE9F34142
:104AC4000368002104469E7F10F026FC002838D19C
:104AD40002252368002B6AD020469D77FFF7AEFF9E
:104AE400D4F8008011F07DFC4FF47A72A0FB02032D
:104AF40002FB0131C00B40EA4140C90BC8E908017F
:104B04002046FFF7BDFF236800279A7FAA424ED1B3
:104B1400062D41D1062E4AD0204610F0F5FB30BBBD
:104B24005B7C23BB234941F2CD63234A23480FF026
:104B34004FFF23480FF04CFF41F2CD611E480FF0A8
:104B44003EFF204610F0DBFB11F0D3FA68B10921D7
:104B5400204610F0E1FB0028BAD00A21204610F0CC
:104B6400DBFBC0F10605EDB2B3E70325B1E7204650
:104B7400082110F0DBFB0023224602200093114998
:104B840000F0A2FB204610F0BFFB80B9204602B023
:104B9400BDE8F04110F0EBBB062E08D120460821F9
:104BA40010F0D3FB3B46224601200097E7E702B012
:104BB400BDE8F081F08E0100C68E01007E78010010
:104BC400C38E0100000010D0054B064A934205D065
:104BD400054A1068002808BF18467047002070472F
:104BE400380500207C050020A817002037B50546AD
:104BF400FFF724FF0021284610F08EFB002839D14E
:104C0400284610F077FB044600B38468F4B12846C4
:104C140010F075FB70B91A4941F27873194A1A48B1
:104C24000FF0D6FE19480FF0D3FE41F27871154803
:104C34000FF0C5FE11F05DFAF8B1284610F05AFBEA
:104C44000121836828469847041E0DDB002128466D
:104C540010F06CFB002308202A460D49009300F055
:104C640033FB2846FFF72AFF2846FFF709FF2046B3
:104C740003B030BD6FF07704F6E76FF00504F3E797
:104C84002F950100C68E01007E780100C38E0100BD
:104C9400000010D037B50546FFF7D0FE00212846A6
:104CA40010F03AFBF0B1284610F024FB044628B17A
:104CB40084681CB12846A047041E0DDB0021284649
:104CC40010F043FB002304202A460849009300F017
:104CD400FBFA2846FFF7F2FE2846FFF7D1FE2046EE
:104CE40003B030BD6FF07704F6E700BF000010D0CA
:104CF40008B5024610F008FB034610465BB110F0FD
:104D0400FEFA83689B6823B19847032814BF0023E5
:104D14000123184608BD10F0EDFA06498142F8D186
:104D24002AB113681BB19B689B7E012BEEE700231D
:104D34009B7EFFDEA80500202DE9F8430C460546BE
:104D440088B381B30846FBF71DFA0F2806462DD811
:104D5400194FDFF8688000F10109474519D918494E
:104D640041F62913174A18480FF032FE17480FF07E
:104D74002FFE41F6291113480FF021FEAF4206D051
:104D84004A46214607F1080011F0EFFD88B1443787
:104D9400E3E7F3D32146721C05F1080011F0B7FDD7
:104DA4000020BDE8F8836FF01500FAE76FF05A00B1
:104DB400F7E76FF07700F4E7380500207C05002062
:104DC4002F8F0100C68E01007E7801009B7D0100BB
:104DD4002DE9FF47414C4FF0FF324FF0FF3340487D
:104DE40010F0C3FA0026A0463E4DDFF8FC903F4F7A
:104DF400AC4257D93E4941F697133E4A3E480FF01C
:104E0400E7FD3E480FF0E4FD41F6971139480FF0F5
:104E1400D6FD1022002104F1080011F09EFD204669
:104E240010F06DFAD0F808A0BAF1000F14D0DAF837
:104E340000308BB104F1180011F0B7F904F12C0023
:104E440011F0B3F9DAF800302046984794F840306E
:104E540023F0030384F84030237A83B92046FFF714
:104E640047FF78B1264A1368591C1160254A10215E
:104E740068460FF065F969462046FFF75DFF013685
:104E84004434B5E7204610F035FA814505D11E4A71
:104E94001368591C11601D4AE9E73B685A1C3A60C3
:104EA4001B4AE4E7B5D39EB14423A5EB0805B5FB43
:104EB400F3F5AE420CD0174941F6B9130D4A0E482A
:104EC4000FF086FD14480FF083FD41F6B9119DE7FC
:104ED400034804B0BDE8F04710F055BA3805002087
:104EE400F40300207C050020A80500209C17002066
:104EF400158F0100C68E01007E7801009B7D0100A4
:104F0400A41700204F8F0100A0170020568F010026
:104F14005C8F0100628F0100C38E010038B50F4C15
:104F24000F4DAC4218D90F4941F6D1130E4A0F4820
:104F34000FF04EFD0E480FF04BFD41F6D1110A481B
:104F44000FF03DFD0321204610F0E6F910B920468C
:104F5400FFF74CFE4434E4E7F4D338BD38050020B1
:104F64007C050020158F0100C68E01007E780100AB
:104F74009B7D01002DE9F04117460546F8B1022951
:104F840002D0082918BF062138464FF03A08DCB28F
:104F94006E185CB115F8011B0123412210F086FA4A
:104FA400033CB54200F8018BE4B2F2D187424FF0E2
:104FB400000306D000F8013C3846BDE8F081024801
:104FC400FBE71846F9E700BF948F01004FF0FF326A
:104FD4000121014811F006B9AC170020014601482F
:104FE40010F07EBAD00400200146014810F078BACF
:104FF4000405002010B404460846646804498C4241
:1050040002D110BCFFF7EABF10BCFFF7EDBF00BF31
:10501400600300202DE9F043554E9DB002AD0022FF
:1050240000232946534806F02DFB10B11DB0BDE8FE
:10503400F0834FF0FF324FF0FF334F4806F00AFC85
:105044004E4CDFF83C8144452CD94E49FD234E4A51
:105054004E480FF0BDFC4E480FF0BAFCFD214A4803
:105064000FF0ADFCDDE91801D4E9002381EA030760
:10507400374215D1C1F31307074309D0C3F313070C
:10508400174305D00B400240C3F313031A4307D060
:10509400E3681A9A0193169B0093A7682B46B847B6
:1050A4001034D0E7DED33B4F3C6824B14FF0000905
:1050B400D4F800802CB9304810F05AFA08F0ACFB50
:1050C400ACE7DDE91823D4E9041083EA000C1CEAF8
:1050D400060F30D1C3F3130C52EA0C0C0AD0C0F300
:1050E400130C51EA0C0C05D003400A40C3F313031C
:1050F4001A4320D0169B33B3A560169BE3600301CB
:1051040061682AD58A6912B11A9B9A4213D1DDE9E2
:105114001823C4E904231A9B8B612368B9F1000F97
:1051240013D17A683B60944200D17B6000236068AD
:10513400236006F09DFEB8F1000F16D0D8F80030B9
:1051440044469846B6E7A360D8E7C9F800307B68C0
:105154009C4208BFC7F80490E8E71A9B20460093D6
:10516400DDE918238847A146E5E74346E8E700BFA1
:105174000000F0376C04002008040020546E010085
:10518400546E0100CA8F01009E8F01007E780100D9
:105194009B7D0100C417002000210C4B1A6802B942
:1051A400704782420FD1026839B959681A6088423F
:1051B40000D15A600023036070470A605A68904225
:1051C40008BF5960F6E711461268E8E7C4170020E3
:1051D400002200230020204970B5C1E900230346C2
:1051E40002461E4C1E4DAC4216D908B1C1E900322C
:1051F4001C49A4231C4A1D480FF0EAFB1C480FF06D
:10520400E7FBA42118480FF0DAFBD4E9006010345E
:10521400024333430120E6E7F7D358B1C1E9003232
:105224001448006848B10468002540B90DB1C1E9CB
:10523400003270BD03460246F2E70446F4E7D0E9C3
:1052440004502B43024324B1256820462C460125F3
:10525400EBE72546F9E700BF100B0020546E010070
:10526400546E0100CA8F01009E8F01007E780100F8
:105274009B7D0100C417002010B504464FF0FF3297
:105284004FF0FF330D4806F0E5FA2046FFF784FFA0
:105294000B4B1A6822605A681C6002B95C60094BA7
:1052A400D4E90412D3E9004021430243C3E90012C4
:1052B4000248BDE8104010F05BB900BF08040020AC
:1052C400C4170020100B00202DE9F8430D46914629
:1052D400C1F3017225499846D1E9003432EA1472C7
:1052E4000646089F3FD1C5F3065232EA14523AD11A
:1052F40025EA040420EA0303C4F31304234332D14C
:105304004FF0FF324FF0FF33194806F0A3FA194B60
:1053140068221846002111F020FB0346B8F1000F63
:1053240008D03FB1502F19D83A46414611F0EFFA50
:1053340003460765C3E91665C3F8609000230D4969
:105344004FF420320C4810F021FF094810F010F9F6
:10535400BDE8F84309490A4810F0A8BF0448BDE86D
:10536400F84310F005B9BDE8F88300BF100B002026
:105374001C040020A80A00206C040020E400002083
:10538400180B00207FB5FFF723FF0023CDE904337A
:10539400084B0948039307F051F903AB00934FF40A
:1053A40000624FF0FF330549034807F061F907B085
:1053B4005DF804FBF88F0100180B0020A0540020B6
:1053C40037B540230C460A490093411A4911054652
:1053D4002346084A084810F0CDF8014628B128466B
:1053E400234603B0BDE83040184703B030BD00BFCA
:1053F400E0170020E9550100286B0100C9B2032918
:1054040008B509D909490A487E230A4A0FF0E0FA87
:105414007E2108480FF0D3FA0C22036901FB023302
:10542400D3F8880000F0070008BD00BF3E900100DB
:105434007E7801000190010070B5C9B203290346CA
:1054440000690BD919491A484FF4E873194A0FF047
:10545400BFFA4FF4E87117480FF0B1FAEFF3118671
:10546400202484F31288BFF36F8F0C2505FB0104FD
:10547400D4F8884014F0C00401D0A24212D1012211
:1054840005FB0100C0F88820002086F31188BFF3D3
:105494006F8F30B90C225B6802FB01335B6898475D
:1054A400002070BD4FF0FF30EFE700BF3E900100D9
:1054B4007E7801000190010070B50D46064904464E
:1054C400411A491140220548FFF7B6FF2B46014611
:1054D4002046BDE870401847E0170020286B010003
:1054E4002DE9F8430022012107460520FDF77EFF40
:1054F400114803F023FF0446C0B903F053FF2546C7
:105504004FF00C094FF001083E690C4906EB4510B9
:105514000FF0BBFB031E0CDB09FB05660135042DF4
:10552400C6F88880F0D12046BDE8F8836FF0040403
:10553400F9E71C46F7E700BF05560000BC70010000
:1055440010B50022012386B06C46CDE9022304ABDA
:10555400CDE90433074A6B46CDE9004410F03BF82B
:1055640028B94FF480420023684606F005FD06B0D2
:1055740010BD00BF0D56010010B5EFF311842023B8
:1055840083F31288BFF36F8F074A136823F0020175
:10559400DB07116002D4012003F060FF84F311885B
:1055A400BFF36F8F10BD00BF901800200C22124B68
:1055B400014602FB0033002030B4D3E92052C3F883
:1055C4008000EFF31180202484F31288BFF36F8FDF
:1055D400D3F8884004F0C00444F00204C3F88840BF
:1055E40080F31188BFF36F8F1DB12B4630BC034885
:1055F400184730BC704700BFE0170020286B01003B
:1056040008B5092822D8DFE800F00513212121215B
:105614002115110F134BD3F8880010F007001FD188
:10562400BDE80840FFF7C2BF0220F9E70320F7E70F
:105634000120F5E70C4940F2FA230C4A0C480FF01C
:10564400C7F940F2FA2109480FF0B9F906494FF4B5
:105654004173064A06480FF0BBF94FF44171F2E773
:1056640008BD00BFE01700203DA401000190010027
:105674007E78010010B4EFF31180202282F31288A7
:10568400BFF36F8F18490B6843F0020413F0010352
:105694000C601CD04FF05023D3F80C14D3F80C3406
:1056A40013F0010313D0EFF3118182F31288BFF3D7
:1056B4006F8F0E4AD2F8883003F0C00343F0020320
:1056C400C2F8883081F31188BFF36F8F012380F310
:1056D4001188BFF36F8F1BB1002010BCFFF766BFAA
:1056E400012010BC03F080BE90180020E0170020B9
:1056F4002DE9F041012206464349D1E8EF3FC1E8D4
:10570400E02F0028F9D1A3B9404941484B60CB6050
:105714008A60FCF7E1F900280BDA3E4940F2A32342
:105724003D4A3E480FF054F940F2A3213A480FF0A5
:1057340046F9002E50D0731E012B5AD8012E07D1E2
:105744004FF05023D3F81C3403F00303022B43D04F
:1057540010F0BCFD054658B1EFF31188202383F304
:105764001288BFF36F8F01254FF050242C4F22E095
:105774002C4B1B78002BEFD04FF050230222804695
:10578400C3F80823F0E74DB340460FF024FCD4F8E7
:105794001835DBB2012B0ED1D4F804215AB1002202
:1057A400C4F80421D4F804210222C4F818252022C4
:1057B400C7F88021A360D4F81824D4F81834D2038D
:1057C400E1D503F00303022B01D0012EDBD155B147
:1057D40088F31188BFF36F8FBDE8F0810021212089
:1057E40008F032F9D3E74FF050230222C3F8042320
:1057F400F2E70D4940F2B523074A08480FF0E8F8EC
:1058040040F2B52192E700BFDC170020CC1700203E
:1058140000180020017F0100019001007E78010042
:1058240000E100E09B2C00203DA4010008B50748DE
:1058340010F05FFC38B10648FEF7EAF90448FBF7BC
:1058440053FC002008BD6FF01200FBE7986B0100C9
:10585400595800000A2838B50446074D04D1AB68EE
:105864000D2128465B689847AB6803485B68E1B242
:105874009847204638BD00BF986B0100F7B50F4626
:10588400164648B918491823184A19480FF0A0F8C1
:10589400182116480FF093F8E9B916491923134A49
:1058A40013480FF095F81921F3E7351BB5F5806F10
:1058B40028BF1D4600202A4601AB39190CF0E2FD31
:1058C40068B9019BAB420AD11C44A642EDD809D069
:1058D400162003B0F0BD4FF480630024F5E76FF0A9
:1058E4001500F6E70020F4E7CC9001009C9001003D
:1058F4007E780100DF90010038B5036961B9214960
:105904006423214A21480FF063F821480FF060F81E
:1059140064211D480FF053F8486850B91D496523A8
:10592400194A1A480FF054F81B480FF051F8652132
:10593400EFE7586800B30024884219D108688CB98D
:105944009C685860A14200D19860002008602AB188
:105954005A680A609A68596002B9996000200FE099
:105964002846E9E720609868814208BF9C60ECE71C
:1059740005680446002DF3D1002AE9D16FF0150023
:1059840038BD00BF41910100059101007E780100FE
:105994004A910100599101006B91010008B5036817
:1059A400590914D0012906D14FF6FF7203F01F03E1
:1059B400DA40D2070ED40B490B484FF482630B4AEA
:1059C4000FF006F84FF4826108480EF0F8FF4FF02C
:1059D400FF32EBE70360064B0648012908BF18466F
:1059E40008BD00BFE98901007E780100B689010085
:1059F400002884500025845070B5446801F01F05C8
:105A0400207C86B045EA4015A068002872D0B2F523
:105A1400001F04D1294604F035FB00204EE06068E5
:105A2400667CB2F5800F46624FF0000601A801962D
:105A3400466032D1B3F1007F14BF052304238DF8EF
:105A440004300023CDE904030393E3686E46CB409E
:105A540013F0010F34D1B2F1A07F31D16846009523
:105A6400FFF79CFF009B803350F82330DB0727D4DB
:105A74006A462946A06804F09BF9163018D00296AD
:105A84002946A06803AA04F033F8002816DB012293
:105A94002946A06804F074FABFE7B3F1C06F05D0DB
:105AA400B3F1007F14BF01230223C8E70323C6E731
:105AB4006946A06804F040FA0028E0DA06B070BD38
:105AC40032462946A06804F073F90028D8D19DF81D
:105AD4000010A06804F010FA0028D1D00749084843
:105AE40040F2F113074A0EF073FF40F2F11105483A
:105AF4000EF065FF6FF08500E0E700BF627B0100F8
:105B04007E780100829101002DE9F043466840F25D
:105B14000635337CD00601F01F0747EA431748BF18
:105B2400032302EA050558BFC2F3401387B0B5F555
:105B3400837F14468DF8033043D00DD8062D16D03C
:105B440005D8A5B1022D3ED06FF0150036E0B5F5AD
:105B5400807FF9D101250AE040F20222954234D037
:105B6400B5F5407F33D0B5F5007FEDD10225220392
:105B74002FD5012372688B409360B06880BB03A863
:105B84000397FFF70BFF039B00EB8300C4F3004371
:105B940083F00103C4F34044D0F8002244EA4304F0
:105BA4009DF8033022F4706244EA830422F00F0269
:105BB40044EA05231343C0F80032002007B0BDE8CF
:105BC400F0830725D3E70425D1E70525CFE703258F
:105BD400CDE7630341BF012372688B40D360CCE7F8
:105BE40039460DF1020204F0E3F814F4403F804614
:105BF40017D13946B06804F067F9B8F1000FDCD169
:105C04009DF80210B06804F077F90028D5D01E4939
:105C14001E48FC231E4A0EF0DBFEFC211C480EF03D
:105C2400CEFE4FF0000901ABCDE90199CDE904396D
:105C3400CDF80C903946B06803AA03F059FF4845E3
:105C4400BBDB14F4003314D09DF80330C4F30044D8
:105C540084F001048DF80E308DF80C508DF80D4051
:105C64004B463946B06803AA04F004F80028C4DAA5
:105C7400A3E7CDE904330DF1030303933946B06878
:105C840003AA03F035FFF1E7627B01007E7801008F
:105C9400829101004209034670B502D0012A1ED048
:105CA40070BD144E326951680029F9D0012503F002
:105CB4001F030C689D400029F2D08A682A4012D044
:105CC4004B6873B90C4989230C4A0D480EF080FEC9
:105CD4000C480EF07DFE892108480EF070FE0A4E35
:105CE400E0E7304698471CB1236821461C46E2E7AA
:105CF4002346FAE7606B0100AE91010005910100B3
:105D04007E7801006B910100446B010038B5456851
:105D1400A86890B104F0BEF8014670B9A86804F010
:105D24007BF8044658B902460649A86804F028F8E6
:105D3400224605210D20FDF759FB002038BD6FF0E8
:105D44000400FBE7995C000008B50368590914D006
:105D5400012906D14FF6FF7203F01F03DA40D20780
:105D64000ED40B490B484FF482630B4A0EF030FEFD
:105D74004FF4826108480EF022FE4FF0FF32EBE749
:105D84000360064B0648012908BF184608BD00BF3A
:105D9400E98901007E780100B68901000028845059
:105DA400002584502DE9F04F154607464FF00109B0
:105DB40085B000EB8108B84503D1002005B0BDE8EB
:105DC400F08F3B68C3F3C322082AC3F3080400F22C
:105DD400B4805B498E5C40F2FF12944208BF4FF0DE
:105DE400FF34B3F10C5F4FEA136215D2222A15D89F
:105DF400DFE802F017262B3A2E353A141414144017
:105E04004C1414141414141414144F86898C14147C
:105E1400148F94979A9DA0004E2A28D06FF0850085
:105E2400CCE7C5F80C45621C68D003A80394FFF7BF
:105E34008BFF039B4FF0010A09FA03F383603BE0F5
:105E4400C5F814454FF0000A1BE0C5F80845EAE719
:105E54004FF0000AC5F80845611C25D14EE04FF00B
:105E6400010AC5F80C45F7E7C5F81045EAE7C5F897
:105E74001445D8E7C5F80845002EE3D14FF0000AD1
:105E84000626631C3AD04FF0000B17E0C5F80C450A
:105E9400F2E7C5F860457B88601C03F001032DD050
:105EA400002BC2D14FF0010A03A80394FFF74CFF63
:105EB400039B09FA03F3C3604FF0010B3A6803A88C
:105EC400130444BF4FF0010A4FF0000B01920394F6
:105ED400FFF73AFF039B019A00EB8300C2F34122D0
:105EE4003302D0F8001243EA8203164A43EA0B0352
:105EF4000A40134343EA4A03C0F8003204375AE71E
:105F0400C5F86445C7E7C5F86845C4E7C5F86C45F6
:105F1400C1E7C5F824454FF0010AB2E7C5F82845A2
:105F240081E7C5F83045F6E7C5F83445F3E7C5F829
:105F34003845F0E7C5F83C4575E76FF015003DE7D7
:105F4400785F0200F0F0FCFF2DE9F04104460D46B5
:105F5400476810F0BBF988B14FF02008EFF31186C1
:105F6400314688F31288BFF36F8F60680FF0B3FB7C
:105F740050BB86F31188BFF36F8FEFE71F4B1B787D
:105F8400002BE9D04FF02008642660680FF0A3FBD3
:105F940070B901200FF0C4FE013EF6D1002121208A
:105FA40007F052FDF0E786F31188BFF36F8FF5E732
:105FB400EFF31186314688F31288BFF36F8F606860
:105FC4000FF089FB0028EED0FB6900201D70636888
:105FD400FA691B68C3F844250122C3F84825C3F8AD
:105FE4002001D3F82041C3F85801D3F858019A602E
:105FF40081F31188BFF36F8FBDE8F0819B2C0020E3
:106004002DE9F0410546002201210820FDF7EEF9B3
:106014000820FDF7BBF96C680121E0680FF08CFBE8
:106024006B6819682369C1F82435A27D637D207DDE
:106034001343228B02431343C1F86C356F6800226B
:10604400D7E9004313F001031CD0D5F8108004F104
:106054000C01C4F8A02104F59070C4F88C2008F158
:1060640008020FF092FE061E07DA0121214A224897
:106074000EF0C5FE3046BDE8F08198F8080003F044
:106084003DF901230822C4F80025FA690121C4F866
:1060940044250022C4F84825A1606BB9D4F8203106
:1060A400002BFBD0C4F82021D4F820310123E36075
:1060B4004FF48073C4F80433D4F85831002BFBD068
:1060C4000021C4F800156D68E8682C680FF034FBF3
:1060D4000823C4F800352A7A52B92B6AC4F8343537
:1060E4000123C4F83835C4F81021D4F810212360F2
:1060F4000026BFE7D2910100C46E010038B51149F2
:1061040022F07F45D1E90030D41AE31840F10000B1
:10611400C1E90030A5F50013B3F5400F09D20A4BCD
:106124001B681A0A1B065819084B42F10001C3E9FF
:10613400000108F0E9F901462046BDE8384008F0BE
:106144004BB900BFC80B0020C0180020D00B0020A2
:106154000D4B1868010A0006BFF35F8F0B4BD3F891
:106164000435181841F10001B3F5801F0AD2084B19
:10617400D3E90023904271EB030303D210F1807042
:1061840041F10001704700BFC018002000500150C9
:10619400D00B00202DE9F7432D4BD3F804239107AE
:1061A4000BD5D3F8042142B10022C3F80421294AB3
:1061B400D3F80431136801331360254CD4F8043345
:1061C400DA033FD5244BD3E8EF2F22F00101C3E8D3
:1061D400E01F0028F7D1D30702D4D4F840318BB3A1
:1061E4000025C4F84051D4F84031FFF7B1FFEFF374
:1061F4001182202383F31288BFF36F8F174BD3E9E7
:106204000267B042B94120D3D3E900984FF0FF3080
:106214004FF0FF311D60C3E902014FF48033C4F82D
:106224004833C4F84051D4F8403182F31188BFF3A5
:106234006F8FB9F1000F05D032463B460020CDF8F0
:106244000080C84703B0BDE8F083A946EDE700BF6E
:1062540000500150C0180020B8180020B80B0020CE
:106264002DE9F84F06460F46434DD5E8EF8F28F049
:106274000103C5E8E23F002AF7D14FF480393F4CCF
:10628400C4F80893BFF35F8FBFF36F8FFFF760FF0E
:10629400B04271EB070308F0010840D2384B301AC2
:1062A40067EB0101984271F1000148D2354BD3E903
:1062B40002239F4208BF96423AD04FF0000C26F0CA
:1062C4007F40834603216FF0020EC4F84893C4F85C
:1062D40040C1D4F84031DFF8B0A02BF07F43C4F8BC
:1062E4004035C4F84493D4F80425AEEB02035B4470
:1062F40023F07F4353451BD9D4F840315BB1D4F824
:106304000425131A23F07F43B3F5000F10D9C4F802
:1063140040C1D4F8403101EB020B0131DDE71B4BE6
:10632400D3E8EF1F41F00101C3E8E21F002AF7D1CF
:10633400144B174AC3E902671A6000225A60B8F185
:10634400000F16D0D5E8EF3F43F00103C5E8E23F64
:10635400002AF7D14FF48032084BC3F804230B4BC7
:10636400D3E8AF3FDB0742BF4FF40012094BC3F839
:106374000021BDE8F88F00BFBC1800200050015078
:1063840001008000B80B0020FDFF7F00B81800203A
:106394000161000000E100E070B54FF0FF3000251E
:1063A4004FF0FF31164C174B0226C4F80833C4F8DB
:1063B4004833154BC4F80855C3E902014FF4803340
:1063C4004FF40012C4F80433104B0121C4F80463E1
:1063D4001520C3F880212A46FDF708F81520FCF79C
:1063E400D5FF01230A4AA3600021236009481360F2
:1063F400FFF736FF3046FFF77BF9284670BD00BF34
:106404000050015003000F00B80B002000E100E031
:10641400BC180020FFFF7F00431C10B50F4C05D0B3
:106424008442A8BF0446012CB8BF0124FFF790FEA4
:106434000B4AD2E90031C01AB0F5000F074A0AD25C
:106444002044904228BF1046BDE81040C01841F1D6
:106454000001FFF705BF1046F6E700BFFFFF7F000E
:10646400C80B002008B5FFF773FE024B1B68C01A67
:1064740008BD00BFC80B0020B0B50C4600AFA0B9E2
:106484006C4688B06A461E4B53611E4B4FF4E25172
:1064940093614FF4007393831B4B1C4842F8103FE5
:1064A4000FF05EF9A546BD46B0BDC36823B96C467E
:1064B40088B06A46164BE7E75D6825B96C4688B034
:1064C4006A46144BE0E795F82430002BEBD02D20DE
:1064D40008F0A0FBE86220B96C4688B06A460E4B0F
:1064E400D2E7214604F12C0351F8042B994240F8D9
:1064F400042BF9D10B7803700123AB62D3E700BFFF
:106504000B920100B15F020003000001CC6E010098
:10651400239201003B9201005492010098B500AF10
:10652400A0B96C4688B06A46144B5361144B4FF4BF
:10653400E25193614FF400739383124B124842F873
:10654400103F0FF00DF9A546BD4698BDC3685C68C1
:10655400237E23B16C4688B06A460C4BE5E70B22D8
:106564008B8C206AA4F81930D1F826302A315A438A
:10657400E36110F0CCF901232376E5E70B920100E7
:10658400C65F020003000001CC6E0100819201008D
:1065940080B500AF88B06A46084B4FF4E2510593CA
:1065A400074B084806934FF40073ADF81C30064BB4
:1065B40042F8103F0FF0D4F8BD4680BDA19201000F
:1065C400E15F0200CC6E01000300000180B500AF62
:1065D40088B06A46084B4FF4E6510593074B0848C8
:1065E40006934FF40073ADF81C30064B42F8103F8D
:1065F4000FF0B6F8BD4680BDCB92010005600200E5
:10660400CC6E01000300000198B500AFA0B96C4640
:1066140088B06A46154B4FF4E2510593144B069328
:106624004FF40073ADF81C30124B42F8103F12487F
:106634000FF096F8A54604E0036B23B9703005F01B
:106644008FFFBD4698BD6C468AB06A460B490591DA
:106654000749CDE906134FF40073ADF82030084B19
:106664004FF4115142F8103FE1E700BF0B920100D3
:106674002060020003000001CC6E0100E4920100DE
:1066840004000001F0B58FB000AF044620220021C1
:1066940007F1180010F061F90023464EC7E90033F2
:1066A400C7F8073033782469012B19D96C4688B0B0
:1066B4006A46414B4FF4E2510593404B40480693E0
:1066C4004FF40073ADF81C303E4B42F8103F0FF00E
:1066D40047F8A5466FF00B0420463C37BD46F0BD95
:1066E400394D3A4904F14000E56006F031F8384983
:1066F40004F1700005F0A4FE4FF6FF73A4F8EC302B
:1067040033785A1C3270002B51D101F035FF044606
:10671400A8B16D468AB06A462E4B4FF411510593C9
:10672400264BCDE906304FF40073ADF820302A4BE8
:10673400234842F8103F0FF013F8AD46CCE7274B3F
:106744002748C7E903337B61264BBB61264BFB61BA
:10675400264B3B62264B7B63264B3B63264BFB62FB
:1067640008F052FA384607F1180207F10C0109F053
:1067740067FB45F8080CB0B96C4688B06A461F4BF5
:106784004FF4E25105930D4B0D4806934FF40073FB
:10679400ADF81C300B4B42F8103F0EF0E1FFA5465C
:1067A4004FF0FF3498E705F5FA700FF0FEFC002473
:1067B40092E700BFE12A002009930100815F0200F3
:1067C400CC6E010003000001E00B0020855701009E
:1067D4006B5701002893010004000001E803020044
:1067E40014720100ED6A0000635701000D66000099
:1067F4007D64000021650000497700005C9301007E
:106804002DE9F04194B0002306AF806000F1080147
:1068140005460068BB6009F0C9FA0646C8B96C466B
:1068240088B006AA374B4FF4E2515361364B3748D0
:1068340093614FF400739383354B42F8103F0EF08D
:106844008FFFA5464FF0FF3420463837BD46BDE8DC
:10685400F081E860FCF788F80446C0B1E84688B0E7
:1068640006AA2C4B5361284B4FF4E25193614FF429
:1068740000739383264B254842F8103F0EF070FFB7
:106884003046C5460FF061FE0023EB60DCE730467E
:1068940007F1080108F0BEFD044620B1E84688B0BF
:1068A40006AA1D4BDEE71D4BC7E90600FB6003F19A
:1068B4007E6303F53E2303F53D633B6134233B755F
:1068C400174BC7E90800C7E90A003863B88678603F
:1068D40004933B1D039307F10C03029307F1180380
:1068E400019301230093022103460E4AE86809F04C
:1068F400F7FE04460028A7D0E84688B006AA0A4B4B
:10690400B0E700BF7A930100975F0200CC6E0100EC
:10691400030000019B930100B793010054404024FD
:10692400D29301007B000300D7930100B0B550F867
:10693400AC4C00AF50F8B40CFEF758F9A0B16D465A
:106944008AB06A46134B4FF411510593124BCDE9AB
:1069540006304FF40073ADF82030104B104842F865
:10696400103F0EF03EFFAD46002384F808320FF0CE
:1069740038FD4FF47A72A0FB020302FB0131C00B15
:1069840040EA4140C4F80C0204F5FA700EF02CFF02
:10699400BD46B0BD03940100C660020004000001BE
:1069A400CC6E0100F8B550F8A03C054600AFA3B981
:1069B4006C4688B06A46444B5361444B4FF4E251F1
:1069C40093614FF400739383414B424842F8103F64
:1069D4000EF007FFA546BD46F8BD50F8984C0CB123
:1069E400636823B96C4688B06A463B4BE4E79E680B
:1069F40026B96C4688B06A46384BDDE794F808320D
:106A0400002BE8D1D4F80C321BBB4FF0FF324FF00F
:106A1400FF3304F5FA7004F01DFF012384F80832F3
:106A2400D6F8A820D4F81C321344C4F81C32D6F883
:106A3400AC20D4F820321344C4F8203255F8A00C0A
:106A4400FEF728F9F0B9D4F814320133C4F814323B
:106A540032E00FF0C6FC4FF47A7CA0FB0C320CFB46
:106A64000121DB0BD4F80C2243EA41439B1A41F287
:106A740088324FEAD13161F10001934271F1000192
:106A8400C3DAA8E7D4F818320133C4F818326C46D4
:106A94008AB06A46124B4FF4115105930B4BCDE962
:106AA40006304FF40073ADF820300E4B094842F81D
:106AB400103F0EF096FEA5464FF48032002305F1F8
:106AC400140005F07DFF86E71C940100A36002001A
:106AD40003000001CC6E01002392010037940100F1
:106AE4004F9401000400000198B5044600AFA0B91A
:106AF4006C4688B06A46104B5361104B4FF4E25118
:106B040093614FF4007393830D4B0E4842F8103F8A
:106B14000EF067FEA546BD4698BD00680FF021FD46
:106B240020B96C4688B06A46074BE5E76068A43034
:106B340005F016FDEFE700BF939401001C6102000D
:106B440003000001CC6E0100A79401002DE9F84375
:106B5400044600AFC0B96C4688B06A46384B5361EE
:106B6400384B4FF4E25193614FF400739383364BE7
:106B7400364842F8103F0EF034FE4FF0FF35A5467C
:106B84002846BD46BDE8F88300F114064FF0FF32F5
:106B94004FF0FF33304604F05DFE20B16C4688B000
:106BA4006A462B4BDBE7E368002B45D05868002886
:106BB40042D004F180094A46217C08F03FFC054696
:106BC400B8B16C4688B06A46224B4FF4E251059343
:106BD4001C4B1E4806934FF40073ADF81C301A4B3F
:106BE40042F8103F0EF0FDFDA54630460EF0FCFDC8
:106BF400C6E748460FF094FC80460028F5D11823D8
:106C040006214846144AFEF7B5F96D468AB06A462D
:106C1400124B4FF4215105930A4BCDE90630104B2A
:106C24000A4808930F4B42F8103F0EF0DAFDAD46C8
:106C3400C4F88080A9F804804FF0FF35D5E700BF81
:106C44000B9201000661020003000001CC6E0100FA
:106C5400BF940100DB940100E22A002007950100A3
:106C64000002010304000002F8B5044600AFA0B915
:106C74006C4688B06A46274B5361274B4FF4E25168
:106C840093614FF400739383244B254842F8103FDB
:106C94000EF0A7FDA546BD46F8BD02680AB113680B
:106CA40023B96C4688B06A461E4BE5E71D6925B9D1
:106CB4006C4688B06A461C4BDEE7E96821B96C462D
:106CC40088B06A46194BD7E72E469268686046F842
:106CD400A43B01239376FDF713FD20460EF0A3FA9F
:106CE40020460EF0D0FB3046114905F0A9FB1149AE
:106CF40005F1B80005F02CFD2368002BCBD00C3334
:106D0400D3E8EF1F41F40051C3E8E21F002AC2D0C8
:106D1400F6E700BF6A940100F1600200030000017D
:106D2400CC6E0100239501000B9201002392010017
:106D3400A9690000316900002DE9F04F8FB0804649
:106D440000AFF8B96C4688B06A469B4B4FF4E251E9
:106D540005939A4B9A4806934FF40073ADF81C3090
:106D6400984B4FF0FF3542F8103F0EF03AFDA54620
:106D7400444604F114000EF037FD28463C37BD4666
:106D8400BDE8F08F0FF0B5F98146C0B96C468AB002
:106D9400D8F800306A468C498948059187494FF0F4
:106DA400FF35CDE90613894B4FF421510893884BE5
:106DB40042F8103F0EF015FDA5460024D9E74046E1
:106DC4000EF019FD054630B101210346814A7C4885
:106DD4000EF01EF8F1E7D8F810409CB96E4688B062
:106DE4006A467D4B5361754B4FF4E25193614FF406
:106DF40000739383734B724842F8103F0EF0F1FC1A
:106E0400B546B6E7D4F80CA0BAF1000F15D16D461B
:106E140088B06A46714B5361684B4FF4E2519361F9
:106E24004FF400739383674B654842F8103F0EF0AC
:106E3400D8FCAD466FF004059BE704F114064FF04F
:106E4400FF324FF0FF33304604F004FD054620B115
:106E54006E4688B06A46624BC4E7DAF8043043B938
:106E64006048FFF7CDFC28B16D4688B06A465E4B9A
:106E7400D1E781461E22002107F11800DAF804B098
:106E84000FF06BFD0223D8F800107B61084679608F
:106E9400F9F778F97968024607F126000FF037FD13
:106EA4002146584607F1140209F0B8F80128207465
:106EB40019D96D4688B06A464C4B53613F4B4FF429
:106EC400E25193614FF4007393833E4B3C4842F884
:106ED400103F0EF086FCAD46B9F1000FAAD0414830
:106EE4000EF067FCA6E730460FF05FF97B69666831
:106EF400C4F8883016B1366806B11036023630460A
:106F04000FF00EFB50BB2046FFF720FEF0B16D469C
:106F140088B06A46364B5361284B4FF4E251936173
:106F24004FF400739383274B254842F8103F0EF02B
:106F340058FCAD46217CDAF8040009F073F9002806
:106F4400CAD06D4688B06A462A4BB6E704F180067B
:106F540003230622314660680EF042FA3246217C51
:106F6400DAF8040009F02AFA20B16D4688B06A46BE
:106F7400214BD0E70126D8F8008094F810B04046A1
:106F8400FE6087F810B0F9F7FDF84146024604F1B7
:106F94008C000FF0BCFC5946DAF8040007F10C022F
:106FA40009F0BAF920B16D4688B06A46134BB2E7CE
:106FB40084F89C60DDE600BF6A9401008D600200E5
:106FC400CC6E0100030000013395010000020103AF
:106FD400040000024E9501000B920100239201006F
:106FE400BF940100D80B002080950100A5950100F5
:106FF400CF95010036960100ED9501000B96010036
:107004002DE9F04383B0044600AFC8B96C4688B09C
:107014006A464C4B53614C4B4FF4E25193614FF42D
:1070240000739383494B4A4842F8103F0EF0D9FB52
:10703400A5464FF0FF3420460C37BD46BDE8F0832B
:10704400D0F81080B8F1000F04D16C4688B06A46BD
:10705400404BDFE708F114054FF0FF324FF0FF33E8
:10706400284604F0F7FB10B36E4688B06A463A4BE4
:107074005361354B4FF4E25193614FF400739383A2
:10708400324B334842F8103F0EF0ABFBB54628466E
:107094000EF0AAFB20460EF0B0FB04460028CAD02E
:1070A400012103462D4A2A480DF0B2FEC3E7D8F861
:1070B4000C600EB1736823B96E4688B06A46284BDB
:1070C400D6E798F81010386039713A46706809F0BC
:1070D40023F998B1E94688B06A46224B4FF4E2514D
:1070E4000593194B1A4806934FF40073ADF81C30FE
:1070F400164B42F8103F0EF074FBCD4698F8101072
:10710400706809F08FF898B1E84688B06A46164B63
:107114004FF4E25105930C4B0D4806934FF4007362
:10712400ADF81C30094B42F8103F0EF05AFBC5462F
:1071340070680FF02AFA0028A9D10C480EF039FB28
:10714400A5E700BF6A940100786002000300000113
:10715400CC6E01000B920100BF9401005B9601000C
:10716400239201000B96010036960100D80B0020F3
:107174002DE9F8430E46154600AF00B1C2B96C467E
:1071840088B06A46354B5361354B4FF4E2519361F5
:107194004FF400739383334B334842F8103F0EF09F
:1071A40020FBA5464FF0FF342046BD46BDE8F883DA
:1071B400D0F81090B9F1000F04D16C4688B06A463B
:1071C4002A4BE0E709F114084FF0FF324FF0FF3388
:1071D400404604F03FFB0446A0B16D4688B06A46C1
:1071E400234B4FF4E25105931D4B1F4806934FF474
:1071F4000073ADF81C301B4B42F8103F0EF0F1FA4F
:10720400AD46D1E7D9F80C30C3B15868B0B10FF02E
:10721400A8F9B8B96D4688B06A46164B4FF4E251E6
:1072240005930F4B104806934FF40073ADF81C30D0
:107234000C4B42F8103F0EF0D4FAAD4640460EF027
:10724400D3FAB1E73022214628460FF086FB0B3EE5
:10725400012E9CBF084B2B60F0E700BF6A9401002D
:107264005D60020003000001CC6E01000B9201007E
:10727400BF940100A7940100030C60002DE9F843BA
:107284008946144600AFC0B96C4688B06A463F4B85
:1072940053613F4B4FF4E25193614FF40073938376
:1072A4003C4B3D4842F8103F0EF09BFA4FF0FF353F
:1072B400A5462846BD46BDE8F883D0F81080B8F14D
:1072C400000F04D16C4688B06A46344BE0E708F1FD
:1072D40014064FF0FF324FF0FF33304604F0BAFA91
:1072E4000546A0B16C4688B06A462D4B4FF4E25176
:1072F4000593274B284806934FF40073ADF81C30D0
:10730400244B42F8103F0EF06CFAA546D1E7B9F1D0
:10731400000F2BD12378EBB96378EBB9A378DBB9F1
:10732400E378CBB92379BBB96379ABB96C4688B040
:107334006A461C4B5361164B4FF4E25193614FF470
:1073440000739383134B144842F8103F0EF049FA2C
:10735400A54607E0DB07E9D42368C8F88030A38892
:10736400A8F8843030460EF03FFAA2E7D8F80C3083
:10737400002BF7D058680028F4D00FF0F2F800285A
:10738400F0D16C4688B06A46074BD3E76A94010093
:107394004260020003000001CC6E01000B92010068
:1073A400BF9401008C960100A79401002DE9F84FC9
:1073B40006690D46924600AFC6B96C4688B06A4667
:1073C400A94B5361A94B4FF4E25193614FF40073FD
:1073D4009383A74BA74842F8103F0EF010FA4FF0E2
:1073E400FF35A5462846BD46BDE8F88F96F89C4073
:1073F400012C04D06C4688B06A469F4BE1E7D6F86E
:107404000C90B9F1000F04D16C4688B06A469B4BCE
:10741400D7E706F114084FF0FF334FF0FF32404630
:1074240004F018FAD9F804302BB94FF0FF35404670
:1074340004F0D8FAD6E796F82C30B3B16C4688B08D
:107444006A468F4B4FF4E6510593884B06934FF4ED
:107454000073ADF81C30864B42F8103F85480EF09F
:10746400CEF96FF00F05A546E1E7002D3ED06B780D
:10747400032B29D8E87C38B16B7D002B38D0EB7D09
:10748400002B14BF032002208000C6F828A000F5BA
:10749400F57A504607F0C4FB044658BB6C468AB0E4
:1074A400784A794B0592714A4FF41151CDE9062A75
:1074B4004FF40072ADF820206A466E4842F8103F3F
:1074C4000EF09DF9A546B0E76C468AB06A466F494E
:1074D40005916649CDE906134FF40073ADF82030E9
:1074E400694B4FF4115142F8103FB7E72846CBE7F8
:1074F4002046C9E7524600210FF02FFA002384F8F2
:10750400E93123706370A370E370002D47D02A78AB
:10751400012A04BF227163716B7884F84A306B8846
:10752400A4F8E331AB88A4F8E5312B8AB386AB68C1
:107534005BB31A784AB304F10800024603F1200150
:1075440053F804CB8B4242F804CBF9D1F8F71AFE76
:1075540094F806A0E0710AF10103A371EB68A3B1EA
:107564001A7892B104F12900024603F1200153F87C
:1075740004CB8B4242F804CBF9D1F8F703FE0AF1AD
:10758400020A84F8280084F806A0AB464FF0000AEB
:107594009BF81310F9B95FFA8AF3A4F8E7310023D2
:1075A400B3632246317CD9F8040008F0BDFC0546DB
:1075B40000284CD06D4688B06A46354B4FF4E251F2
:1075C40005932A4B06934FF40073ADF81C30284BF7
:1075D40042F8103F14E09BF81200D8B1012819D0EA
:1075E4006D468AB06A462B4B0593204BCDE9063095
:1075F4004FF400734FF411511384234B42F8103F9E
:107604001C480EF0FCF8AD464FF0FF35204607F05D
:1076140013FB0CE707F048FD04EB8A03C3F8EA0107
:1076240001300BD105EB4A036D468AB06A46DB7C18
:10763400194905910D49CDE90613D9E70AF1010A63
:10764400BAF1030F0BF1020BA2D15346A5E70123B4
:10765400306386F82C304FF47022002306F140008A
:1076640005F026F9D2E700BF0B9201006161020028
:1076740003000001CC6E0100A496010023920100D6
:10768400B9960100F596010004000001D6960100A8
:1076940061970100329701004A970100F8B5C66866
:1076A400044600AFC6B96C4688B06A46204B4FF416
:1076B400E25105931F4B204806934FF40073ADF835
:1076C4001C301E4B42F8103F0EF099F8A5464FF0BF
:1076D400FF342046BD46F8BD00F114054FF0FF32DB
:1076E4004FF0FF33284604F0B5F87068E8B1217C08
:1076F400002208F05BFC044698B16E4688B06A46E6
:107704000F4B4FF4E25105930A4B0B4806934FF489
:107714000073ADF81C30094B42F8103F0EF06FF8BF
:10772400B546284604F05EF9D3E74FF0FF34F8E796
:107734002392010042610200CC6E010003000001AB
:10774400619701002DE9F0471E46836A04460F46FF
:107754008CB0C3B14FF0000AB0F83480DFF8F09079
:1077640001F1260597F8243053450FD85EB96068B7
:1077740032463146A36A984784F82C60A66204F125
:10778400400005F023F90CB0BDE8F087B8F1000F14
:1077940002D0A36B4345E9D22822002168460FF0AA
:1077A400DCF815F8012C4423212A28BF212203FBED
:1077B4000A738DF82120D96C8DF82210196D8DF87B
:1077C4002310D3F855300C2B8CBF172319F8033032
:1077D4008DF8243095F8403033B1D90730D413F004
:1077E400020F14BF01230323294668468DF826306F
:1077F4000FF08DF8AB8C286AADF82C3006238DF889
:107804002E30442303FB0A730A9003F15802D3F881
:107814005D30022B16D1D2F80930642293FBF2F3C7
:107824008DF82730A36A6A46002160689847A36BE5
:107834000133A36305F0F0FF0AF1010A443591E72F
:107844000223D1E7032BEDD195F83B30E8E700BFE5
:107854003561020037B5C21C4FF0FF314FF0FF30E5
:1078640022F00305CDE900012A460421054803F06E
:10787400EBFB044618B12A4600210FF06EF82046AF
:1078840003B030BDC803002007B54FF0FF31C21C60
:107894004FF0FF3022F00302CDE900010421034838
:1078A40003F0D2FB03B05DF804FB00BFB00300207B
:1078B40008B50EF096FD044AA0FB020302FB013357
:1078C400C00B40EA434008BD40420F0008B50246E1
:1078D4000B46034850210CF09FFE002008BD00BF5A
:1078E400FA2A0020014610B1014803F0D3BB7047C7
:1078F400C8030020014610B1014803F0CBBB704718
:10790400B003002098B50E4C00AF02460B4620464B
:1079140050210CF081FE88B06A460A4B4FF4E651C0
:10792400CDE905344FF40073ADF81C30064B07481D
:1079340042F8103F0EF092F80020BD4698BD00BFFB
:107944004A2B00203277010003000001CC6E0100B5
:1079540098B50E4C00AF02460B4620464FF480719A
:107964000CF05AFE88B06A46094B4FF4E251CDE957
:1079740005344FF40073ADF81C30064B064842F84A
:10798400103F0EF06BF80020BD4698BD9A2B0020E6
:107994003277010003000001CC6E0100F8B500AF9E
:1079A400044600F0C5FB054600F0E0FE80B16C46DD
:1079B4008AB06A461B4B53611B4B4FF41151C2E909
:1079C40006304FF400731384184B42F8103F15E04F
:1079D400AE6800F087FBB04740B2B8B16C4688B0DF
:1079E4006A46134B4FF4E25105930F4B06934FF441
:1079F4000073ADF81C300F4B42F8103F0E480EF0E8
:107A04002DF8A54600242046BD46F8BD0EF0CEF85C
:107A140020B16C468AB06A46084BCCE70123256046
:107A24002371F0E78397010024620200040000013F
:107A3400A597010003000001CC6E0100C19701006D
:107A440080B500AF88B06A46084B4FF4E251059305
:107A5400074B084806934FF40073ADF81C30064BEF
:107A640042F8103F0DF0FAFFBD4680BDE5970100D6
:107A74004F620200CC6E010003000001074B19683D
:107A840019B10B690BB1CB680BB9FFF7D9BF002251
:107A940000230348183104F087BE00BFE01800201B
:107AA400080E0020F8B5482000AF0E4615460DF02C
:107AB40059FF204C2060B8B96C4688B06A461E4B0A
:107AC4004FF4E25105931D4B1D4806934FF4007388
:107AD400ADF81C301B4B42F8103F0DF0BFFFA5461C
:107AE4004FF0FF30BD46F8BDC0E9036516491830B4
:107AF40004F02EFE1549206800F060FC0028F1D047
:107B04006D4688B06A46124B4FF4E25105930B4B15
:107B14000B4806934FF40073ADF81C30094B42F840
:107B2400103F0DF09BFFAD462068FFF7E3FE0023F6
:107B34002360D5E7E0180020FB970100646202008F
:107B4400CC6E010003000001B97D0000817A0000C1
:107B540027980100B0B58AB0134C00AF206800F03C
:107B6400E1FC0546B0B16C4688B06A460F4B4FF451
:107B7400E25105930E4B0F4806934FF40073ADF892
:107B84001C300D4B42F8103F0DF068FFA546283716
:107B9400BD46B0BD20683946183004F073FF206834
:107BA400FFF7A8FE2560F2E7E01800203E980100E8
:107BB4007F620200CC6E010003000001F8B50D469F
:107BC400DC1C036824F00304114600AF2246284657
:107BD400DB689847B0B16E468CB00B4A0B4B0592EC
:107BE4000B4ACDE90840CDE906254FF40072ADF803
:107BF40028206A464FF45151064842F8103F0DF0D0
:107C04002DFFB546BD46F8BD589801000600000199
:107C140078610200CC6E010080B500AF88B06A467E
:107C2400084B4FF4E2510593074B084806934FF471
:107C34000073ADF81C30064B42F8103F0DF00EFFF8
:107C4400BD4680BD829801008D610200CC6E0100AA
:107C5400030000014FF0FF324FF0FF3313B504214E
:107C6400CDE900230748142203F0EEF9044620B9B5
:107C7400FFF7D2FF204602B010BD142200210EF0FF
:107C84006CFEF7E7B003002080B500AF88B06A4609
:107C9400084B4FF4E2510593074B084806934FF401
:107CA4000073ADF81C30064B42F8103F0DF0D6FEC1
:107CB400BD4680BDAD980100A5610200CC6E0100F7
:107CC4000300000180B500AF88B06A46084B4FF44A
:107CD400E2510593074B084806934FF40073ADF83F
:107CE4001C30064B42F8103F0DF0B8FEBD4680BD77
:107CF400AD980100BF610200CC6E010003000001D9
:107D040080B500AF88B06A46084B4FF4E251059342
:107D1400074B084806934FF40073ADF81C30064B2C
:107D240042F8103F0DF09AFEBD4680BDE098010078
:107D3400DE610200CC6E01000300000180B500AFDB
:107D440088B06A46084B4FF4E2510593074B084844
:107D540006934FF40073ADF81C30064B42F8103F05
:107D64000DF07CFEBD4680BDE0980100F361020089
:107D7400CC6E01000300000180B500AF88B06A46F4
:107D8400084B4FF4E2510593074B084806934FF410
:107D94000073ADF81C30064B42F8103F0DF05EFE48
:107DA400BD4680BD0E9901000D620200CC6E01003B
:107DB4000300000198B5124B00AF1B681BB11A6990
:107DC4000AB1D868A0B96C4688B06A460D4B5361B5
:107DD4000D4B4FF4E25193614FF4007393830B4BBB
:107DE4000B4842F8103F0DF039FEA546BD4698BD3C
:107DF40090470028FAD06C4688B06A46054BE6E7FF
:107E0400E01800203A9901003E62020003000001DC
:107E1400CC6E01005899010080B500AF88B06A4665
:107E2400084B4FF4E2510593074B084806934FF46F
:107E34000073ADF81C30064B42F8103F0DF00EFEF7
:107E4400BD4680BD6A9401009C620200CC6E0100B4
:107E54000300000180B500AF88B06A46084B4FF4B8
:107E6400E2510593074B084806934FF40073ADF8AD
:107E74001C30064B42F8103F0DF0F0FDBD4680BDAE
:107E840076990100BF620200CC6E0100030000017C
:107E940098B51C4600AF052A66D8DFE802F0031542
:107EA40025354555884273D04FF48B63394A3A4996
:107EB4003A480CF08DFD214639480CF089FD4FF409
:107EC4008B6134480CF07BFD884261D140F25B4306
:107ED400304A344931480CF07BFD214630480CF0DF
:107EE40077FD40F25B41ECE7884251DB40F25E43B0
:107EF400284A2D4929480CF06BFD214628480CF0EE
:107F040067FD40F25E41DCE7884241DD40F26143B7
:107F1400204A264921480CF05BFD214620480CF0FC
:107F240057FD40F26141CCE7884231DC40F26443C2
:107F3400184A1F4919480CF04BFD214618480CF00B
:107F440047FD40F26441BCE7884221DA40F26743CE
:107F5400104A184911480CF03BFD214610480CF01A
:107F640037FD40F26741ACE76C4688B06A46124B75
:107F74004FF4E2510593114B114806934FF40073EB
:107F8400ADF81C300F4B42F8103F0DF067FDA546CD
:107F9400BD4698BD9D990100CB9901007E780100F2
:107FA400DB990100E0990100F0990100FF990100BB
:107FB4000F9A01001E9A01002E9A0100D462020059
:107FC400CC6E0100030000010149083004F0C0BB7D
:107FD400575B010013B50024104804F02FFB23461F
:107FE4004FF400620E490D48009404F041FB0D4922
:107FF4000A480EF071F90C4804F020FB6FF00E03F0
:108004004FF4006209490848009404F031FB084920
:1080140005480EF061F9204602B010BDA80E0020FC
:1080240000D20020579A0100080E002000CA002048
:10803400639A01000020054B42019A5C22B1013091
:108044006428F9D14FF0FF30704700BFE4180020D6
:1080540098B500AF0146FFF7EDFF431C17D16C46FE
:1080640088B06A460E4B05930E4B06934FF400738B
:10807400ADF81C300C4B42F8103F0C4800234FF471
:10808400E251FAF7A7F90020A546BD4698BD0124A0
:10809400074B420103EB40109C540177F5E700BF06
:1080A400719A0100E462020003000001CC6E010039
:1080B400E4180020C0E905210149043004F0C0B9E6
:1080C400935B0100037F012B03D1011D03480EF0D4
:1080D400EDB813B9011D0248F9E77047080E0020F6
:1080E400A80E002038B56C2200210C480EF035FC97
:1080F4004FF4D073094D0124AB804FF400036B623D
:10810400074B1022FF2105F12C00EB64EC710EF0FB
:1081140024FC044B6C64EB63284638BD64250020C2
:10812400909A0100481618160048704764250020EC
:1081340000487047F400002003460A462DE9F04148
:108144001979DB880068134303F03002302A06698A
:10815400D0E901470ED1294940F2F733284A29488A
:108164000CF036FC28480CF033FC40F2F73124487C
:108174000CF025FC254A264D1A40AA420CD125496B
:1081840040F2FB331E4A1F480CF022FC22480CF03C
:108194001FFC40F2FB31EAE703F00602042A09D18E
:1081A4001E4940F2FE33164A16480CF011FC40F208
:1081B400FE31DCE701251A4A24689A4305FA01F5E1
:1081C40008BF83F44023254223F480120CD11549BF
:1081D40040F211430A4A0B480CF0FAFB12480CF027
:1081E400F7FB40F21141C2E73468DB074CBF2C4374
:1081F400AC4334603B68BDE8F0411847CB9A0100BA
:108204009A9A01007E780100049B01000200030099
:1082140002000100419B01008E9B0100DD9B0100D7
:1082240001001000109C01004E9C0100034610B593
:108234000A4619790123006803FA01F143680469C5
:108244001B6819420ED10E4940F2A2630D4A0E4832
:108254000CF0BEFB0D480CF0BBFB40F2A2610948D8
:108264000CF0ADFB2368194218BF82F0010222B161
:108274008368DB68BDE81040184783681B69F9E729
:10828400109C01009A9A01007E7801004E9C010026
:1082940010B500210548FFF7C9FF044618B1044989
:1082A40004480DF07DFC204610BD00BFD4730100CE
:1082B400609C0100D46E010010B500210748FFF74F
:1082C400B5FF044618B9BDE81040FFF7E1BF044903
:1082D40004480DF065FC204610BD00BFDC730100AE
:1082E4007A9C0100D46E010010B500210548FFF707
:1082F40023FF044618B1044904480DF051FC2046FC
:1083040010BD00BFDC730100929C0100D46E01001B
:1083140010B500210748FFF70FFF044618B9BDE860
:108324001040FFF7E1BF044904480DF039FC204632
:1083340010BD00BFD4730100AE9C0100D46E0100D7
:10834400F8B50123184C1370254600230139014464
:108354002768B84210D36668B0420DD8B9420BD32F
:10836400B14209D8032B13D1002313700F4A002004
:10837400126882F828300AE001330B2B04F10C0454
:10838400E6D10B490B480DF00BFC4FF0FF30F8BD64
:108394004FF49072DA40D20701D50749F2E70C2274
:1083A40002FB03531B7AE1E710010020D0250020D3
:1083B400CB9C0100D46E0100089D01002DE9F84317
:1083C4000646884600AF474D28460DF092FE034608
:1083D400C8B96C4688B029686A464348CDE90501A6
:1083E4004FF40071ADF81C10404942F8101F4FF4CF
:1083F400E2513F48F9F7EEFFA5466FF0120420461C
:10840400BD46BDE8F8834FF480313A48FFF794FE47
:10841400044630B11723384A012135480CF0F8FCE2
:10842400EDE7D5E90129D9F818402B691CB3126886
:1084340012020ED4314940F2A533314A31480CF0CE
:10844400C7FA31480CF0C4FA40F2A5312C480CF0BC
:10845400B6FA1B684FF0A07213F4000F14BF4FF06C
:1084640000734FF0806317212846A047044628B1C3
:108474001723264AD0E76FF05704F9E766B9244971
:1084840040F2EC631E4A1F480CF0A2FA21480CF09B
:108494009FFA40F2EC61D9E7B8F1000F0CD11E4904
:1084A40040F2ED63164A17480CF092FA1B480CF0A0
:1084B4008FFA40F2ED61C9E74FF40003C6F8048077
:1084C400B360D9F81C304BB1012231462846984795
:1084D4000446002893D01723114A9DE76FF05704F0
:1084E400F9E700BF606B01002A9D01000300000151
:1084F400D46E0100E4730100489D0100109C01004A
:108504009A9A01007E7801004E9C01006C9D010046
:10851400419101009D9D010050990100C39D0100FE
:10852400F19D010038B5002105460E48FFF704FE11
:10853400044638B117230C4A01210C480CF068FC9E
:10854400204638BD0A488368DB6943B12246294680
:10855400984704460028F3D01723064AECE76FF047
:108564005704F9E7E47301001B9E0100D46E010077
:10857400606B01003C9E010098B500AF224C204680
:108584000DF0B7FD0346B8B921686C4688B06A4659
:108594001E48C2E905014FF4007191831C4942F859
:1085A400101F4FF4E2511B48F9F714FFA5466FF072
:1085B40012042046BD4698BD20460DF09AFD0346A0
:1085C40028B921686C4688B06A461348E1E7134924
:1085D4001348FFF7B1FD044620B112490D480DF0D0
:1085E400DFFAE6E74FF4B0110F48FFF7A5FD0446A4
:1085F4000028DED00D4907480DF0D2FA00210848C2
:10860400FFF79AFDD5E700BF606B0100699E01008A
:1086140003000001D46E0100849E010000031600D3
:10862400D4730100A09E0100DC730100C49E01000C
:1086340073B514460E460DF1070221460546FFF7B1
:108644007FFE70B9094B9DF807201B683AB15B693E
:1086540022463146284602B0BDE8704018471B69DF
:10866400F6E74FF0FF3002B070BD00BFD425002004
:10867400014800F017BD00BF9401002001460148E5
:1086840000F0E4BA9401002001480DF0E9BA00BFFB
:1086940094010020014800F079BA00BF9401002041
:1086A40010B5FFF7F7FF041E05DA044904480DF07E
:1086B40077FA204610BD0024FBE700BFE79E0100C7
:1086C400D46E010010B50120FFF7D8FF044628B18D
:1086D400074908480DF064FA204610BDFFF7D4FF9F
:1086E400041E01DA0449F4E7BDE81040FFF7D8BFDF
:1086F400FB9E0100D46E01000F9F01004FF48073B4
:1087040007B504220193054B0DEB02011B680448D5
:10871400DB689847002003B05DF804FBD4250020F3
:10872400208C04001FB504225C2003A9FFF780FFFE
:10873400044630B109490A480DF032FA204604B023
:1087440010BD039A074B9A42F8D0012100920448C5
:10875400054A0CF067FB4FF0FF34EFE7239F01005D
:10876400D46E010020000042479F010098B500AF7D
:10877400FFF7DEFC374B1860FFF7D6FC364B18606A
:10878400364C20460DF0B5FC0346B8B921686C465A
:1087940088B06A463248C2E905014FF400719183FA
:1087A400304942F8101F4FF4E2512F48F9F712FEF6
:1087B400A5466FF012042046BD4698BD20460DF034
:1087C40098FC034628B921686C4688B06A46274855
:1087D400E1E727492748FFF7AFFC044620B12649C3
:1087E40021480DF0DDF9E6E74FF400312348FFF7A7
:1087F400A3FC044640B122491B480DF0D1F90021E5
:108804001C48FFF799FCD6E701211A48FFF70EFD33
:10881400044630B11B4914480DF0C2F9FFF778FD46
:10882400C9E70021212005F00FF901211348FFF7C2
:10883400FDFC044640B114490B480DF0B1F9002188
:108844000C48FFF7F3FCE9E70021212005F0FCF8D0
:10885400B1E700BFD4250020D0250020606B0100C3
:10886400699E010003000001D46E0100849E010092
:1088740000030200D4730100A09E0100DC73010018
:10888400C49E0100609C0100839F010008B5FFF7AE
:1088940013FD30B9FFF73CFD18B9024B1860024BC9
:1088A400186008BDD4250020D025002038B9044B19
:1088B4001B685B791BB101F130000DF086B970477C
:1088C4000C260020074B1B685B794BB140B9064B63
:1088D4004FF0FF3218694FF0FF3330300DF077B9A5
:1088E400704700BF0C2600209401002070B5046975
:1088F4000546124E20460DF06CF904F148000DF0C7
:1089040064F93378BBB922460D490E4801F012FFD1
:108914000D4B0E4A1B68D2F840161B7904460B43D4
:10892400C2F84036B0FA80F35B09337028460DF084
:1089340062F9204670BD0024F8E700BF9A2C00209D
:10894400B1880000D82500200C26002000B0025079
:10895400F0B5064685B0A9B14D68C5B1D5E9005357
:108964008868B0B1D0E90070A0B19BB1984209D138
:10897400581C09280B7810D902210090144A154874
:108984000CF050FA6FF01504204605B0F0BD2B46EC
:10899400E6E7074601331844EBE78DF8083040F268
:1089A4000113ADF80A3000238DF8090030698DF801
:1089B4000C308DF80D200DF00CF93A46294602A82A
:1089C40001F0E6FE044630460DF015F9DCE700BF81
:1089D400A79F0100D46E01007FB5FF238DF80330FB
:1089E4000DF10303002201930123CDE90232052393
:1089F40003A98DF80C30064801AB04920593FFF7E8
:108A0400A7FF0028A8BF9DF8030007B05DF804FB8A
:108A14009401002038B5044600690DF0DAF82569A0
:108A24000022002305F148000DF0D1F82B6D4BB165
:108A34002046BDE838400DF0DEB840F26760002102
:108A440005F002F801F012FF05460028F5D101F007
:108A540041FF014B1D70EBE79A2C00202DE9F74FE5
:108A6400404D0746284689461646FFF73FFF044611
:108A740000286DD128690DF0ACF87B4203F00303A4
:108A840007F0030558BF5D426D4205F00305B5428A
:108A940028BF3546D9F1000303F0030309F0030AA4
:108AA40058BFC3F1000ACAF1000A0AF0030AB2452A
:108AB40028BFB246731BA6EB0A0626F0030623F072
:108AC4000308B045C8BFB04603F0030BC8BFA3EB0F
:108AD400060BB8F1000F12D009EB0A0641463046E6
:108AE4007A190DF0FFFA0446FFF7ECFE6CBB55450E
:108AF40005D04246314609EB05000DF015FF85B15E
:108B0400C5F1040604216846BA1B0DF0EBFA0446CD
:108B1400FFF7D8FECCB92A4648460DEB06010DF006
:108B2400F6FEBBF1000F1AD07A19082168464244B8
:108B34000DF0D8FA0446FFF7C5FE34B908EB05007A
:108B44005A46694648440DF0E2FE06480DF053F8D3
:108B54000448FFF75FFF204603B0BDE8F08F5C4692
:108B6400F3E700BF9401002008B501F0E3FD054BD5
:108B7400054A1B68D2F840161B7900200B43C2F843
:108B8400403608BD0C26002000B00250002373B507
:108B940006460A258DF8073030460DF107010DF021
:108BA40073F8044660B99DF807309A0708D59DF814
:108BB400070083070CD501220A4B83F823200EE01B
:108BC4002120002104F040FF013DE5D1002CEED02E
:108BD40005480121054A0CF012F94FF0FF3002B0AC
:108BE40070BD00BFD8250020D46E0100CA9F0100CB
:108BF40030B589B00DF10703012203930023CDE9B9
:108C0400042307933F238DF8143003AB05468DF8F6
:108C140007100693FFF76AFE044628B9024605A921
:108C24002846FFF795FE04462846FFF7F3FE002C7E
:108C340005DA01212346034A03480CF0E9F82046EB
:108C440009B030BDEB9F0100D46E01000B22024B32
:108C540083F82320FFF7CCBFD825002008B501F006
:108C640089FE10B10248FFF7D5FE002008BD00BF01
:108C7400940100202DE9F04786B0DFF85C81C379C8
:108C840000AFC8F80000002B58D0042303228270E0
:108C940043700021514807F10C020CF0F0FC041E53
:108CA40040DBFB684E4A19791868FDF77BF8041E0F
:108CB40038DB0125002201212B20FAF797FB494BD1
:108CC400494ED3F810A0D8F80030002486F8295073
:108CD40086F82A504FF0502983F828504FF44173F6
:108CE4003460F48386F82350B383348486F82240B6
:108CF400C9F8B85520460DF0F8F9524630463B49BC
:108D0400FFF732FF0223C9F8B83520460DF0EDF91C
:108D1400FFF762FE041E13DA354A23462946354816
:108D24000CF076F8D8F800000C30012211460DF052
:108D340059FA20461837BD46BDE8F0871A46A6E71B
:108D4400737FE4B2023B012B05D9357F033D012D2E
:108D54008CBF00250125C4F38013AB422E4619D0E5
:108D6400FB1C01227B60002384F04004C7E902233A
:108D74007B611C483B1D07F10C01FC703A733B619D
:108D8400FFF7E6FD041E0AD1FFF726FE041E07DBEB
:108D9400E307F9D41348FFF73DFE0024C2E7C1DA24
:108DA400154A164B6D468AB0002E18BF13466A4604
:108DB40013490794CDE905134FF40073ADF820303F
:108DC400104B42F8103F00234FF411510948F9F7B2
:108DD40001FBAD46A6E700BF0C260020EC730100A2
:108DE40000B0025094010020D8250020B188000072
:108DF4000AA00100D46E010042B4010004A00100E5
:108E04001AA001000400000110B50B4B1B681B7A6B
:108E14008BB10A4C236803B13AB1094A1368013390
:108E24001360084AC2F8983502E004339842F4D13A
:108E340001440439216010BD0C26002008260020BE
:108E44000426002000B00250F8B541EA00031343A1
:108E54009B0700AF00F0030601F0030526D06C4623
:108E64008EB0003E18BF0126003D18BF012512F048
:108E7400030218BF01220B924FF40072ADF83020A8
:108E84006A46DFF82CC00B4BCDF814C0DFF828C0BD
:108E94000891CDE906C009960A9542F8103F0023CF
:108EA40044F240410548F9F795FAA546BD46F8BD98
:108EB4002BA0010008000001FD620200D46E010035
:108EC4002DE9F743804615468946304FFFF7BCFF2E
:108ED40038684FF0FF32436A0C3048EA03084FF019
:108EE400FF330CF074FE002229464046FFF78CFF46
:108EF400B9F1000F46D0002D44D0042D01D9AB07A1
:108F040040D118F0030F3DD1214E3046FFF7EEFC5F
:108F1400044648BB4FF0FF324FF0FF3330690CF08A
:108F240056FE30690CF055FE032D424627D8042125
:108F34000DEB01000DF0D6F80446FFF7C3FC6CB945
:108F44002A46494601A80DF0E2FC042142460DEBF5
:108F540001000DF0C4F80446FFF7B4FC0C480CF013
:108F64004AFE30690CF031FE0948FFF753FD3868BA
:108F74000C300CF02AFE204603B0BDE8F0832946ED
:108F84004846E6E76FF01504F1E700BF0C26002021
:108F940094010020F8B5054614460E46104FFFF71D
:108FA40053FF38684FF0FF32436A0C301D434FF0D3
:108FB400FF330CF00CFE002221462846FFF724FF65
:108FC4005EB124B122463146FFF748FD04463868B5
:108FD4000C300CF0FAFD2046F8BD6FF01504F6E7EE
:108FE4000C2600202DE9F04F87B04FF0040ADFF87B
:108FF400A0908046D9F800B00D469BF8284000AFF9
:10900400A6000AEB8404142C1ED96D468AB06A4665
:10901400204B0593204BCDE90634142308934FF4D9
:109024000073ADF824301D4B42F8103F00234FF479
:1090340031511B48F9F7CEF96FF00B04AD462046C9
:109044001C37BD46BDE8F08F22460021381D0DF0C7
:1090540084FC4FF0FF334FF0FF320BF10C000CF0A7
:10906400B6FD012251464046FFF7CEFE2246391D89
:10907400FFF7F4FC0446D9F800000C300CF0A5FD11
:1090840006F11803DE1956F8143C2B60D7E700BF2D
:109094000C26002051A00100EF620200050000012F
:1090A400D46E010030B587B00DF1030200230192A4
:1090B40001228DF80330CDE9022305933F238DF877
:1090C4000C3001AB05460493FFF710FC044628B9A5
:1090D400024603A92846FFF73BFC04462846FFF74F
:1090E40099FC002C05DA01212346034A03480BF0BE
:1090F4008FFE204607B030BD9BA00100D46E010056
:1091040008B50CF0FDFD58B1614BD3F8202A3AB9EB
:109114000D21C3F8201A0121C3F81C19C3F81C2916
:109124000022D30003F57F03D3F80013013107D0E5
:10913400D3F800130132D3F80433202A0B60F0D1A2
:109144000CF0DEFD002840F09A800CF0D9FD40B10F
:10915400504B514AC3F830254FF050230122C3F835
:1091640058254FF47F03D3F83021D3F83431072A3C
:1091740006D1023B012B9EBF0022484BC3F84C256D
:109184000CF0BEFD50B14FF05023D3F80024D107AA
:1091940042BF0022C3F81421C3F818214FF47F03FF
:1091A400D3F83021D3F83431072A09D14FF05023B2
:1091B400D3F80024D20744BF6FF00102C3F800249F
:1091C4000CF09EFD18B16522314BC3F80C274FF407
:1091D4007F03D3F83021D3F83431072A16D12F4B2B
:1091E400D3F82034002B11DA4FF050230322C3F8B4
:1091F400182501229A60D3F80421002AFBD000220A
:10920400C3F804210122DA60C3F818254FF47F0360
:10921400D3F83021D3F83431072A20D1023B022B72
:109224001DD97E221A4B1B49C3F80C27C3F83C29CD
:109234007F231B4AC2F818310023C1F8043EC1F849
:10924400083E01F54821C1F81031C2F82431C2F8B2
:109254002C3102F5FF1202F58052C2F8A032114AF5
:10926400D2F88C3043F44063C2F88C300E4A0F4B72
:109274001168C3F84415D269C3F84C2508BD2922E6
:10928400034BC3F80C270322C3F83C275DE700BF58
:1092940000400050009003504400EFBE00200350F3
:1092A4000020005000ED00E00080FF00006000504E
:1092B400014B1860704700BF1026002010B50B4BFF
:1092C4001446186858B90A490A4840F2F3130A4A7E
:1092D4000BF07EFB40F2F31107480BF070FB0CF02F
:1092E40021FD0028A4BF2070002010BD10260020FE
:1092F400F2A001007E780100B5A001000123024A1A
:109304008340C2F80435704700700150014B0020BF
:109314001B68184714260020014B1B68184700BF20
:1093240014260020014B09201B681847142600202E
:10933400014B08201B6818471426002010B5144C54
:10934400237913BB01232371124B0028206018BF1B
:10935400184600F0BDF8D0B923680F48002B08BFA9
:10936400184600F097F990B923680C48002B08BF01
:10937400184600F003FA50B923680948002B08BFC7
:109384001846BDE8104000F015B96FF0770010BD25
:109394001426002011930000299300001D9300005F
:1093A4003593000008B50C4B1A794AB90B490C489F
:1093B400B1230C4A0BF00CFBB1210A480BF0FFFA65
:1093C4001B6843B10520FAF703F820B9BDE808404B
:1093D4000520F9F7DBBF08BD1426002045A10100D4
:1093E4007E78010008A1010008B5174B1B795BB911
:1093F400164940F20513164A16480BF0E9FA40F2F2
:10940400051113480BF0DBFA032813D8DFE800F04A
:1094140002060A0EBDE8084000F0C2B9BDE80840E3
:1094240000F068B8BDE8084000F046B9BDE808405F
:1094340000F0CEB808494FF49273054A05480BF082
:10944400C7FA4FF49271DCE71426002045A101000D
:1094540008A101007E7801003DA4010008B5174B66
:109464001B795BB9164940F22B13164A16480BF0C8
:10947400AFFA40F22B1113480BF0A1FA032813D8CA
:10948400DFE800F006020A0EBDE8084000F060B80C
:10949400BDE8084000F0DAB9BDE8084000F03CB986
:1094A400BDE8084000F0C4B808494FF4A573054A64
:1094B40005480BF08DFA4FF4A571DCE71426002063
:1094C40045A1010008A101007E7801003DA401002E
:1094D400074B0246187938B91A6001221A714FF005
:1094E4005023C3F8142570476FF07700704700BF0E
:1094F4001C26002008B512490B794BB911491248B2
:109504007723124A0BF064FA772110480BF057FACC
:109514004FF050230022C3F80021D3F80021012288
:109524001A60096811B1C3F8042308BDD3F80021F7
:10953400002AFBD00022C3F80021D3F80031F4E75D
:109544001C26002045A101007E78010063A10100D2
:1095540008B5084B1B794BB9074908488923084AC1
:109564000BF036FA892106480BF029FABDE80840C9
:109574000CF035BC1C26002045A101007E780100BA
:1095840063A101004FF05023D3F80423D2070DD573
:10959400D3F8002152B10022C3F80021D3F80021EE
:1095A4000122C3F80823024B1B681847704700BF09
:1095B4001C260020054B0246187918B91A600122AE
:1095C4001A7170476FF07700704700BF242600209F
:1095D40008B5134A13794BB9124913486123134A46
:1095E4000BF0F6F9612111480BF0E9F94FF0502323
:1095F4000021C3F82011D3F82011012199611268C8
:1096040022B14FF48072C3F8042308BDD3F820219B
:10961400002AFBD00022C3F82021D3F82031F4E73C
:109624002426002045A101007E780100A6A10100A6
:1096340008B5084B1B794BB9074908487323084AF6
:109644000BF0C6F9732106480BF0B9F9BDE80840E0
:109654000CF0E1BB2426002045A101007E78010026
:10966400A6A101004FF05023D3F80423D2050ED550
:10967400D3F820215AB10022C3F82021D3F82021A5
:109684004FF48072C3F80823014B1B6818477047D6
:1096940024260020074B0246187938B91A600122A3
:1096A4001A714FF05023C3F8802570476FF077008C
:1096B400704700BF2C26002008B5134A13794BB914
:1096C400124913486723134A0BF082F967211148A2
:1096D4000BF075F94FF050230021C3F82411D3F88F
:1096E400241101211962126822B14FF40072C3F8E7
:1096F400042308BDD3F82421002AFBD00022C3F898
:109704002421D3F82431F4E72C26002045A10100BC
:109714007E780100EEA1010008B5084B1B794BB916
:10972400074908487923084A0BF052F97921064879
:109734000BF045F9BDE808400CF087BB2C2600204F
:1097440045A101007E780100EEA101004FF05023F5
:10975400D3F8042392050ED5D3F824215AB100225C
:10976400C3F82421D3F824214FF40072C3F808234A
:10977400014B1B68184770472C260020074B0246F4
:10978400187938B91A6001221A714FF05023C3F8BE
:10979400182570476FF07700704700BF342600200B
:1097A40010B5264C23794BB925492648E523264A8A
:1097B4000BF00EF9E52124480BF001F94FF050238A
:1097C400D3F81814D3F81824C9031BD502F00302E4
:1097D400022A02D0012A12D101224FF05023C3F8E9
:1097E40018250022C3F80421D3F8042101229A6029
:1097F4002268A2B9D3F80421002AFBD017E00CF0A8
:109804003EFBE9E7D3F81424D207E5D5D3F81C24AA
:1098140002F00302013A012AF1D822681AB10222A5
:10982400C3F8042310BDD3F80421002AFBD000227E
:10983400C3F80421D3F80431F4E700BF3426002030
:1098440045A101007E78010035A2010008B5094B4D
:109854001B795BB9084909484FF49173084A0BF026
:10986400B7F84FF4917106480BF0A9F8BDE8084029
:109874000CF005BB3426002045A101007E780100D0
:1098840035A20100F8B54FF0502301250026D3F886
:1098940004431E4F04F0820404B9F8BDB4FA84F002
:1098A400C0F11F00830003F580739BB203F15023C2
:1098B40005FA00F2196892B224EA02040029EBD0F6
:1098C4001E601B684FF05023022AC3F8082311D1ED
:1098D400D3F81814D3F8181401F00301012903D0A4
:1098E4003B68C0B29847D7E7C3F81825C3F80423E8
:1098F4009960D1E7064907484FF4F573064A0BF01F
:1099040067F84FF4F57104480BF059F83426002039
:109914003DA401007E78010035A20100034A4309F9
:10992400D35C00F01F001844C0B270470D630200FE
:1099340010B504460846FFF7F1FF04EB4000838AA4
:10994400DA051CD5C3F3432123F4F853838204F1CD
:10995400120204F1720032F8023F13F4807F03D044
:10996400C3F3432399420AD09042F4D1002204EB7A
:10997400C1035A6004F178000CF0EEF900B910BD8F
:10998400054906484FF4DB73054A0BF021F84FF400
:10999400DB7103480BF013F8627B01007E78010051
:1099A40078A2010008B50268014610460CF080FA5E
:1099B40058B910494FF482630F4A10480BF008F865
:1099C4004FF482610C480AF0FAFF02F01F035209B7
:1099D4000B600BD0012A0BD0094940F21943064A07
:1099E40006480AF0F5FF40F21941EBE7054808BDC7
:1099F4000548FCE7E9890100B68901007E78010089
:109A04003DA401000025845000288450072808B58F
:109A14000BD90849084840F2A733084A0AF0D8FF8E
:109A240040F2A73105480AF0CAFF800000F58070B3
:109A340008BD00BFEBA201007E780100B6A20100C0
:109A4400024611F0010010B50BD18B07C1F34000A1
:109A54000DD50749086A50600862003818BF012014
:109A640005E0044C236A13602362002BEDD010BD83
:109A74000028845000258450F7B504460846FFF7B3
:109A84004DFF04EB4006B38A0D46DB072AD520467A
:109A94000CF000FB294620460CF01CFA50B120467D
:109AA4000CF047FA0023276807EB8000C0F8103554
:109AB400C0F81035204600242946FFF739FFB48248
:109AC40001A80195FFF76EFF019B00EB8300D0F81E
:109AD4000022064B134043F00203C0F80032204634
:109AE40003B0F0BD6FF01500FAE700BFF0F0FCFF23
:109AF4002DE9F0430E461746044685B058B95A4935
:109B04005A4840F25E435A4A0AF062FF40F25E410C
:109B140057480AF054FF0846FFF700FFD7F80080C3
:109B24000546B8F1000F19D020460CF0F7F918BB20
:109B34004346CDE900008DF80E008DF80F000DF1BD
:109B44000F0230460DF10E010CF01CFA04EB450235
:109B5400938A23F0020343F0010393827B689BB34F
:109B64003146204693F80080D3F804900CF0CBF9EA
:109B740028B1B9F1000F1FD06FF0150027E004EBF6
:109B84004500838A23F4604323F020038382B9F1E0
:109B9400000F11D0B8F1030FEED87B6821685B6821
:109BA40093F800C04FEA8C031944B8F1000F11D1A7
:109BB400C1F81085C1F8108504EB4502938A23F09F
:109BC4001C0343EA88039382BB6843BB002005B0AF
:109BD400BDE8F083D1F8102522F00302C1F8102566
:109BE40022681344D3F8102522F44F3222F4407231
:109BF400C3F810253202D3F8101502F47C5242EA5D
:109C040008420A43C3F8102504EB4C03A3F87C6014
:109C1400838A43EA4C3343F020038382CCE7314602
:109C2400D3E900782046FFF783FE002FCED0636887
:109C34009F4206D004F178000CF074F8002804DA8E
:109C4400C5E7A3689845F5D1002004EBC003C3E938
:109C5400017804EB4505AB8AC0B243EA402343F4E0
:109C64008073AB82B2E700BFF5A201007E780100E9
:109C740078A201002DE9FF410C4616461F46054611
:109C840058B93C493C484FF48D633C4A0AF0A0FE65
:109C94004FF48D6139480AF092FE0846FFF73EFE04
:109CA400804616B328460CF02EF918B928460CF055
:109CB40011F908BB214628460CF017F910B1737846
:109CC400012B19D001238DF80F300023721CCDE92C
:109CD40000632046B31C0DF10F010CF053F905EBA2
:109CE4004802938A43F003039382002F3FD0214616
:109CF40028460CF008F920B96FF0150004B0BDE84F
:109D0400F08100223E782B6805EB480003EB8603C4
:109D1400C3F81025C3F81025838A4FEA860C23F470
:109D2400604323F020038382797801B32A68BF78E3
:109D34006244D2F81035090423F4991323F4F85338
:109D4400C2F81035230201F4403103F47C530B4371
:109D54003905D2F8105501F480110B432B43C2F896
:109D64001035838A43EA463343F02003838200207C
:109D7400C4E700BFF5A201007E78010078A20100CB
:109D840008B558B90749084840F27143074A0AF030
:109D94001FFE40F2714105480AF011FEC0E90312AA
:109DA40008BD00BFF5A201007E78010078A2010081
:109DB40070B51546044658B9134940F27A43134A1C
:109DC40013480AF005FE40F27A4110480AF0F7FD04
:109DD4004AB9104940F223330C4A0D480AF0F8FD01
:109DE40040F22331F1E70CF075F848B10846FFF76B
:109DF40095FD04EB40040020A38A5B0B2B7070BD1F
:109E04006FF01500FBE700BFF5A2010078A2010086
:109E14007E78010000A30100F8B5044658B9194939
:109E240019484FF49163194A0AF0D2FD4FF4916135
:109E340016480AF0C4FD90F88C5090F88D70F5B96E
:109E44006022294614300CF088FD114B266853F823
:109E54003770AF420ED1002546F30730C6F87C5167
:109E6400D6F87C31F9F792FA0123284684F88C302D
:109E7400A367F8BDE8B2FFF7C9FD0135E9E76FF064
:109E84007700F6E7F5A201007E78010078A20100D0
:109E94001874010008B558B90849094840F28F43BD
:109EA400084A0AF095FD40F28F4106480AF087FD02
:109EB40090F88C00003818BF012008BDF5A20100FD
:109EC4007E78010078A2010008B558B9074908480E
:109ED40040F29D43074A0AF07BFD40F29D4105484C
:109EE4000AF06DFDBDE80840FFF7C6BDF5A201000C
:109EF4007E78010078A2010008B558B90A490B48D8
:109F040040F2A4430A4A0AF063FD40F2A44108481F
:109F14000AF055FD074B90F88D0003EB8000BDE877
:109F240008400BF019BF00BFF5A201007E780100C4
:109F340078A201001402002010B50C4658B90C494F
:109F44000C4840F2AB430C4A0AF042FD40F2AB41EC
:109F540009480AF034FD094B90F88D0003EB8000AA
:109F64000BF0E0FE0028A4BF2070002010BD00BF4D
:109F7400F5A201007E78010078A2010014020020FD
:109F84002DE9F3410D461646044658B938494FF4B5
:109F9400A563384A38480AF01BFD4FF4A5613548DB
:109FA4000AF00DFD0BF0A1FF48B9344940F23543E6
:109FB400304A31480AF00CFD40F23541EFE72046C3
:109FC4000BF088FF2768F8B120460BF09CFF804611
:109FD400D0B920460BF0ADFF0546FFF717FD47F853
:109FE40000803B58236803EB8503D3F8102542F027
:109FF4000102C3F8102526B101232268AB40C2F840
:10A00400043302B0BDE8F081D7F80433002BA4BFB9
:10A014004FF00043C7F804334EB9194940F24F4397
:10A02400144A15480AF0D4FC40F24F41B7E72846D9
:10A03400FFF774FC04EB4004A38AC3F38203042BEC
:10A0440011D0052B11D001A80195FFF7ABFC019BA2
:10A054000169D94001F001010231284602B0BDE88E
:10A06400F0410BF0DCBF0321F7E70221F5E700BF65
:10A07400F5A2010078A201007E7801000AA3010084
:10A084002BA3010008B558B90749084840F22F53DB
:10A09400074A0AF09DFC40F22F5105480AF08FFC54
:10A0A400BDE808400BF0F6BFF5A201007E78010080
:10A0B40078A201002DE9F04F07468DB058B97349D5
:10A0C400734840F25C63734A0AF082FC40F25C61BC
:10A0D40070480AF074FC804658F804AB90F88D4040
:10A0E400DAF804136C4BC9B2504653F8342041F0EB
:10A0F40000410BF0A3FF051E39DA0023CDE90A3332
:10A10400654BE60003EBC40463680AA8194601938F
:10A11400FFF796FC331D04934FF0000B5F4B0DF1DA
:10A1240028090393039A5C4912F8013B0392049AA9
:10A1340002EBD3028A5C03F0070322FA03F3DB0782
:10A144001BD40BF10103022B4FF0010B09F104099D
:10A15400E8D14FF00041002250460BF06FFF019907
:10A164000AA8FFF76DFC0028D6D125F0004501248C
:10A17400002D74D10DB0BDE8F08F494B5B440593BD
:10A18400D9F800100029DCD091FAA1F1B1FA81F1DB
:10A19400059B1C7841EA44142046FFF7BFFB07EBFC
:10A1A4004000828AC808C2F38203CDE906230293E1
:10A1B400012319F8006001F0070103FA01F126EA0E
:10A1C400010109F8001009A80994FFF7EBFB0999AC
:10A1D400069A803150F8216012F0100F079BC6F3E5
:10A1E400014623D021464046029A0BF0ACFE09A852
:10A1F4000994FFF7D7FB099BF6B2803350F823305C
:10A20400C3F301439E4207D1002120460BF007FF10
:10A21400314620460BF003FF09A80994FFF7C2FB5F
:10A224000122099B02FA03F30362A9E7022E14BF79
:10A2340002210321204606930BF0F1FE069B032B1B
:10A2440003D0022E07D1012BE6D121464046029AC3
:10A254000BF079FEE0E7032EDED1022BF4E795FA4A
:10A26400A5F3B3FA83F304FA03F225EA020503F52E
:10A27400A2725AF8222007EB43034046B3F87C103D
:10A28400C2F301420BF05FFE72E700BFF5A20100CA
:10A294007E78010078A20100187401001D63020099
:10A2A4001D63020000220121054B83F83820054B71
:10A2B400C3F808131961C3F80025C3F800217047D7
:10A2C4003C26002000B0025070B5114D6C6BA4B157
:10A2D4004FF47A735C430A23B4FBF3F40D4ED6F8BF
:10A2E40000316BB995F8393053B90A200BF018FDD9
:10A2F400013CF4D16FF0730008E04CF25034EDE708
:10A3040095F8393003F0FF00002BF3D170BD00BF86
:10A314003C26002000B0025010B500220124094B55
:10A32400C3F80045C3F800211C6028B1FFF7CCFF37
:10A3340020B9054B83F83840002010BD6FF073003E
:10A34400FBE700BF00B002503C26002070B53A4C39
:10A3540094F8305005B148B9384939487623394A18
:10A364000AF036FB762137480AF029FB00F06046F4
:10A37400B6F1005F59D1860757D1012D05D09D4212
:10A3840056D194F83850002D52D000262E4D022B71
:10A394000BBFC5F81025C5F80425C5F81405C5F884
:10A3A40008050CBFC5F81815C5F80C1584F83960F4
:10A3B40026680CBF08250425BEB994F838306BB163
:10A3C4000022214B05F1A045C3F80021012305F526
:10A3D4002C352B60BDE87040FFF776BF0120FFF7F6
:10A3E4009BFF10F1740FEBD170BDA66826B1E0603D
:10A3F4006161E2610020F7E784F830300123A26153
:10A40400114AA0602161C2F80061C2F8043394F8D3
:10A41400382002F0FF0012B9FFF77EFFEAE705F1EA
:10A42400A04505F52C352B60E4E76FF00C00DBE765
:10A434006FF00F00D8E700BF3C26002072A3010094
:10A444007E78010036A3010000B00250084B9A68E0
:10A454005A621A699A629A69DA62DA689A6032B15F
:10A464005A691A61DA699A610022DA6070477047A2
:10A474003C26002010B5440914D0012C06D14FF617
:10A48400FF7300F01F00C340DB070ED410491148CE
:10A494004FF48263104A0AF09BFA4FF482610E482B
:10A4A4000AF08DFA4FF0FF33EBE70C4B0C4A012C0A
:10A4B40018BF1A4602EB8002D2F80002094B03408F
:10A4C40043EA012343F00203C2F8003210BD00BF87
:10A4D400E98901007E780100B689010000258450D5
:10A4E40000288450F0F0FCFF10B50E4B0238D3F86E
:10A4F4003C26D3F83836072813D8DFE800F0110FCC
:10A504000D0B0A080604100EC871100C8871100A8D
:10A5140048710A711A0ECA701A0C8A701A0A4A70A3
:10A524000B7010BD00B00250023807281FD8DFE8B6
:10A5340000F02927251123211F04CB791B068A79D2
:10A5440043EA02434A7943EA02230A7913430E4A4F
:10A55400C2F83C36CB781B068A7843EA02434A7831
:10A5640043EA02230A781343074AC2F8383670478D
:10A574000023E4E70023E5E70023E6E70023EBE715
:10A584000023ECE70023EDE700B0025038B590F863
:10A59400293004461BB190F82A20002A6FD1606844
:10A5A400FF2800F0BF80A168FF2900F0BB80E268AB
:10A5B400FF2A00F0B78025690E2D40F0B3801128E2
:10A5C40040F0B080122940F0AD800D2A40F0AA80FE
:10A5D4006269FF2A02D00F2A40F0A480A269FF2AF0
:10A5E40002D0102A40F09E80DBB903211120FFF72E
:10A5F40041FF0321A068FFF73DFF0321E068FFF757
:10A6040039FF20690321FFF735FF6069FF2802D075
:10A614000321FFF72FFFA069FF2802D00321FFF7D2
:10A6240029FF94F82A3053BB6268404BFF2A08BFC5
:10A634004FF0FF32C3F82425A268FF2A08BF4FF069
:10A64400FF32C3F82825E268FF2A08BF4FF0FF3223
:10A65400C3F830252269FF2A08BF4FF0FF32C3F840
:10A6640034256269FF2A08BF4FF0FF32C3F838254A
:10A67400A269FF2A08BF4FF0FF32C3F83C25636A82
:10A684002B4A2A49536394F8293082F83A302368D4
:10A69400C1F84035A37F657F207F9B0143EAC50352
:10A6A4000343E07F43EAC013C1F844354FF47F030A
:10A6B400D3F83001D3F8343107280ED1022B0CD053
:10A6C40094F82300D1F8443518BB43F44033C1F85F
:10A6D40044354FF4C063C1F84036144894F8203030
:10A6E400D0F8001621F07F4121F0FF010B4394F8CC
:10A6F400211043EA016394F8221043EA416394F879
:10A70400231043EA0173C0F80036136833B90020FC
:10A7140038BD23F4003343F48033D8E72B20F8F713
:10A7240035FEF4E76FF01500F2E700BF00B0025009
:10A734003C26002010B558B9114912484FF4D37380
:10A74400114A0AF045F94FF4D3710F480AF037F96A
:10A754000E4C94F8303063B9C4E90012FFF716FFC9
:10A7640050B90123C4E9020084F8303084F8380079
:10A7740010BD6FF07700FBE76FF01500F8E700BF3E
:10A78400BDA301007E78010036A301003C26002011
:10A794002DE9F041DFF8BC80054698F830000F46FB
:10A7A400144658B92C494FF4F8732C4A2C480AF033
:10A7B4000FF94FF4F87129480AF001F9012845D13D
:10A7C40098F838305BB30123264EC6F8083377BBBC
:10A7D400002788F83970C6F80071AB786A781B03D3
:10A7E40043EA02232A781343EA7843EA42332A7974
:10A7F40043EA82336A7943EAC233C6F83436FFF750
:10A8040063FD743018D12B796BB9174940F22223B8
:10A81400124A13480AF0DCF840F22221CBE7FFF792
:10A824007BFD7430CFD16FF07300BDE8F081394601
:10A834006878FFF779FECBE7C6F800710CB9002001
:10A84400F3E721466878FFF74FFEF8E76FF00F0053
:10A85400EBE700BF3C260020C6A3010036A301009D
:10A864007E78010000B00250F2A301001FB5144B22
:10A8740093F830305BB91349134840F2B723134AB5
:10A884000AF0A6F840F2B72110480AF098F800231D
:10A894000F4A02A802920DF1070211468DF8073003
:10A8A400ADF80C30FFF774FF30B99DF8073013F0A2
:10A8B400010F18BF6FF00F0005B05DF804FB00BF77
:10A8C4003C260020C6A301007E78010036A30100C7
:10A8D400050200012DE9F843214E96F830305BB9AA
:10A8E4002049214840F2D723204A0AF071F840F267
:10A8F400D7211E480AF063F82B20F8F755FDFFF71F
:10A90400D1FC96F83A3033BB194BD3F82405D3F86D
:10A914002895C0B2D3F83085D3F83475D3F83855B8
:10A92400D3F83C450BF0D8FB5FFA89F00BF0D4FB6D
:10A934005FFA88F00BF0D0FBEDB2F8B20BF0CCFB71
:10A94400FF2DE4B202D028460BF0C6FBFF2C02D048
:10A9540020460BF0C1FB002386F83030BDE8F883B5
:10A964003C260020C6A301007E78010036A3010026
:10A9740000B00250034B93F83000003818BF012098
:10A98400704700BF3C26002010B5224BD3F80021AD
:10A9940092B10022204CC3F8002194F8381094F8A6
:10A9A400302071B90121032A84F8381005D0042A13
:10A9B40005D0022A00D1996010BD5960FCE7D96026
:10A9C400FAE7032A19D0042A19D0022A04D1012350
:10A9D40084F82030FFF73AFDA36813B9012384F803
:10A9E400303094F8393003F0FF0013B9D4E9003162
:10A9F4009847002384F82030DEE70223E8E70322A7
:10AA040084F82020D3F81C256262D3F8203584F81A
:10AA14002830E1E700B002503C26002038B54369F5
:10AA240005463BB90024EA686042537843F00103C9
:10AA3400537038BD984704460028F3D000F1FF0353
:10AA4400FE2B0ED92123094A09490A4809F0C0FFFF
:10AA540029680948224609F0BBFF2121034809F06F
:10AA6400AEFFEB6844421C70DDE700BF04A40100A4
:10AA740027A401007E7801003FA4010010B504461C
:10AA8400F7F74CFB03480121034A0AF0B8F92046C2
:10AA94000BF03AFB9C6E010064A401002DE9F8431D
:10AAA40004460D4600AFEFF31188202383F3128888
:10AAB400BFF36F8F04283D4A98BF3D4BE9468AB0E7
:10AAC4009668117C98BF53F820306A4688BF394B8A
:10AAD400CDE9073140F201333748ADF82430374B24
:10AAE400CDE9050442F8103F00234FF431513448B6
:10AAF400F7F770FCCD4645B1EB69C3F3080323B106
:10AB04000121304A2E480AF07AF92EB130460BF072
:10AB1400E6FB08B1037803B92B48E9468AB06A46D4
:10AB24002A4B0790CDE9053640F20133ADF82030C9
:10AB3400274B42F8103F00234FF411512048F7F7F8
:10AB440049FC3246CD4629462046F9F7D3FB29462F
:10AB54002046FFF793FF042C0CD11E4987231E4A7D
:10AB64001E4809F035FF1E4809F032FF87211A48B4
:10AB740009F025FF85B1EB69C3F3080363B1022C27
:10AB84000AD018498E23144A144809F021FF1648A4
:10AB940009F01EFF8E21EAE788F31188BFF36F8F57
:10ABA4003046F8F7C9FCBD46BDE8F8837826002096
:10ABB4002874010073A4010089A4010005000001A8
:10ABC4009C6E0100B1A4010081A40100D2A4010083
:10ABD400040000010CA50100EAA401007E78010034
:10ABE40029A501003DA401005EA5010038B50A4B6A
:10ABF40053F82040013053F82050A54200D838BD06
:10AC0400606830B1037EDB0701D4FFF707FF083427
:10AC1400F3E723689847FAE73C740100012270B512
:10AC2400374B86B003201A70FFF7E0FFF9F78EFA6E
:10AC34000BF075FC0420FFF7D9FF324C324DAC42C7
:10AC4400264628D931494423314A324809F0C0FE06
:10AC5400314809F0BDFE44212D4809F0B0FE54F8F6
:10AC64000C3C059354F8103C049354F8143C03939F
:10AC740054F8183C029354F81C3C019354F8203CBB
:10AC8400009354E90A2354E90C0101F0A3FF54F89A
:10AC9400303C5E65D3E7AE4204F13004DFD302F00A
:10ACA40087FC184CAC421FD918496823184A194824
:10ACB40009F08EFE184809F08BFE6821CCE7D4E930
:10ACC4000A23B3F1FF3F08BFB2F1FF3F05D052EAB8
:10ACD4000301206803D102F007FF3034E2E70F4993
:10ACE400183003F031FAF8E7E9D302F0D3FCF5F7B2
:10ACF40033FC0B4A938923F00103938106B070BDA2
:10AD04009B2C0020F86D0100F86D0100FAA50100EC
:10AD1400D9A501007E7801009B7D0100A1D100002E
:10AD2400C80F00200023012270B586B0CDE90423AA
:10AD34000F220193CDE9023214234FF4A0720E4D79
:10AD44000E4E03FB00550E4906EBC016044602FBEB
:10AD540000110C4B3046009501F03CFF337C2C7401
:10AD640023F004033374084B013403EBC423EE6073
:10AD74006B6006B070BD00BF78260020480F00202D
:10AD840000E2002025B4000000DA00207FB5002096
:10AD9400FFF72CFF344B03F5006282F3088883F33A
:10ADA4000A88E023314C84F822300023E3772376A9
:10ADB4006376A37684F82030626A42F4E022626209
:10ADC40084F82330F8F748FAF8F7A0FB4FF0FF3384
:10ADD400A362E362F8F706FEF8F756FCF7F7CAF841
:10ADE400234801F0ADFF234B234A93420ED9234954
:10ADF400CC23234A234809F0EBFD234809F0E8FD5E
:10AE0400CC211F4809F0DBFD1C33EEE7FCD3F9F736
:10AE14006DF90120FFF7EAFE02201C4CFFF7E6FE65
:10AE240002F0F2FC1A4B00255C611A4B41F25042CD
:10AE3400059301231849CDE903532046174BCDE967
:10AE44000155009501F0C6FE0646237C204623F0FA
:10AE54000403237402F014F92846FFF763FF314614
:10AE640020460E4AF8F732FB00DA002000ED00E03D
:10AE740048100020286B0100D06B010027A60100B8
:10AE8400D9A501007E7801009B7D0100C80F002038
:10AE9400782600203FA6010040E3002021AC0000FA
:10AEA4002DE9F04F06468BB0DDE914A7CDE9051274
:10AEB4003B46524608A80BF096FADDE90834D04622
:10AEC400CDE90234B94606F11404EFF311852021CB
:10AED40081F31288BFF36F8F204603F0DBF860B96B
:10AEE4008423354A3549364809F072FD21463548F0
:10AEF40009F06EFD8421304835E0204603F0EEF879
:10AF0400EFF3058111B157EA0A0321D14FF0200B69
:10AF140006F10C0307933046DDE90512169B9847AA
:10AF2400074610B958EA09081FD1204603F0C0F8B3
:10AF3400002839D14FF499731F4A2349204809F056
:10AF440047FD2146214809F043FD4FF49971D2E7AA
:10AF54001F4958231F4A1A4809F03AFD1E4809F0B0
:10AF640037FD58211B4809F02AFDDDE9022308A812
:10AF74000BF05EFADDE908A729462046CDE900A7D3
:10AF8400079A02F053F9D046B946EFF311858BF3D3
:10AF94001288BFF36F8F204603F07CF800289FD0FF
:10AFA400204603F09BF8B6E785F31188BFF36F8F53
:10AFB40038460BB0BDE8F08F6B7B0100987B010035
:10AFC4007E780100AD7B0100C37B0100DA7B0100C8
:10AFD40069A6010047A60100C38E010038B50D4CD7
:10AFE4000D4DAC4213D90D4925230D4A0D4809F0E6
:10AFF400EFFC0D4809F0ECFC2521094809F0DFFCC1
:10B004002046D4E901120BF087F81834E9E7F7D3A6
:10B01400002038BD80030020E0030020AEA601001C
:10B0240047A601007E7801009B7D01001FB5054CF9
:10B03400CDE9002302940A460021FFF731FF04B052
:10B0440010BD00BF0349010030B54B1E0B4285B053
:10B054000CD00B4989230B4A0B4809F0B9FC0B4867
:10B0640009F0B6FC8921074809F0A9FC084BDDE981
:10B0740008450293CDE90045FFF712FF05B030BD46
:10B084006378010047A601007E7801009B780100E7
:10B09400410A0000F8B505460E4600F11404EFF32A
:10B0A4001187202383F31288BFF36F8F204602F0A9
:10B0B400F1FF68B984231B4A1B491C4809F088FC2A
:10B0C40021461B4809F084FC8421164809F077FCCA
:10B0D400204603F003F828463146F5F7F9FB05F15D
:10B0E4000C0002F049FB28B139462046BDE8F8407F
:10B0F4000BF043B9204602F0DBFF68B94FF49973B3
:10B10400084A0C49094809F063FC21460A4809F039
:10B114005FFC4FF49971D8E787F31188BFF36F8F01
:10B12400F8BD00BF6B7B0100987B01007E780100B5
:10B13400AD7B0100C37B0100DA7B010038B50E4C06
:10B144000E4DAC4212D90E49A2230E4A0E4809F004
:10B154003FFC0E4809F03CFCA2210A4809F02FFCF0
:10B1640020460AF0E3FF20B92034EAE7F8D30020B0
:10B1740038BD6FF01500FBE760030020800300205A
:10B18400ECA60100C7A601007E7801009B7D0100AA
:10B194002DE9F74305460F4691461C4600F1080683
:10B1A400EFF31188202383F31288BFF36F8F3046A7
:10B1B40002F070FF60B98423314A3249324809F001
:10B1C40007FC3146314809F003FC84212C4826E071
:10B1D400304602F083FF2B691BB33B601C68EB69AC
:10B1E4002C610133EB6114B96A6993421FD0EB6897
:10B1F400E41A09D4D5E905235A43A24204D9B4FB7D
:10B20400F3F203FB124494B12149F723214A1E4867
:10B2140009F0DEFB204809F0DBFBF7211D4809F0AB
:10B22400CEFB59EA040214D16FF00B043B603046A4
:10B2340002F03EFFF0B94FF49973114A17491248CE
:10B2440009F0C6FB3146164809F0C2FB4FF4997168
:10B25400BCE7CDE900942A464146304601F0E6FFBA
:10B26400044618B90F4B9B685B693B60204603B0EA
:10B27400BDE8F08388F31188BFF36F8FF6E700BF52
:10B284006B7B0100987B01007E780100AD7B01009F
:10B2940009A70100C7A6010085A70100C37B01001F
:10B2A400DA7B0100782600202DE9F843C3680546BF
:10B2B400CB1A0E4623D4D0E90512514399421ED924
:10B2C400B3FBF2F102FB1133CBB900F10807EFF342
:10B2D4001189202484F31288BFF36F8F384602F05B
:10B2E400D9FED8B98423414A4149424809F070FB48
:10B2F4003946414809F06CFB84213C480CE03F4945
:10B3040040F21F133E4A3B4809F062FB3D4809F0F6
:10B314005FFB40F21F113A4809F051FB384602F036
:10B32400DDFED5F81080B8F1000F40D1EFF31183A2
:10B3340084F31288BFF36F8F83F31188BFF36F8F89
:10B344005BB93149BB23314A2A4809F041FB3048F3
:10B3540009F03EFBBB212D48DEE72C68A54226D030
:10B364002CB3A3683BB92B49A423284A214809F0EC
:10B374002FFBA421EFE7D4E9003213605A60237C49
:10B38400C4E9008823F002032374C4F8088004F19C
:10B39400180002F0B5FF2046C4F87C80666101F015
:10B3A4006FFE49463846BDE8F8430AF0E6BF2B690C
:10B3B40038463360EB692E61013BEB6102F078FEA5
:10B3C40068B94FF49973094A13490A4809F000FB14
:10B3D4003946124809F0FCFA4FF499718DE789F364
:10B3E4001188BFF36F8FBDE8F88300BF6B7B01004A
:10B3F400987B01007E780100AD7B01003DA4010033
:10B40400C7A60100A0A70100EDA70100C2A7010083
:10B41400C38E010005A80100C37B0100DA7B010093
:10B4240008B50D4B9B6893F90E30002B09DB2024E3
:10B43400EFF3118384F31288BFF36F8F09F0B2FD29
:10B44400F6E7064906481C23064A09F0C1FA1C21FE
:10B45400044809F0B4FA00BF782600203DA8010092
:10B464007E7801001CA8010008B583684BB90B491C
:10B474000B48A4230B4A09F0ABFAA421094809F0AC
:10B484009EFAD0E9003213605A600023027CC0E9BE
:10B49400003322F002020274836008BD05A8010093
:10B4A4007E780100C2A701002DE9F74F04468846C3
:10B4B40092461F469DF83090EFF3058373B152EA2C
:10B4C40007030BD062499923624A634809F080FA62
:10B4D400624809F07DFA99215E4819E004F10805F3
:10B4E400EFF311864FF0200B8BF31288BFF36F8FAD
:10B4F400284602F0CFFD68B98423594A5949564871
:10B5040009F066FA2946584809F062FA8421544839
:10B5140009F055FA284602F0E1FD626A23699A426D
:10B524007BD2EFF311838BF31288BFF36F8F83F316
:10B534001188BFF36F8F5BB94C49BB234C4A464813
:10B5440009F046FA454809F043FABB214848DFE7C9
:10B554002768BC4217D0B7B13846FFF785FF07F11B
:10B56400180002F0CDFE4146E26878690BF0CFF98D
:10B5740000233846FB6701F083FD314628460AF074
:10B58400FCFE002458E0206A6769B84207D3A36927
:10B594005A1E904203D8E268191A914207D23549DB
:10B5A400B4232C4A2C4809F013FAB42194E7B9F1D6
:10B5B400000F28D041460BF0AAF9236AE26813442D
:10B5C400A2692362934201D163692362636A04F12D
:10B5D400280001336362102103F0BCF904460028FB
:10B5E400CBD1284602F064FD68BB4FF499731C4A22
:10B5F4002149194809F0ECF92946204809F0E8F9ED
:10B604004FF4997183E7E1698F4218BF0B46981A8A
:10B614004146E0610BF07BF9D8E75AEA07030FD003
:10B62400174B22469B683146C3F814802846CDE95F
:10B6340000A701F0FBFD0446204603B0BDE8F08FEF
:10B644006FF02204CDE786F31188BFF36F8FF3E721
:10B6540069A6010065A801007E780100C38E01007F
:10B664006B7B0100987B0100AD7B0100EDA701001D
:10B67400C2A7010087A80100C37B0100DA7B010097
:10B68400782600202DE9F7430446884617461D46D0
:10B69400EFF3058383B152EA05030DD060494FF4FB
:10B6A4009773604A604809F093F9604809F090F98B
:10B6B4004FF497715B4818E004F10806EFF3118921
:10B6C400202383F31288BFF36F8F304602F0E2FC2D
:10B6D40068B98423564A5749534809F079F93146E1
:10B6E400554809F075F98421514809F068F9304644
:10B6F40002F0F4FC636A002B67D0E2684046E1691B
:10B704000BF005F9E369E2681344A269E36193422B
:10B7140004BF6369E361636A013B6362EFF311830E
:10B72400202282F31288BFF36F8F83F31188BFF353
:10B734006F8F5BB94149BB23414A3B4809F048F943
:10B744003A4809F045F9BB213D48CEE72568AC42AB
:10B754004BD0002D4AD02846FFF786FE05F118008D
:10B7640002F0CEFD206A6369984207D3A3695A1E8A
:10B77400904203D8E2681B1A934209D231494FF42C
:10B78400A473284A284809F023F94FF4A47191E7D7
:10B7940069690BF0BCF8236AE26828461344A2697D
:10B7A4002362934204BF63692362636A0133636261
:10B7B4000024EC6701F064FC494630460AF0DDFDE4
:10B7C4002546284603B0BDE8F08357EA05031FD099
:10B7D4001D4B22469B684946C3F814803046CDE988
:10B7E400007501F023FD0546EBE70025304602F025
:10B7F4005FFC80B94FF499730D4A14490A4809F063
:10B80400E7F83146124809F0E3F84FF499716BE711
:10B814006FF02205EAE789F31188BFF36F8FD0E751
:10B8240069A6010065A801007E780100C38E0100AD
:10B834006B7B0100987B0100AD7B0100EDA701004B
:10B84400C2A7010087A8010078260020C37B01005D
:10B85400DA7B01002DE9F341044617461E46EFF357
:10B86400058565B154497323544A554809F0B0F825
:10B87400544809F0ADF87321504809F0A0F8EFF3EB
:10B884001188202383F31288BFF36F8F4E4802F090
:10B8940001FC60B984234D4A4D49494809F098F8A0
:10B8A40049494C4809F094F884214848E5E746485A
:10B8B40002F014FC484BE2689B6892B1A06898427D
:10B8C40027D057EA06022CD13F4802F0F1FB90B191
:10B8D40088F31188BFF36F8F6FF00F0002B0BDE8DB
:10B8E400F08193F90E100132C4E902323648216125
:10B8F40002F0DEFB78B94FF49973344A3749304883
:10B9040009F066F83049364809F062F84FF4997145
:10B91400CBE72169E7E788F31188BFF36F8F002035
:10B92400DCE793F90E1090F90E30994205DA99424A
:10B93400A8BF19460AF031FC054622464146CDE926
:10B944000076214801F072FC0028E8D0EFF311865C
:10B95400202383F31288BFF36F8F1B4802F09AFBF6
:10B96400002897D0184802F0B9FBA068C0B123683A
:10B9740021699C420AD04BB193F90E309942A8BF79
:10B9840019466FF07F039942B8BF19460AF005FCC7
:10B9940030B131460C480AF0F0FC6FF00A009DE724
:10B9A400002DF6D1084802F083FB0028A3D086F3CB
:10B9B4001188BFF36F8FF0E74FA901002DA9010093
:10B9C4007E78010061A90100982600206B7B0100AC
:10B9D400987B0100AD7B010078260020C37B010029
:10B9E400DA7B0100F8B50546EFF3058363B15549E9
:10B9F400EA23554A554808F0EBFF554808F0E8FF9C
:10BA0400EA21514808F0DBFF8368002B00F09480A2
:10BA1400504A9268934240F09280C3684BB94E49B1
:10BA24004FF48173484A494808F0D2FF4FF48171BA
:10BA3400E7E7012B03D0013BC3600020F8BDEFF31F
:10BA44001187202484F31288BFF36F8F434802F0D8
:10BA540021FB60B98423424A42493C4808F0B8FFBC
:10BA64003E49414808F0B4FF84213D48CAE73B48B9
:10BA740002F034FB2969A8680AF08FFBEFF3118305
:10BA840084F31288BFF36F8F83F31188BFF36F8F32
:10BA94005BB93649BB23364A2C4808F099FF354830
:10BAA40008F096FFBB213248ACE72C68AC4215D1B4
:10BAB40000232A48C5E9023302F0FAFA002836D1F5
:10BAC4004FF49973264A2C49204808F081FF2349F2
:10BAD4002A4808F07DFF4FF49971C6E7002CE7D09F
:10BAE400A3683BB92649A423214A184808F070FFEB
:10BAF400A421D8E70026D4E9003213605A60237CDD
:10BB0400C4E9006623F002032374A66004F118005C
:10BB140002F0F6FBAC6094F90E3020462B61E66728
:10BB240001F0AEFA39460D480AF027FC85E787F3A1
:10BB34001188BFF36F8F80E76FF015007EE74FF039
:10BB4400FF307BE74FA901002DA901007E78010099
:10BB540061A901007826002086A90100982600200A
:10BB64006B7B0100987B0100AD7B0100EDA7010018
:10BB7400C2A70100C38E0100C37B0100DA7B010070
:10BB840005A8010008B583684BB90B490B48A423E9
:10BB94000B4A08F01DFFA421094808F010FFD0E962
:10BBA400003213605A600023027CC0E9003322F0A3
:10BBB40002020274836008BD05A801007E780100BA
:10BBC400C2A701002DE9F04704460F4691469A4664
:10BBD4009DF8208000F10805EFF31186202383F3FC
:10BBE4001288BFF36F8F284602F054FA60B9842399
:10BBF400504A5149514808F0EBFE2946504808F094
:10BC0400E7FE84214B481DE0284602F067FAB8F1AC
:10BC1400000F00D06768EFF31183202282F31288AB
:10BC2400BFF36F8F83F31188BFF36F8F63B94549F7
:10BC3400BB23454A414808F0CBFE444808F0C8FEFF
:10BC4400BB21414808F0BBFE234653F80C8F9845AE
:10BC540019D0B8F1000F16D04046FFF793FF08F152
:10BC6400180002F04DFB00234046C8F87C30C8F8A9
:10BC7400149001F005FA314628460AF07EFB0024B0
:10BC84002046BDE8F087BAF1000F14D0082002F076
:10BC94009DFF002846D00122C0F80490026001688C
:10BCA40001F003015FB922680A4302606268206000
:10BCB4006AB960600BE04846C9F800A0EFE73A684B
:10BCC400032A24D801606168D9B9C4E9000004F1E9
:10BCD4001400042102F03EFE04460028CBD128467D
:10BCE40002F0E6F908BB4FF49973124A1849134855
:10BCF40008F06EFE2946174808F06AFE4FF4997161
:10BD040080E70A6802F0030202430A60D1E722F0E6
:10BD140003020A4302603A6802F0030240EA0203A3
:10BD24003B60D4E76FF00B04D9E786F31188BFF3C7
:10BD34006F8FA5E76B7B0100987B01007E78010083
:10BD4400AD7B0100EDA70100C2A70100C38E010075
:10BD5400C37B0100DA7B01002DE9F74306469046D8
:10BD64001F4600F10805EFF31189202383F312889D
:10BD7400BFF36F8F284602F08DF968B98423254AF2
:10BD84002549264808F024FE2946254808F020FEC7
:10BD94008421204808F013FE284602F09FF93468F5
:10BDA400FCB12368726823F00303944220464FF0E9
:10BDB4000101336008BF73600AF0FEF904462846A7
:10BDC40002F076F9E8B94FF49973124A1549134809
:10BDD40008F0FEFD2946144808F0FAFD4FF4997165
:10BDE400D7E758EA0703EAD049462846CDE9008751
:10BDF40006F10C0201F01AFA38B90C4B9B685C6925
:10BE040003E089F31188BFF36F8F204603B0BDE8C8
:10BE1400F08300BF6B7B0100987B01007E780100FA
:10BE2400AD7B0100C37B0100DA7B01007826002092
:10BE340008B583684BB90B490B48A4230B4A08F097
:10BE4400C7FDA421094808F0BAFDD0E90032136007
:10BE54005A600023027CC0E9003322F0020202741B
:10BE6400836008BD05A801007E780100C2A7010017
:10BE740070B50446EFF31186202585F31288BFF3CD
:10BE84006F8F334802F006F960B98423314A32498E
:10BE9400324808F09DFD2E49314808F099FD84216F
:10BEA4002C4818E02A4802F019F9EFF3118385F3BE
:10BEB4001288BFF36F8F83F31188BFF36F8F63B959
:10BEC4002849BB23284A254808F082FD274808F062
:10BED4007FFDBB21244808F072FD2568AC4212D0D6
:10BEE4008DB12846FFF7A4FF05F1180002F008FA07
:10BEF40000232846EB6701F0C3F83146BDE87040E3
:10BF040013480AF03ABAD4E902329A4218BF01330C
:10BF14000221A36004F1100002F01CFD0028ECD102
:10BF24000B4802F0C5F868B94FF49973094A1049EF
:10BF34000A4808F04DFD06490E4808F049FD4FF443
:10BF44009971ADE786F31188BFF36F8F70BD00BFA1
:10BF54009C2600206B7B0100987B01007E78010009
:10BF6400AD7B0100EDA70100C2A70100C38E010053
:10BF7400C37B0100DA7B0100F7B5044616461D4673
:10BF8400EFF305837BB152EA05030CD02D498823D6
:10BF94002D4A2E4808F01CFD2D4808F019FD882173
:10BFA400294808F00CFDEFF31187202383F312884E
:10BFB400BFF36F8F274802F06DF860B98423264AD7
:10BFC4002649224808F004FD2249254808F000FDCE
:10BFD40084212148E5E71F4802F080F8A368D3B123
:10BFE400013B1C48A36002F063F868B94FF49973ED
:10BFF400194A1C49154808F0EBFC16491A4808F080
:10C00400E7FC4FF49971E4E787F31188BFF36F8F6E
:10C01400002003B0F0BD56EA05030BD10D4802F031
:10C0240047F80028E2D087F31188BFF36F8F6FF0D1
:10C034000F00EEE722463946CDE90065054801F0D8
:10C04400F5F8E6E7BDA901009DA901007E7801008D
:10C05400C38E01009C2600206B7B0100987B0100AD
:10C06400AD7B0100C37B0100DA7B01002DE9FF41B8
:10C074000446794EEFF31187202383F31288BFF32C
:10C084006F8F764802F006F868B98423744A7549BC
:10C09400754808F09DFC7149744808F099FC8421A6
:10C0A4006F4808F08CFC6D4802F018F8D4F88450FE
:10C0B400F5B9022104F19C000AF0A4F8002840D04C
:10C0C40004F1940500220121284601F09FFE002876
:10C0D400F8D100234FF0FF3202934FF0FF3339467B
:10C0E400CDE900235D4804F18C0201F0EDFEC1E7C7
:10C0F400D4F888202B68954208BFC4F88830C4F867
:10C104008430D4F89C30554843F00203C4F89C3082
:10C11400EB68D5F8048023F0040343F00103EB60DB
:10C1240001F0C6FFF8B94FF499734D4A50494E488F
:10C1340008F04EFC49494F4808F04AFC4FF4997105
:10C14400AEE7D4F89C30DD06C3D5C4F89C00434860
:10C1540001F0AEFF0028E6D087F31188BFF36F8F9C
:10C1640004B0BDE8F08187F31188BFF36F8FB8F195
:10C17400000F0AD140493C4840F2F3233F4A08F0FB
:10C1840027FC40F2F3213D488BE72846C047EFF3F4
:10C194001187202383F31288BFF36F8F2F4801F098
:10C1A40079FF00283FF471AF2C4801F097FFEB684A
:10C1B400D90623F0010236D4EA60EB689A0716D553
:10C1C400306823F00203EB6088B10022036870B189
:10C1D40041688D4235D103686ABB7268336090420E
:10C1E40000D17360002340F8083BFFF741FED4F808
:10C1F4009C3023F00203C4F89C30DB0529D4D4F826
:10C204008450003D18BF0125144801F051FF002857
:10C2140089D087F31188BFF36F8F002D3FF42AAFC5
:10C2240001F0FAFA26E723F01103EB6005F11000A0
:10C23400FFF71EFEC1E713607368984208BF72607F
:10C24400D0E702461BB1196818460B46BFE71946EA
:10C25400FAE70025D8E700BFA0260020A826002082
:10C264006B7B0100987B01007E780100AD7B0100AF
:10C27400C37B0100DA7B01004CAA01000AAA010079
:10C2840070B5C3680546C3F340069B070C460DD53D
:10C294000122002104F1080009F0A4FF0023236017
:10C2A400054B65605A681AB9C3E90044304670BD4D
:10C2B40014605C60FAE700BFA0260020F8B5C368EC
:10C2C40004469A070E46C3F340054FD45F074FD484
:10C2D4000B680BB983680B60E368D80736D5A3688D
:10C2E4005BB92549254840F25713254A08F070FBED
:10C2F40040F25711224808F062FB02253360376888
:10C3040067B3204B9A68D7F880309A4220D109F05D
:10C31400DDFF80F00100C0B2D7F89C30D907C3F329
:10C3240080021ED502B308B300232360D7F88830F7
:10C3340083B9C7E92144384609F07EFFE36843F036
:10C344000403E3603368A3602846F8BD0125D6E7FB
:10C354000020E1E71C60C7F88840ECE76FF01505A2
:10C3640006E06FF0120503E01B07DDD56FF00F0543
:10C3740000233360E8E700BF2BAA01007E780100A8
:10C384000AAA01007826002073B50446EFF311854C
:10C39400202383F31288BFF36F8F224801F07AFEC3
:10C3A40068B98423204A2149214808F011FB1D491A
:10C3B400204808F00DFB84211B4808F000FB1948B5
:10C3C40001F08CFE00230193D4E90423B3F1004F60
:10C3D40008BF012A11D0134801F06AFEE0B94FF4F6
:10C3E4009973114A1449124808F0F2FA0D49134896
:10C3F40008F0EEFA4FF49971DEE70321201FA4F14F
:10C40400100609F0FFFE0028E5D0A369304601A913
:10C414000193FFF753FFDEE785F31188BFF36F8FB6
:10C4240002B070BDA82600206B7B0100987B010040
:10C434007E780100AD7B0100C37B0100DA7B010043
:10C4440038B50D46044648B90C499C230C4A0D489E
:10C4540008F0BEFA9C210A4808F0B1FA39B90A4931
:10C464009D23074A074808F0B3FA9D21F3E71022F9
:10C4740000210AF072FA656038BD00BFF0AA01001D
:10C484000AAA01007E7801004CAA010037B50C46C7
:10C49400019059B9284940F27D13284A284808F0E8
:10C4A40097FA40F27D11254808F089FA4B684BB998
:10C4B40024494FF4BF73214A214808F089FA4FF404
:10C4C400BF71F0E7EFF31185202383F31288BFF3E4
:10C4D4006F8F1D4801F0DEFD60B984231B4A1C499F
:10C4E400174808F075FA18491A4808F071FA8421B7
:10C4F4001648D9E7144801F0F1FD204601A9FFF7D9
:10C50400DDFE0446104801F0D3FD68B94FF4997379
:10C514000E4A11490A4808F05BFA0B490F4808F023
:10C5240057FA4FF49971E3E785F31188BFF36F8FDE
:10C53400204603B030BD00BFF0AA01000AAA0100E2
:10C544007E78010046AA0100A82600206B7B01002A
:10C55400987B0100AD7B0100C37B0100DA7B010005
:10C564000146014809F0A2BEE810002038B504468F
:10C5740058B9284940F22B23274A284808F028FABA
:10C5840040F22B21244808F01AFAC368DB0509D5C8
:10C5940023494FF40B73204A204808F019FA4FF44A
:10C5A4000B71EFE7EFF31185202383F31288BFF3B8
:10C5B4006F8F1C4801F06EFD60B984231A4A1B4931
:10C5C400164808F005FA1749194808F001FA8421B9
:10C5D4001548D8E7134801F081FD204609F033FEE1
:10C5E4000446104801F064FD68B94FF499730E4A8B
:10C5F40010490A4808F0ECF90A490F4808F0E8F92C
:10C604004FF49971E4E785F31188BFF36F8F2046E7
:10C6140038BD00BFF0AA01000AAA01007E7801001B
:10C6240063AA0100A82600206B7B0100987B01000F
:10C63400AD7B0100C37B0100DA7B010008B558B96A
:10C644000849094840F22633084A08F0C1F940F283
:10C654002631064808F0B3F9A02200210AF07DF93A
:10C6640008BD00BF31AA01007E7801000AAA0100BA
:10C67400F0B589B004460E9D58B92F4940F25333A2
:10C684002E4A2F4808F0A4F940F253312B4808F001
:10C6940096F949B92B494FF45573284A284808F0AC
:10C6A40097F94FF45571F1E7D0F89C0010F00100B0
:10C6B40009D0254940F25533204A214808F088F929
:10C6C40040F25531E2E7C4E9210004F18C00C4E9E9
:10C6D400230004F19400C4E9250055B32879002807
:10C6E40040F2011008BF0120C4F89C0000204FF064
:10C6F400FF364FF0FF37CDE90330CDE90100CDE936
:10C7040006672046114B009400F0D4FA55B129680D
:10C7140011B1204609F0E0FD6B791BB1A38943F008
:10C724000103A381204601F0DFF9C4F8804009B079
:10C73400F0BD0120D8E700BFF1C101000AAA010041
:10C744007E780100E9AA0100B5AA010071C00000C9
:10C7540038B50D46044658B90F4940F20F430F4A05
:10C764000F4808F035F940F20F410C4808F027F95A
:10C7740049B90C494FF48263084A094808F028F97A
:10C784004FF48261F1E7302200210AF0E6F84FF419
:10C7940080736560E36038BDEFAA01000AAA010056
:10C7A4007E7801004CAA0100F7B50C4616461D46DA
:10C7B400019058B9334940F28643334A334808F06C
:10C7C40007F940F28641304808F0F9F849B9304990
:10C7D40040F287432C4A2D4808F0FAF840F287418A
:10C7E400F1E7EFF31187202383F31288BFF36F8FF0
:10C7F400284801F04FFC60B98423274A274923487D
:10C8040008F0E6F82349264808F0E2F88421224893
:10C81400DAE7204801F062FCE36813F01E0F27D129
:10C8240055EA060216D1204601A9FFF747FD044642
:10C83400184801F03DFCE8B94FF49973164A1949B8
:10C84400124808F0C5F81349174808F0C1F84FF426
:10C854009971DCE743F00803E360019B04F11000E5
:10C86400A36232462B46114901F06EFC0124DFE736
:10C874000024DDE787F31188BFF36F8F204603B0F0
:10C88400F0BD00BF31AA01000AAA01007E780100B0
:10C89400EFAA0100A82600206B7B0100987B010011
:10C8A400AD7B0100C37B0100DA7B01008DC3000076
:10C8B40001460148FFF778BFE8100020F7B50C46A1
:10C8C40016461D46019058B9324940F2A943324AEE
:10C8D400324808F07DF840F2A9412F4808F06FF87B
:10C8E40049B92F4940F2AA432B4A2C4808F070F862
:10C8F40040F2AA41F1E7EFF31187202383F3128872
:10C90400BFF36F8F274801F0C5FB60B98423264A23
:10C914002649224808F05CF82249254808F058F8CE
:10C9240084212148DAE71F4801F0D8FB204609F0AA
:10C9340074FC55EA060316D1204601A9FFF7BEFC94
:10C944000446184801F0B4FBE0B94FF49973164A51
:10C954001849124808F03CF81249174808F038F80A
:10C964004FF49971DDE7E36804F1100043F0080324
:10C97400E360019B3246A36210492B4601F0E4FBBD
:10C984000124DEE787F31188BFF36F8F204603B0DD
:10C99400F0BD00BF31AA01000AAA01007E7801009F
:10C9A400EFAA0100A82600206B7B0100987B010000
:10C9B400AD7B0100C37B0100DA7B01008DC3000065
:10C9C40001460148FFF77ABFE810002038B5044655
:10C9D40058B92349234840F2CB43234A07F0F8FFD0
:10C9E40040F2CB41204807F0EAFFEFF31185202302
:10C9F40083F31288BFF36F8F1C4801F04BFB60B9BF
:10CA040084231B4A1B49174807F0E2FF17491A48B9
:10CA140007F0DEFF84211648E5E7144801F05EFBC9
:10CA2400204609F0FAFB204609F00DFC04460F48A5
:10CA340001F03EFB68B94FF499730D4A0F49094858
:10CA440007F0C6FF09490E4807F0C2FF4FF4997179
:10CA5400E1E785F31188BFF36F8F204638BD00BF2F
:10CA6400EFAA01007E7801000AAA0100A82600208E
:10CA74006B7B0100987B0100AD7B0100C37B01004F
:10CA8400DA7B01002DE9F0410E46054658B93A49D2
:10CA940040F2DC43394A3A4807F09AFF40F2DC415D
:10CAA400364807F08CFF49B9364940F2DD43334A32
:10CAB400334807F08DFF40F2DD41F1E709F006FC51
:10CAC400044648B1304940F2DE432C4A2C4807F072
:10CAD4007FFF40F2DE41E3E7EFF31188202383F385
:10CAE4001288BFF36F8F294801F0D4FA60B9842308
:10CAF400274A2849224807F06BFF2449264807F0B3
:10CB040067FF84212248CCE7204801F0E7FAEB686C
:10CB140003F01F03002B14BF012700270AD0284667
:10CB240009F07BFB284609F08EFB31462846FFF7C7
:10CB3400A7FB0446154801F0BBFA68B94FF4997392
:10CB4400134A16490E4807F043FF1049144807F0EA
:10CB54003FFF4FF49971D5E788F31188BFF36F8FC6
:10CB64003CB14FF0FF324FF0FF3306F10800FFF7FE
:10CB740003FA3846BDE8F081EFAA01000AAA0100D1
:10CB84007E780100A1AA010092AA0100A826002033
:10CB94006B7B0100987B0100AD7B0100C37B01002E
:10CBA400DA7B01000A4B9A68137C13F001030ED15F
:10CBB400526E1168B1F1F03F09D04FF0F0311160BD
:10CBC40083F31188BFF36F8F0223184602DF704787
:10CBD400782600202DE9FF470F9D04460F2D0F46B0
:10CBE400994643D12D4B994544D104F15803C4E9E6
:10CBF4001633109B4FF00008A3810423073222F060
:10CC040007063246AA212374A5733846C4E9068868
:10CC1400C4F8088084F80F8009F09FFE4FF0F033C9
:10CC240007EB060A51463B602046F6F77DF80E9B5B
:10CC3400C51D25F00705E566C4E9197602930D9B29
:10CC4400AAEB050501930C9B2A46009339464B46F3
:10CC54002046F6F71FFC124BC4F854809B6803B1BE
:10CC64001B6F2846236704B0BDE8F08705F1100365
:10CC74001E2BBAD940F24B230A4A0B490B4807F042
:10CC8400A7FE29460A486FF00F030E2207F0A0FE04
:10CC940040F24B21034807F092FE00BF25B4000088
:10CCA4007826002004AB010027AB01007E78010048
:10CCB400A7AB0100F0B587B00446DDE91276EFF3C7
:10CCC400058575B1194940F21733194A194807F017
:10CCD4007FFE194807F07CFE40F21731144807F034
:10CCE4006EFE0595109D04950F9D03950E9D02956E
:10CCF4000D9D01950C9D0095FFF76CFFB6F1FF3F6C
:10CD040008BFB7F1FF3F05D056EA070305D1204617
:10CD140000F0EAFE204607B0F0BD3A46334604F17F
:10CD24001800064901F010FAF4E700BF4FA901000A
:10CD340004AB01007E780100D8AB0100A1D1000052
:10CD44000123037483810023C0E919330367014B72
:10CD5400986070477826002070B590F91020037C05
:10CD6400002A49DBD90647D163F07F030374264BBD
:10CD7400984209D1254926485223264A07F028FE1D
:10CD84005221244807F01BFE234C224652F8183F38
:10CD9400E169934207D1C0E900210860E0610FE036
:10CDA4008B42F8D01B68002BF5D093F90E6090F9F4
:10CDB4000E50AE42F4DD5968C0E900310860586095
:10CDC400A569954200D005B9E568A3685BB9134924
:10CDD400EA23134A0E4807F0FBFD124807F0F8FD5A
:10CDE400EA210F48CEE71A7CD20606D1DA897F2AD7
:10CDF40003D9AA690AB9636170BDAB4202D028465F
:10CE040001F0C2F86561F7E7480F00201FAC01008C
:10CE14007E780100FDAB0100782600206CAC010097
:10CE240040AC0100C38E010038B590F910200146D2
:10CE3400002A037C1BDA224A03F07F039042037426
:10CE440009D120495A23204A204807F0C1FD5A211C
:10CE54001D4807F0B4FDDC0707D51D495B231A4ABA
:10CE64001A4807F0B5FD5B21F2E709F03AFA194DCB
:10CE74002A4652F8184FAB68944200D004B9EC68C3
:10CE84008B4214D05BB91449EA23144A0F4807F0C3
:10CE94009FFD134807F09CFDEA211048D9E71A7C4E
:10CEA400D20604D1DA897F2A01D9A2692AB1A34220
:10CEB40002D0204601F068F823466B6138BD00BFFC
:10CEC400480F00201FAC0100FDAB01007E7801007B
:10CED40093AC0100782600206CAC010040AC01004A
:10CEE400C38E010008B583684BB909490948A423D6
:10CEF400094A07F06DFDA421074807F060FD09F019
:10CF0400F0F9037C23F0020303740023836008BD5B
:10CF140005A801007E780100C2A7010010B50446EF
:10CF2400FFF740FE124A936884B1197C11F0090F8F
:10CF34000CD11049D923104A104807F049FD104874
:10CF440007F046FDD9210C4807F039FD6FF00A01BE
:10CF5400D9670C499C674B6843F080534B600023AE
:10CF640083F31188BFF36F8F9368D86F10BD00BF30
:10CF740078260020D6AC0100ACAC01007E7801001C
:10CF84003FAD010000ED00E070B504460D46F9B96F
:10CF9400EFF30586E6B91A4B5A699B689A4217D093
:10CFA40001F086F878B940F26D13164A164917480D
:10CFB40007F00EFD2146164807F00AFD40F26D11F8
:10CFC400104807F0FCFC3046BDE87040FFF7A6BFF0
:10CFD400204601F06DF868B94FF49973094A0A497B
:10CFE4000A4807F0F5FC2146094807F0F1FC4FF424
:10CFF4009971E5E785F31188BFF36F8F70BD00BFAA
:10D00400782600206B7B0100C37B01007E78010041
:10D01400DA7B010038B5184CA168E0690B688142DD
:10D0240014BF1A46002249680B605960A368E1697D
:10D034002AB9124AC3E900210B60E3610AE092F9BC
:10D044000E5093F90E00854212DD5168C3E90021A8
:10D054000B605360A569094B9D4200D005B9E56892
:10D06400A3689D4202D0284600F08EFF656138BD5A
:10D074008A42DED01268DBE7782600209026002062
:10D0840038B50446EFF31185202383F31288BFF3E8
:10D094006F8F174800F0FEFF68B98423154A1649BC
:10D0A400164807F095FC1249154807F091FC8421B5
:10D0B400104807F084FC0E4801F010F82046FFF7F2
:10D0C4004BFE0B4800F0F4FF68B94FF49973094A1A
:10D0D4000C490A4807F07CFC05490B4807F078FC2A
:10D0E4004FF49971E4E785F31188BFF36F8F38BD6E
:10D0F400AC2600206B7B0100987B01007E78010048
:10D10400AD7B0100C37B0100DA7B010038B5044626
:10D11400EFF31185202383F31288BFF36F8F184830
:10D1240000F0B8FF68B98423164A1749174807F076
:10D134004FFC1349164807F04BFC8421114807F0B3
:10D144003EFC0F4800F0CAFFA36813B12046FFF766
:10D15400C9FE0B4800F0ACFF68B94FF49973094A53
:10D164000C490A4807F034FC05490B4807F030FC29
:10D174004FF49971E2E785F31188BFF36F8F38BDDF
:10D18400AC2600206B7B0100987B01007E780100B7
:10D19400AD7B0100C37B0100DA7B010038B5A0F14F
:10D1A4001804EFF31185202383F31288BFF36F8FE4
:10D1B400174800F06FFF68B98423164A16491748C8
:10D1C40007F006FC1249164807F002FC84211148B6
:10D1D40007F0F5FB0E4800F081FF204609F0AFF898
:10D1E4000B4800F065FF68B94FF49973094A0D497B
:10D1F4000A4807F0EDFB06490B4807F0E9FB4FF43A
:10D204009971E4E785F31188BFF36F8F38BD00BFD0
:10D21400AC2600206B7B0100987B01007E78010026
:10D22400AD7B0100C37B0100DA7B01002DE9F047EF
:10D23400DFF8D4A0354D1746DDE90898DAF8082060
:10D24400334BA84204460E461A600BD1314932488A
:10D2540040F2B923314A07F0BBFB40F2B9212F4811
:10D2640007F0ADFBEFF31183202383F31288BFF3A0
:10D274006F8F284600F00EFF60B98423284A29499D
:10D28400254807F0A5FB2946274807F0A1FB842180
:10D294002348E5E7284600F021FFDAF8085039462C
:10D2A400284609F026F8B8F1FF3F08BFB9F1FF3F5F
:10D2B40006D04A4643461D4905F1180000F044FFD4
:10D2C400204600F0F5FE68B9194940F26D13144A7E
:10D2D400114807F07DFB2146164807F079FB40F220
:10D2E4006D11D5E7094800F0E3FE40B9104940F25A
:10D2F4006D130B4A084807F06BFB0449ECE7304612
:10D30400BDE8F047FFF70ABE78260020AC260020CF
:10D31400B026002067AD01007E780100FDAB01005E
:10D324006B7B0100987B0100AD7B0100A1D1000063
:10D33400C37B0100DA7B010070B50546EFF311866B
:10D34400202383F31288BFF36F8F1B4800F0A2FEE3
:10D3540068B98423194A1A491A4807F039FB16494F
:10D36400194807F035FB8421144807F028FB1248BC
:10D3740000F0B4FE2C68A54215D014B12046FFF786
:10D38400B1FD0D4800F094FE78B94FF499730B4A3F
:10D394000E490C4807F01CFB07490D4807F018FB21
:10D3A4004FF49971E0E70024EBE786F31188BFF3AB
:10D3B4006F8F204670BD00BFAC2600206B7B010040
:10D3C400987B01007E780100AD7B0100C37B0100E6
:10D3D400DA7B01002DE9F04104460D46EFF3118795
:10D3E400202383F31288BFF36F8F594800F052FE55
:10D3F40060B98423574A5849584807F0E9FA544910
:10D40400574807F0E5FA8421524818E0504800F0E4
:10D4140065FE237C03F01F02002A0CBF01260026B0
:10D4240062D103F07F0323744E4B9C4209D14E49D1
:10D434005A234E4A494807F0CBFA5A214B4807F081
:10D44400BEFA204608F04DFF237C6DB243F0800302
:10D45400DA07A573237407D545495323434A3F4844
:10D4640007F0B6FA5321E9E7DFF80881424652F89B
:10D47400183FD8F81C10934208D1C4E900210C606D
:10D48400C8F81C400DE08B42F7D01B68002BF4D089
:10D4940093F90E00A842F6DD5968C4E900310C6026
:10D4A4005C60D8F81840944200D00CB9D8F80C400D
:10D4B400D8F808309C4202D0204600F065FDC8F838
:10D4C4001440234800F0F4FD00283AD14FF4997336
:10D4D400204A2949214807F07BFA1D49274807F0CB
:10D4E40077FA4FF499718FE79B0728D5A16841B962
:10D4F40023491A48A423234A07F06AFAA42121489D
:10D504009DE720466DB208F0ECFEA5730B689942C6
:10D5140009D14B68C4E900131C604C60D1E74A6828
:10D524009342F6D01B68002BF3D093F90E20AA4245
:10D53400F5DD5A68C4E9003214605C60C1E7A57384
:10D54400BFE787F31188BFF36F8F3046BDE8F081E2
:10D55400AC2600206B7B0100987B01007E780100E3
:10D56400AD7B0100480F00201FAC0100FDAB0100A2
:10D5740093AC010078260020C37B0100DA7B010014
:10D5840005A80100C2A70100034648B9EFF30582CC
:10D5940032B9064A51699268914201D0FFF7BEBC84
:10D5A40083F31188BFF36F8F704700BF7826002084
:10D5B40010B5EFF31184202383F31288BFF36F8F28
:10D5C400284800F067FD60B98423274A2749284882
:10D5D40007F0FEF92349274807F0FAF98421224885
:10D5E40012E0204800F07AFDEFF3058373B122497D
:10D5F40040F23B33214A1E4807F0EAF9204807F07D
:10D60400E7F940F23B311D4807F0D9F91D4B9A6800
:10D61400D37B012B0CD11C494FF44F73174A144888
:10D6240007F0D6F9164807F0D3F94FF44F71EAE73B
:10D63400013BD3730B4800F03BFD68B94FF4997379
:10D64400094A12490A4807F0C3F90649104807F085
:10D65400BFF94FF49971C2E784F31188BFF36F8F58
:10D6640010BD00BFAC2600206B7B0100987B01003D
:10D674007E780100AD7B01004FA90100FDAB0100E4
:10D68400C38E010078260020A0AD0100C37B0100F9
:10D69400DA7B010070B5EFF31186202383F312883F
:10D6A400BFF36F8F2A4800F0F5FC68B98423294A38
:10D6B40029492A4807F08CF92549294807F088F9AF
:10D6C4008421244807F07BF9264D214800F006FD0B
:10D6D400AB68DA7B6AB9244940F24D33234A1F48C8
:10D6E40007F076F9224807F073F940F24D311F48EC
:10D6F400E8E7EFF3058161B11E4940F24E331B4A5E
:10D70400164807F065F91A4807F062F940F24E31FD
:10D71400EDE70132DA732A4652F8184F944200D0EA
:10D7240004B9EC681A7CD20604D1DA897F2A01D9BB
:10D73400A2692AB19C4202D0204600F025FC23466F
:10D744006B613146BDE870400148FFF71DBC00BF66
:10D75400AC2600206B7B0100987B01007E780100E1
:10D76400AD7B010078260020D1AD0100FDAB0100A6
:10D77400C38E01004FA9010038B50446EFF31185AB
:10D78400202383F31288BFF36F8F184800F082FCC4
:10D7940068B98423164A1749174807F019F9134939
:10D7A400164807F015F98421114807F008F90F48C5
:10D7B40000F094FC204608F0E2FD04460B4800F01B
:10D7C40077FC68B94FF49973094A0D490A4807F080
:10D7D400FFF806490B4807F0FBF84FF49971E3E7AB
:10D7E40085F31188BFF36F8F204638BDAC26002027
:10D7F4006B7B0100987B01007E780100AD7B01000A
:10D80400C37B0100DA7B0100024B03F11802C3E978
:10D81400062270477826002070B5EFF3058373B1B4
:10D8240038494FF49063384A384807F0D1F83848FB
:10D8340007F0CEF84FF49061334807F0C0F8EFF3E7
:10D844001186202383F31288BFF36F8F314800F0D1
:10D8540021FC60B98423304A30492C4807F0B8F8D9
:10D864002C492F4807F0B4F884212B48E5E72D4CC8
:10D87400284800F033FCA168E0690B68814214BFBA
:10D884001A46002249680B605960A368E1692AB905
:10D89400254AC3E900210B60E3610AE092F90E50C6
:10D8A40093F90E00854223DD5168C3E900210B6022
:10D8B4005360A5691C4B9D4200D005B9E568A36877
:10D8C4009D4202D0284600F05FFB1248656100F0DB
:10D8D400EFFB88B940F26D130F4A14490B4807F067
:10D8E40077F80C49124807F073F840F26D11BCE761
:10D8F4008A42CDD01268CAE73046BDE87040FFF7CF
:10D904000DBB00BF4FA90100FDAB01007E780100F3
:10D91400C38E0100AC2600206B7B0100987B0100C4
:10D92400AD7B01007826002090260020C37B0100F7
:10D93400DA7B01002DE9F04106460C46EFF305873A
:10D9440077B134494FF49363334A344807F040F8CD
:10D95400334807F03DF84FF493612F4807F02FF850
:10D9640050EA010304D1FFF757FF0020BDE8F0811E
:10D97400EFF31188202383F31288BFF36F8F2948B4
:10D9840000F088FB60B98423274A2849234807F01C
:10D994001FF82449264807F01BF884212248DDE7B4
:10D9A400244D204800F09AFBA868234B1860FFF729
:10D9B4003BFAA868234632462049183000F0C4FBDD
:10D9C400AA680446137C174843F00403137400F058
:10D9D4006FFB68B940F26D13134A19490F4806F0FA
:10D9E400F7FF1049174806F0F3FF40F26D11D5E731
:10D9F4004046FFF793FAAB68D3E90A23B3F1004F2B
:10DA040008BFBA42B1D108F0E8FC201A20EAE0705D
:10DA1400ACE700BF4FA90100FDAB01007E78010017
:10DA2400C38E0100AC2600206B7B0100987B0100B3
:10DA3400AD7B010078260020B0260020A1D1000093
:10DA4400C37B0100DA7B010070B506460D46EFF397
:10DA5400058474B1114940F2C643114A114806F0D5
:10DA6400B7FF114806F0B4FF40F2C6410C4806F077
:10DA7400A6FFFFF75FFFB5F1FF3F08BFB6F1FF3F19
:10DA84001FBF47F6FF734FF47A72E0FB0234D80BE2
:10DA94000CBF4FF0FF3040EA444070BD4FA9010075
:10DAA400FDAB01007E780100C38E01000C4908B56E
:10DAB4008C464FF4004E0021C0FB0EC1002360468B
:10DAC400084AF2F745FBC117FFF734FF47F6FF7327
:10DAD40000220449E0FB0132DB0B43EA424008BD6B
:10DAE4003F420F0040420F0038B50446EFF3118562
:10DAF400202383F31288BFF36F8F204800F0CAFA03
:10DB040068B984231E4A1F491F4806F061FF1B4958
:10DB14001E4806F05DFF8421194806F050FF17489F
:10DB240000F0DCFA237C5B0710D504F1180000F048
:10DB3400E7FB237C204623F004032374FFF70CF94E
:10DB44002946BDE838400D48FFF71EBA0B4800F0DF
:10DB5400AFFA68B94FF49973094A0D490A4806F0B7
:10DB640037FF06490B4806F033FF4FF49971D3E7AA
:10DB740085F31188BFF36F8F38BD00BFAC2600203A
:10DB84006B7B0100987B01007E780100AD7B010076
:10DB9400C37B0100DA7B0100014B9868704700BF2A
:10DBA400782600202DE9F84304468789EFF3118590
:10DBB400202383F31288BFF36F8F824800F06AFA40
:10DBC40068B98423804A8149814806F001FF7D4970
:10DBD400804806F0FDFE84217B4806F0F0FE79487B
:10DBE40000F07CFA237C180717D5764800F060FA19
:10DBF40068B94FF49973744A7749754806F0E8FE9A
:10DC04007049764806F0E4FE4FF49971E4E785F331
:10DC14001188BFF36F8FBDE8F883D90943F0080278
:10DC240040F083802274A36813B12046FFF75AF9A9
:10DC340004F1180000F064FBA66D04F15808B04527
:10DC440011D04FF0000976B13046FFF74BF906F1D9
:10DC5400180000F055FB3046C6F87C90FFF77CF8BE
:10DC6400A66DB045EFD1DFF87881D8F808309C4232
:10DC74007AD1EFF30589B9F1000918BF4FF0010912
:10DC8400D8F81860574A964200D00EB9D8F80C60FC
:10DC9400B34202D0304600F077F92046C8F8146049
:10DCA40007F076F9B9F1000F02D04F48FFF748F8B2
:10DCB400D8F808309C426AD1EFF30586002E66D16D
:10DCC400A389DA071FD53F4800F0F2F9002890D065
:10DCD40085F31188BFF36F8F86F31188BFF36F8FBD
:10DCE4000423184602DFEFF31185202383F31288FF
:10DCF400BFF36F8F334800F0CDF900283FF461AFD4
:10DD0400304800F0EBF92F4800F0D2F978BB40F22C
:10DD14006D132D4A30492E4806F05AFE29492F48E2
:10DD240006F056FE40F26D1156E7304A03F07F03C9
:10DD340043F008039442237408D12D495A232D4AF1
:10DD4400234806F045FE5A212A4846E7D90707D555
:10DD540029495B23274A1E4806F03AFE5B21F3E774
:10DD6400204608F0BEFA5EE74FF0000988E728462F
:10DD7400FFF7D4F821494FF4EE731E4A144806F015
:10DD840027FE1F4806F024FE4FF4EE71DCE70D4831
:10DD940000F08EF900283FF42CAF85F31188BFF30F
:10DDA4006F8FFB077FF537AF40F2A253114A154935
:10DDB400074806F00DFE2146134806F009FE40F21E
:10DDC400A251C1E7AC2600206B7B0100987B0100C7
:10DDD4007E780100AD7B0100C37B0100DA7B01008A
:10DDE400782600209026002048100020480F0020AC
:10DDF4001FAC0100FDAB010093AC010002AE0100B9
:10DE04000DAE01002FAE01003AAE01002DE9F8433A
:10DE1400064688461746EFF31189202383F31288B8
:10DE2400BFF36F8F214800F035F9054668B98423A4
:10DE34001F4A2049204806F0CBFD1C491F4806F024
:10DE4400C7FD84211A4806F0BAFD184800F046F9C7
:10DE54003468A6421FD004B32046C4F87C806761AE
:10DE6400FFF740F804F1180000F04AFA2046FEF7E4
:10DE740073FF0E4800F01CF988B94FF499730C4AEB
:10DE84000F490D4806F0A4FD08490E4806F0A0FD10
:10DE94004FF49971D6E70025EBE72546E9E789F3C6
:10DEA4001188BFF36F8F2846BDE8F883AC260020A5
:10DEB4006B7B0100987B01007E780100AD7B010043
:10DEC400C37B0100DA7B0100D3B5DDE90667089C5A
:10DED400CDE90067FFF7AAF91CB1034B9B685B69A6
:10DEE400236002B0D0BD00BF78260020027C034628
:10DEF40012F01F0210D10A4988420DD0094908685E
:10DF040068B1D9897F2909D893F90E20064B1B687B
:10DF14009A42B8BF002070470020704710467047EF
:10DF2400480F00201C020020B426002008B568B168
:10DF34000F4B98420AD303F11802904206D21822DA
:10DF4400C01AB0FBF2F302FB13034BB109490A48B0
:10DF54003F230A4A06F03CFD3F21084806F02FFD06
:10DF64000122074BC0105843064B1A5408BD00BF8A
:10DF7400C810002080AE01007E78010058AE010078
:10DF8400ABAAAAAA9C2C002070B50C4B0C4D1E7C8D
:10DF9400FFF7ACFF182303FB06550446284600F0A0
:10DFA400AFF90022074B9A553CB1621E2846BDE8E2
:10DFB40070400549D31700F0C7B870BD782600201B
:10DFC400C81000209C2C002031DF000038B5EFF38E
:10DFD4001185202383F31288BFF36F8F234800F049
:10DFE40059F868B98423224A2249234806F0F0FCF0
:10DFF4001E49224806F0ECFC84211D4806F0DFFC93
:10E004001A4800F06BF81E4B1E4A9C681068A04228
:10E0140013D1FFF7B9FF154800F04AF800BB4FF4DD
:10E024009973134A1849144806F0D2FC0F4917484B
:10E0340006F0CEFC4FF49971DFE700211B7C1160E0
:10E04400134AD35C002BE6D02046FFF74FFF00288D
:10E05400E1D0237CDB0601D1FEF7DCFF2046D8E7C4
:10E0640085F31188BFF36F8F38BD00BFAC26002045
:10E074006B7B0100987B01007E780100AD7B010081
:10E0840078260020B0260020C37B0100DA7B010043
:10E094009C2C0020006838B1044B00F003001B7C6A
:10E0A400C01A18BF0120704701207047782600204D
:10E0B400002302680360EFF30581074B986811B1F0
:10E0C400017CC90705D41B7C1843831A5842584164
:10E0D40070470120704700BF78260020024B1A7C4D
:10E0E4009B6813430360704778260020024B18682E
:10E0F400984208BF0020704720020020034B1B6891
:10E104000BB9F8F7AFB90020704700BFB82600205C
:10E1140030B570B10B4B5B6898420AD0036843B1C9
:10E12400D3E90421D0E90445121941EB0501C3E9FF
:10E134000421D0E9003213605A600023C0E900339F
:10E1440030BD00BF20020020B3F1FF3F08BFB2F191
:10E15400FF3F2DE9F84F04469B4615461F4600F045
:10E16400B280D0F80090B9F1000F0CD05749642365
:10E17400574A584806F02CFC574806F029FC6421FD
:10E18400534806F01CFC8160EFF31188202383F3CD
:10E194001288BFF36F8F5148FFF77CFF824660B946
:10E1A40084234F4A4F494B4806F012FC4B494E48D2
:10E1B40006F00EFC84214A48E3E74848FFF78EFF47
:10E1C400BBF1000F494A1FDBFFF798FF06460135F4
:10E1D4004BF1000B454A2D184BEBE073D2E90017C5
:10E1E400C4E904536D1843EB0707FFF77FFF0346A9
:10E1F400DFF8FCE0DEF80490EBB9C4E900E9C9F803
:10E204000040CEF8044028E06FF00103D2E9001288
:10E214005B1A4FF0FF3161EB02025B1B62EB0B02F6
:10E22400012B72F10001BCBF01234A464FF0000AE2
:10E23400C4E90432D9E7D3E9041CD4E904208A42AE
:10E2440070EB0C0B2EDA891A5A686CEB0000C3E9E8
:10E254000410C4E9003214605C60FFF747FF844295
:10E264000ED1244B1B685BB9BAF1000F02D1FFF742
:10E2740045FF0646304608F099F80021F8F7CCF837
:10E284001648FFF715FFB0B94FF49973144A1A49A9
:10E29400104806F09DFB1149184806F099FB4FF40D
:10E2A400997188E7521A60EB0C004B45C4E90420CD
:10E2B400A3D01B68A0E788F31188BFF36F8F2846AB
:10E2C4003946BDE8F88F00252F46F8E74FB0010026
:10E2D4002BB001007E780100C38E0100BC26002013
:10E2E4006B7B0100987B0100AD7B0100E0100020F6
:10E2F40020020020B8260020C37B0100DA7B010045
:10E3040070B50446EFF31186202383F31288BFF31C
:10E314006F8F2A48FFF7BEFE68B98423284A29492B
:10E32400294806F055FB2549284806F051FB84216D
:10E33400234806F044FB2148FFF7D0FE23683BB393
:10E34400FFF7D4FE05462046FFF7E2FE00224FF019
:10E354000043A542C4E9042312D000241748FFF760
:10E36400A7FE20BB4FF49973154A1949164806F0C5
:10E374002FFB1249174806F02BFB4FF49971D7E78E
:10E38400FFF7BCFE08F012F80021F8F745F8E4E7BF
:10E39400D4E90423B3F1004F08BF012A04D10022B9
:10E3A4004FF00043C4E904236FF01504D6E786F365
:10E3B4001188BFF36F8F204670BD00BFBC260020BC
:10E3C4006B7B0100987B01007E780100AD7B01002E
:10E3D400C37B0100DA7B01002DE9F047DFF80491EB
:10E3E4000246C9F80000FFF781FE8846044600266D
:10E3F4000027DFF8F4A04FEAE27CDAE9001354B115
:10E40400D4E90450AA427CEB000E1EDAAD1A60EB8C
:10E414000C00C4E904500024521843EB0C032046BA
:10E42400CAE90023C9F8004007F0C0FF2146F7F706
:10E43400F3FF2E48FFF73CFED0B188F31188BFF3F9
:10E444006F8FBDE8F047FFF7C1BD691843EBE57373
:10E454002046C4E90467CAE90013FFF759FE012204
:10E464004FF000432148C4E90423FFF721FE78B9A3
:10E474004FF499731E4A1F491F4806F0A9FA1B4915
:10E484001E4806F0A5FA4FF49971194806F097FA58
:10E4940088F31188BFF36F8F2046A3689847EFF382
:10E4A4001188202383F31288BFF36F8F0F48FFF77F
:10E4B400F1FD58B984230E4A11490F4806F088FA31
:10E4C4000A49104806F084FA8421DEE70748FFF77A
:10E4D40005FED9F80020521BC9F80020FFF706FEFC
:10E4E400044688E7B8260020E0100020BC2600205F
:10E4F4006B7B0100C37B01007E780100DA7B0100A5
:10E50400987B0100AD7B010010B5EFF3118420234B
:10E5140083F31288BFF36F8F0B48FFF7BBFD68B915
:10E5240084230A4A0A490B4806F052FA06490A4863
:10E5340006F04EFA8421054806F041FA0248FFF736
:10E54400CDFD204610BD00BFBC2600206B7B010022
:10E55400987B01007E780100AD7B010070B5EFF37C
:10E564001186202383F31288BFF36F8F1A48FFF7B5
:10E5740091FD68B98423194A19491A4806F028FA02
:10E584001549194806F024FA8421144806F017FAAC
:10E594001148FFF7A3FDFFF7B1FD144AD2E9004586
:10E5A400041945EBE0750C48FFF782FD68B94FF498
:10E5B40099730A4A0E490B4806F00AFA06490D48AF
:10E5C40006F006FA4FF49971DFE786F31188BFF37A
:10E5D4006F8F2046294670BDBC2600206B7B01004E
:10E5E400987B01007E780100AD7B0100E0100020E3
:10E5F400C37B0100DA7B0100F8B50446EFF3118711
:10E60400202383F31288BFF36F8F5A48FFF742FD2C
:10E6140068B98423584A5949594806F0D9F95549E3
:10E62400584806F0D5F98421534806F0C8F95148F2
:10E63400FFF754FDD4E90423B3F1004F08BF012AC6
:10E6440013D04C48FFF734FD002840F08E804FF47F
:10E654009973494A4C494A4806F0BAF945494B4826
:10E6640006F0B6F94FF49971DEE7D4E90A566A1C4C
:10E6740046F10003022A73F1000334D3013D46F14D
:10E68400FF36002EBCBF00252E4607F0AAFE01303F
:10E6940041F10001401946EB0101012871F100012B
:10E6A4005ADB07F09EFE6FF00203013041F10001D6
:10E6B400401946EB010183426FF000438B4150DB6C
:10E6C40007F08FFE013041F100016FF001024019A3
:10E6D40046EB01034FF0FF31121A61EB03032046AE
:10E6E4002B49FFF731FD236B256A01332363D5B131
:10E6F4002048FFF7DDFC0028A9D087F31188BFF379
:10E704006F8F2046A847EFF31187202383F31288E5
:10E71400BFF36F8F1748FFF7BDFC00283FF479AFB4
:10E724001448FFF7DBFC54F8185FA54289D0002D8C
:10E7340087D02846FEF7EAFC00230E48EB67FFF774
:10E74400B7FC002883D087F31188BFF36F8F284666
:10E75400BDE8F840FEF794BC6FF001024FF0FF33C0
:10E76400BDE700224FF00043B9E787F31188BFF3F8
:10E774006F8FF8BDC02600206B7B0100987B0100E1
:10E784007E780100AD7B0100C37B0100DA7B0100D0
:10E79400FDE500002DE9F843064614461D46914662
:10E7A4009846EFF31187202383F31288BFF36F8F0A
:10E7B4002748FFF76FFC68B98423264A264927486F
:10E7C40006F006F92249264806F002F98421214878
:10E7D40006F0F5F81E48FFF781FCB5F1FF3F08BFCE
:10E7E400B4F1FF3F11D11A48FFF762FC50BB4FF45C
:10E7F4009973184A1B49194806F0EAF814491A484B
:10E8040006F0E6F84FF49971E1E7002D0ADB012CDC
:10E8140075F100032246BCBF0122002512F1FF3925
:10E8240045F1FF383046FFF76BFDDDE90823C6E903
:10E834000A2300234A463363304643460B49FFF715
:10E8440083FCD0E787F31188BFF36F8FBDE8F883AB
:10E85400C02600206B7B0100987B01007E780100BC
:10E86400AD7B0100C37B0100DA7B0100FDE5000004
:10E8740070B50546EFF31184202686F31288BFF3A2
:10E884006F8F2D48FFF706FC68B984232B4A2C4967
:10E894002C4806F09DF828492B4806F099F8842165
:10E8A400264806F08CF82448FFF718FC2846FFF7A2
:10E8B40027FD90B12048FFF7FBFB002837D14FF428
:10E8C40099731E4A21491F4806F082F81A492048C4
:10E8D40006F07EF84FF49971E2E76B6ACBB1164803
:10E8E400FFF7E6FB0028EAD084F31188BFF36F8FAB
:10E8F40028466B6A9847EFF3118486F31288BFF3B6
:10E904006F8F0D48FFF7C6FB0028BED00A48FFF7FB
:10E91400E5FB05F11800FEF70FFD0028CAD0FEF74D
:10E92400AFFB2146BDE87040034807F026BD84F3E1
:10E934001188BFF36F8F70BDC02600206B7B010070
:10E94400987B01007E780100AD7B0100C37B010050
:10E95400DA7B0100F8B505460E46EFF31187202354
:10E9640083F31288BFF36F8F1F48FFF793FB68B9D7
:10E9740084231E4A1E491F4806F02AF81A491E48D5
:10E9840006F026F88421194806F019F81648FFF70E
:10E99400A5FB2C68A5421CD0D4E9003213605A6050
:10E9A400002331462046C4E9003307F06EFD0E48CB
:10E9B400FFF77EFB78B94FF499730C4A0F490D4861
:10E9C40006F006F808490E4806F002F84FF499716B
:10E9D400D9E70024EBE787F31188BFF36F8F201E7C
:10E9E40018BF0120F8BD00BFC42600206B7B0100C6
:10E9F400987B01007E780100AD7B0100C37B0100A0
:10EA0400DA7B010070B504460D46EFF3118620232E
:10EA140083F31288BFF36F8F2048FFF73BFB68B97D
:10EA240084231F4A1F49204805F0D2FF1B491F4871
:10EA340005F0CEFF84211A4805F0C1FF1748FFF7FF
:10EA44004DFB01212068E5608442A16011D1134887
:10EA5400FFF72EFBE0B94FF49973114A1449124899
:10EA640005F0B6FF0D49134805F0B2FF4FF4997154
:10EA7400E1E7D0E9003213605A600023C0E90033B3
:10EA840007F003FD3146054807F077FC002070BD10
:10EA940086F31188BFF36F8FF8E700BFC426002008
:10EAA4006B7B0100987B01007E780100AD7B010047
:10EAB400C37B0100DA7B01002DE9F84F05460C46C3
:10EAC400924607F003FC002863D1344B9B681E6F09
:10EAD400002E5ED06F1E3D420BD031491823314ABF
:10EAE400314805F075FF314805F072FF18212D48B3
:10EAF4001CE004344DD245F0040B06F11408EFF386
:10EB04001189202383F31288BFF36F8F4046FFF7E8
:10EB1400C1FA68B98423264A2649234805F058FFD8
:10EB24004146254805F054FF8421214805F047FF5C
:10EB34004046FFF7D3FA224659463046D0470446AA
:10EB44004046FFF7B5FA68B94FF49973184A1B4960
:10EB5400154805F03DFF4146194805F039FF4FF4CB
:10EB64009971E2E789F31188BFF36F8F8CB144F890
:10EB7400046B7DB13C420DD035230A4A11490A4841
:10EB840005F026FF21462A460F4805F021FF3521CE
:10EB9400ADE700242046BDE8F88F00BF78260020AA
:10EBA40063780100B2B101007E7801009B78010016
:10EBB4006B7B0100987B0100AD7B0100C37B0100EE
:10EBC400DA7B0100D6B1010008B201000146024A15
:10EBD4000020FFF771BF00BF0349010007B5074BD1
:10EBE4004FF48052009306494FF0FF330548FDF778
:10EBF4003FFD002003B05DF804FB00BF5474010026
:10EC040090F70020E8100020014B1860704700BF07
:10EC1400C8260020014B1B681B681847C826002023
:10EC2400014B1B685B681847C8260020014B1B6812
:10EC3400DB681847C8260020014B1B689B681847EF
:10EC4400C8260020014B1B681B691847C8260020F2
:10EC5400014B1B685B691847C8260020014B1B68E1
:10EC64009B691847C8260020014B1B68DB691847BD
:10EC7400C8260020014B1B689B6D1847C82600203E
:10EC8400014B1B68DB6D1847C8260020014B1B682D
:10EC94001B6E1847C8260020014B1B685B6E184783
:10ECA400C8260020014B1B689B6E1847C82600200D
:10ECB400014B1B68DB6E1847C8260020014B1B68FC
:10ECC4001B6F1847C82600200FB407B5064B04A9CC
:10ECD4001B6851F8040B9B6F0191984703B05DF8D2
:10ECE40004EB04B0704700BFC82600200FB407B57A
:10ECF400064B04A91B6851F8040BDB6F019198477C
:10ED040003B05DF804EB04B0704700BFC8260020D0
:10ED1400024B1B68D3F88430184700BFC826002074
:10ED2400024B1B68D3F88C30184700BFC82600205C
:10ED3400024B1B68D3F89030184700BFC826002048
:10ED4400024B1B68D3F89430184700BFC826002034
:10ED5400024B1B68D3F89C30184700BFC82600201C
:10ED6400024B1B68D3F8A430184700BFC826002004
:10ED7400024B1B68D3F8A830184700BFC8260020F0
:10ED8400024B1B68D3F8AC30184700BFC8260020DC
:10ED9400024B1B68D3F8B430184700BFC8260020C4
:10EDA400024B1B68D3F8BC30184700BFC8260020AC
:10EDB400024B1B68D3F8C430184700BFC826002094
:10EDC400024B1B68D3F8C830184700BFC826002080
:10EDD400024B1B68D3F8D830184700BFC826002060
:10EDE400024B1B68D3F8DC30184700BFC82600204C
:10EDF400024B1B68D3F8E430184700BFC826002034
:10EE0400024B1B68D3F8F430184700BFC826002013
:10EE1400024B1B68D3F8F830184700BFC8260020FF
:10EE2400024B1B68D3F8FC30184700BFC8260020EB
:10EE3400024B1B68D3F80031184700BFC8260020D6
:10EE4400024B1B68D3F80431184700BFC8260020C2
:10EE5400024B1B68D3F80831184700BFC8260020AE
:10EE6400024B1B68D3F80C31184700BFC82600209A
:10EE7400024B1B68D3F81031184700BFC826002086
:10EE8400024B1B68D3F81431184700BFC826002072
:10EE9400024B1B68D3F81831184700BFC82600205E
:10EEA400024B1B68D3F81C31184700BFC82600204A
:10EEB400024B1B68D3F84C31184700BFC82600200A
:10EEC400024B1B68D3F85031184700BFC8260020F6
:10EED400024B1B68D3F85431184700BFC8260020E2
:10EEE400024B1B68D3F85831184700BFC8260020CE
:10EEF400024B1B68D3F85C31184700BFC8260020BA
:10EF0400024B1B68D3F86031184700BFC8260020A5
:10EF1400024B1B68D3F86431184700BFC826002091
:10EF2400024B1B68D3F86831184700BFC82600207D
:10EF3400024B1B68D3F86C31184700BFC826002069
:10EF4400014B1B689B6B1847C8260020014B1B68AC
:10EF5400DB6B1847C826002010B4034C2468246CCB
:10EF6400A44610BC604700BFC826002010B4034C60
:10EF74002468646CA44610BC604700BFC826002007
:10EF8400024B1B68D3F89431184700BFC8260020F1
:10EF9400024B1B68D3F89831184700BFC8260020DD
:10EFA400024B1B68D3F89C31184700BFC8260020C9
:10EFB400024B1B68D3F8A031184700BFC8260020B5
:10EFC400024B1B68D3F8A431184700BFC8260020A1
:10EFD400024B1B68D3F8A831184700BFC82600208D
:10EFE400024B1B68D3F8AC31184700BFC826002079
:10EFF400024B1B68D3F8B031184700BFC826002065
:10F00400024B1B68D3F8B831184700BFC82600204C
:10F01400F8B5054610460C461746FFF7F1FFB4EB6A
:10F02400500F024607D223461B491C48FFF75EFED9
:10F034004FF0FF30F8BD10F001012AD016491848EE
:10F04400FFF754FEF4E73B5CA3F14106192E09D8FF
:10F054002033DBB2A3F16106052E17D91A460E49F7
:10F064001048EDE7A3F13006F6B2092EF2D8264493
:10F07400C307F4B247BF6C5400242401E4B248BF70
:10F08400013101309042DED10846D3E7573BDEB26E
:10F09400EDE708460C46F5E73B63020039B2010090
:10F0A4006DB201009BB2010030B5054693B00C4629
:10F0B40048226846184907F02AFC2DB1012D15D0C5
:10F0C4002A46164916480EE0631E0C2B06D8052264
:10F0D40040F6671314FB023013B030BD0E2C18D069
:10F0E40022460E490F48FFF701FE0FE06A4624232B
:10F0F40032F8021BA14205D104EB840404F59C50B0
:10F104000830E9E7013B13F0FF03F1D14FF0FF3082
:10F11400E2E740F6B410DFE7F06E01001F6302007F
:10F12400DFB20100C2B2010070B5284A0C4609687A
:10F13400914205D02648FFF7D9FD4FF0FF3070BD4E
:10F144006268042A02D004212248F4E7A3681E0E50
:10F15400012EC3F30741C3F30725DBB208D0012214
:10F1640031461D48FFF7C2FD1C48FFF7BFFDE4E729
:10F17400022902D002221A48F4E70E2D03D00E22EF
:10F1840029461848EEE7092B03D0092219461648E8
:10F19400E8E7C168E368012906D002290FD051B11C
:10F1A4001248FFF7A3FD04E099070CD41048FFF7B9
:10F1B4009DFD1048D9E75A0705D40F48F7E7DB0649
:10F1C40001D40E48F3E70020B9E700BFAF1EADDE5F
:10F1D400F9B2010027B3010055B3010013B40100D3
:10F1E40080B30100B1B30100E2B301008BB40100AC
:10F1F40026B401009FB4010046B4010065B40100C7
:10F204002DE9F04717461C46894609B102B11BB9DE
:10F214002748FFF76BFD06E0332A09D83422394624
:10F224002448FFF763FD4FF0FF384046BDE8F08700
:10F23400FFF77AFF8046002837D01F48E9E7032DFF
:10F244002ED8DFE805F02328021E2260DAF8043005
:10F254006360DAF8043001351E44D9F80430AB4257
:10F26400E3D909EB060ADAF804300836F118B94292
:10F2740009EB0602E3D92A4639461048FFF736FD62
:10F28400D1E7A260DAF80430E360E2E72261DAF859
:10F2940004306361DDE7A261DAF80430E361D8E7A2
:10F2A40029460748FFF722FDD3E705463426D4E76D
:10F2B4006E940100BAB40100E0B40100F2B401009C
:10F2C4001CB5010038B50D4C05462178806802F064
:10F2D40063F980B9217BA86802F05EF950B101237B
:10F2E4000C2202FB0344064962680648FFF7FEFC51
:10F2F4004FF0FF3038BD0023F2E700BF28020020A2
:10F30400BA63020031B50100F8B5144C0646002575
:10F314002746227A2178B06800F0E4FB50B10C2330
:10F3240003FB05730E495A680E48FFF7DFFC4FF0E4
:10F33400FF30F8BD2178B06802F080F930B10C23B9
:10F3440003FB057306495A680748EEE76B1C022B5A
:10F354004FF0010504F10C04EBD0DAE72802002099
:10F36400A46302004FB5010070B5010073B50646F1
:10F374000D46FFF7A7FF30B120492148FFF7B6FC3F
:10F384004FF0FF3413E02A69A2B16B6993B1A96904
:10F3940081B1E86970B1CDE900100121B06800F0D5
:10F3A400DBFA044648B115491648FFF79FFC20468E
:10F3B40002B070BD0022144B1A752A6882B16B68C2
:10F3C40073B1A96861B1E86850B1CDE900100021BA
:10F3D400B06800F0C1FA044628B108490B48E4E7D4
:10F3E4000022094B1A723046FFF78EFF044610B113
:10F3F40002490748C2E701237375D8E78E63020008
:10F4040097B50100ABB5010028020020C6B5010084
:10F41400E1B5010010B50423054A806800F062F8E4
:10F42400044618B103490448FFF760FC204610BDA8
:10F43400040000B078630200F4B5010070B50E4614
:10F4440014460546B4B010B10AB1012908D92049BF
:10F454002048FFF74BFC4FF0FF35284634B070BD11
:10F46400BC22FF2105A8FFF7F9FBA86833AA05A968
:10F4740002F072F9054620B115491748FFF736FC2A
:10F48400EBE74EB9022326A9339A134207D0104959
:10F494001248FFF719FCE0E7042328A9F4E7062241
:10F4A4002046FFF7D5FB204607F03AF80028D4D1D0
:10F4B400637907490393237909480293E378019315
:10F4C400A378009363782278FFF7FEFBC5E700BFBB
:10F4D400596302006A94010010B601003BB60100B2
:10F4E4005EB60100F7B50E4614461F46054620B128
:10F4F40041B925492548FFF7F9FB4FF0FF34204671
:10F5040003B0F0BD02F19243B3F5813F10D302F191
:10F51400A043B3F5443F0BD3114690F85C0000F0D0
:10F52400C5F928B9224618491948FFF7DFFBE4E773
:10F5340000232046694695F85C20CDE9003300F0AD
:10F54400CFF9044620B113491348FFF7CFFBD6E7A0
:10F55400D5F8B80001A9FFF7ABFB284601F014FE6B
:10F56400044648B10B490D48FFF7C0FBD5F8B80075
:10F5740001A9FFF7A3FBC2E73B463146009AA868FE
:10F5840007F00FF9F2E700BF2B64020096B6010002
:10F59400A9B601001A640200C9B60100ECB6010064
:10F5A4002DE9F7430D4617469846064620B14AB959
:10F5B40060496148FFF79AFB4FF0FF34204603B0DF
:10F5C400BDE8F08301F19244B4F5813F4ED301F1DB
:10F5D400A043B3F5443F49D301F07F43B3F1404F17
:10F5E40090F85C0010D000F061F900283ED105F1DC
:10F5F400804303F58003B3F5801F37D32A464D4972
:10F604004E48FFF773FBD7E78A0706D04C494D48AD
:10F61400FFF76CFB4FF0FF3421E00128C1F39502A2
:10F62400304615BF48494949DFF82491DFF8249151
:10F6340000F0F6F80446A0B928F00308B844B84529
:10F644000DD04946304657F8042B00F0E9F805463A
:10F654000028F4D03A494048FFF748FB2C4664B2EE
:10F66400ACE737493D48FFF741FBF8E7294696F8F0
:10F674005C0000F01BF978BBB4F5813F2CD305F195
:10F68400A043B3F5443F27D305F1804303F580033A
:10F69400B3F5801FB2D2AB0749D14FF0FF3428F045
:10F6A4000308B844ED1B4745D9D096F85C30E919F6
:10F6B400C1F31301012B01F12441304657F8042B07
:10F6C40014BF503101F5A87100F0AAF804460028CF
:10F6D400E9D023492348C6E700236946284696F81B
:10F6E4005C20CDE9003300F0FBF8044620B11E494C
:10F6F4001E48FFF7FBFA61E7D6F8B80001A9FFF747
:10F70400D7FA304601F040FD044648B1164918487E
:10F71400FFF7ECFAD6F8B80001A9FFF7CFFA4DE7E6
:10F7240043463A460099B06807F043F8F2E70C49BB
:10F7340010486DE70864020096B60100A9B60100FE
:10F74400F563020000B70100300000A4300100A4FA
:10F75400340000A4340100A446B7010024B701001A
:10F76400D16302009BB70100E3630200C9B6010044
:10F77400ECB6010065B70100F7B5134600220F4649
:10F784000546CDE9002250B121B103F07E42B2F129
:10F79400244F09D03A461D491D48FFF7A7FA4FF0F8
:10F7A400FF34204603B0F0BD90F85C20694618464B
:10F7B40000F096F8044620B114491648FFF796FA6B
:10F7C400EFE7D5F8B80001A9FFF772FA284601F06F
:10F7D400DBFC044648B10D490F48FFF787FAD5F81A
:10F7E400B80001A9FFF76AFADBE70099A86806F0F8
:10F7F400CEFF431C06463860F1D10346009A034904
:10F804000648FFF773FA3446E9E700BF4E64020086
:10F81400B9B70100C9B60100ECB60100E6B70100B2
:10F8240073B50023054616460846CDE900334DB1AD
:10F8340001F07E43B3F1244F09D00A461748184912
:10F84400FFF754FA4FF0FF34204602B070BD69460A
:10F8540095F85C2000F044F8044620B110491148A2
:10F86400FFF744FAF0E7D5F8B80001A9FFF720FA4A
:10F87400284601F089FC044648B109490A48FFF7C3
:10F8840035FAD5F8B80001A9FFF718FADCE73246D3
:10F894000099A86806F080FFF3E700BF1BB80100D9
:10F8A4003C64020043B80100ECB60100012810D802
:10F8B40043420320094A03F0180313441A688A4296
:10F8C40002D85A688A4206D2013803F10803F5D1F6
:10F8D4007047002070470120704700BF6874010022
:10F8E40000F07F43B3F1244F70B504460E4615462D
:10F8F40020D000F19242B2F5813F1DD3B3F1254FE0
:10F904001DD0B3F1304F1DD001462846FFF7CEFF7E
:10F9140040B10E4B53F8253024F07F441C440020A2
:10F92400346006E022460A490A48FFF7DFF94FF03F
:10F93400FF3070BD0023EFE74FF40023ECE74FF4F2
:10F944008023E9E74FF44023E6E700BF6074010039
:10F954005F64020068B801002DE9F04F95B00746D6
:10F964000C461E986AB90A464F485049FFF7BEF93B
:10F974004FF0FF350023284687F85C3015B0BDE80A
:10F98400F08F18B90A464A484849EFE787F85C10EF
:10F9940029B101293FD00A4646484449E6E7464989
:10F9A400464DCDE90E35464B464ECDE910301F9BF2
:10F9B400CDE90C62444ACDE9123114F001030993F4
:10F9C400424B18BF13460DF130080893D8F80030A5
:10F9D4004FF0FF350493D8F80C3000260593D8F87F
:10F9E40004300693D8F80830C3F30B02B2F10009CF
:10F9F40018BF4FF0010909EB133909EB050307920E
:10FA04000A93B1450ADC002DB2D108F1100814ABF9
:10FA14009845AFD0DAE72E492E4DC2E70A9BDDF8B0
:10FA24001CB0B34218BF4FF4805B069B584603EBEF
:10FA34000631059B0B9103EB0635FFF7EBF80B99A9
:10FA4400824678B909982049204A0136002818BF0F
:10FA54000A46CDE9019B049B1F4900961F48FFF706
:10FA640045F985E75A46FFF7F3F85B4629465246BF
:10FA7400384687F85C40FFF793FD0023054687F876
:10FA84005C3048B1731C0093CDE9019B049B089A38
:10FA940011491348FFF72AF95046FFF7CDF8002D16
:10FAA4007FF468AF0136ACE782B80100A4640200B9
:10FAB400A9B80100D2B80100803A0480C0BB048018
:10FAC400FAB80100F5B8010091B601008CB6010046
:10FAD40000C0088000B8098092640200FEB80100EA
:10FAE4003AB9010000232DE9F347074616460D46AF
:10FAF4000193A9B962BB4FF024489246914632491A
:10FB04000423384687F85C500DEB0302FFF748FDE9
:10FB1400044648B32A462D492D48FFF7E7F810E07C
:10FB2400012907D1DFF8AC80CAB9924691464FF05B
:10FB34003041E5E70A4628482449FFF7D7F84FF053
:10FB4400FF340023204687F85C3002B0BDE8F0871C
:10FB54004FF024484BF6C03ADFF88090CFE74FF4DB
:10FB6400DC3ADFF87C90E2E77EB94FF000091D4EE5
:10FB740006EB45163846D6E90012FFF751FE044657
:10FB840078B12A4611491848C7E7524649463846CB
:10FB9400FFF746FE04460028E7D02A460B491348DF
:10FBA400BBE709F10109B9F1040F06F10806E1D137
:10FBB400012241463846FFF733FE04460028C0D0F0
:10FBC4002A4602490A48A8E7500D00B777640200A4
:10FBD4008FB90100000100A46DB901002C2C00A410
:10FBE400302C00A498740100F3B90100C4B90100D9
:10FBF4001EBA010010B50C4606F0B3FC102C0146E9
:10FC040007D801221048A240104008D112F4027F04
:10FC140010D122460D490E48FFF768F807E091F825
:10FC24003030022B0DD909490A48FFF75FF84FF02D
:10FC3400FF3010BD91F83130012BFAD90349064841
:10FC4400F3E70020F5E700BF04A10100FD64020012
:10FC54008EBA01003FBA010067BA010010B50C4624
:10FC640006F07FFC102C07D801230D4AA340134251
:10FC740009D113F4027F0CD12246BDE81040094992
:10FC84000948FFF733B890F83030013380F830304A
:10FC940010BD90F83130013380F83130F8E700BFFF
:10FCA40004A10100DE640200B2BA010010B50C46E2
:10FCB40006F057FC102C07D801230D4AA340134229
:10FCC40009D113F4027F0CD12246BDE81040094942
:10FCD4000948FFF70BB890F83030013B80F830301A
:10FCE40010BD90F83130013B80F83130F8E700BFA7
:10FCF40004A10100BF640200B2BA01002DE9F04181
:10FD04000E461746044628B1C5683DB10F49104850
:10FD1400FEF7ECFF4FF0FF30BDE8F081006806F01D
:10FD24001EFC8046204606F01CFC10B90749094811
:10FD3400EEE7D8F8003013B904490748E8E700684B
:10FD44003A46314698472846E6E700BF1B6602005C
:10FD5400CEBA0100E2BA0100FDBA0100F8B50546C9
:10FD6400006806F0FCFB0746284606F0FAFB002470
:10FD740006467B6C9C4205D3706BFEF763FF002341
:10FD84007363F8BD22460121284602F0F1F830B130
:10FD94002246BDE8F84003490348FEF7A7BF0134F3
:10FDA400E7E700BF6066020023BB0100F8B50E461A
:10FDB400054630B129B1476837B110491048FEF7FC
:10FDC40095FF00242046F8BD6C20FEF729FF044669
:10FDD40010B90A490B48F2E7C0E900560146286801
:10FDE40001F09AF8A06038B904490748FEF77EFF8D
:10FDF4002046FEF721FFE4E7E760E3E7CB66020075
:10FE0400CEBA010049BB01006DBB010010B5C36847
:10FE140004462BB1BDE8104007490848FEF766BF09
:10FE2400806806F093FC2046FFF798FF206BBDE83E
:10FE34001040FEF701BF00BF43660200CEBA0100C6
:10FE44002DE9F041074688B050200E469046FEF753
:10FE5400E7FE054640B92F492F48FEF747FF002526
:10FE6400284608B0BDE8F08106F079FB044620225C
:10FE740000216846FEF7F2FE202241462046FEF7A6
:10FE8400E7FE0B22394604F12000FEF7E1FE0C22C6
:10FE9400314604F12B00FEF7DBFEB4F82D10B4F864
:10FEA4003120E1630A44B4F8351022640A446264E0
:10FEB40043F204420023ADF808206A46A36304EB2E
:10FEC4008301B1F82D0001339081B1F82B10032B7D
:10FED40001F10401518102F10402F0D140F21E63E8
:10FEE4004FF4C87106934FF47A736846CDE9001352
:10FEF4000A4A0B4901F0F0FB286038B90549094862
:10FF0400FEF7F4FE2846FEF797FEA8E700236B6091
:10FF1400A6E700BF0466020091BB010001FD0000DA
:10FF2400050B0100AEBB010027232DE9F047B2F811
:10FF3400E781C56806468A46174603FB08F845B1BB
:10FF440017491848FEF7D2FE4FF0FF352846BDE8A2
:10FF5400F08708F20E2906F004FB4846FEF760FE1F
:10FF6400044610B90E491048ECE70369394643F0DA
:10FF740001030361057245728572C572C0F81CA045
:10FF8400056208F5F5722430FEF762FE4A46214602
:10FF9400304601F091FD05462046FEF74DFED5E7BB
:10FFA400ED650200CEBA0100C8BB01002DE9F041A5
:10FFB400C56806468846174645B115491548FEF7F3
:10FFC40095FE4FF0FF352846BDE8F08106F0C9FAEA
:10FFD4002820FEF725FE044610B90D490E48EEE729
:10FFE400012303720369014643F0010345728572DC
:0CFFF400C572C0F81C8005620361476202
:020000021000EC
:100000002822304601F05AFD05462046FEF716FE2E
:10001000DBE700BFCE650200CEBA0100C8BB01001D
:100020002DE9F84FC36880460C4691463BB14549DF
:100030004548FEF75DFE00273846BDE8F88F06F01C
:1000400092FAD9F800208246102A03D83F4BD340B9
:10005000DB0705D43B493E48FEF74AFE0227EBE7A3
:1000600011464046FFF7C8FD05460028F6D124207A
:10007000FEF7D8FD064620B932493648FEF738FE6D
:10008000ECE749464FF0010BC0E9008451F80C3B06
:100090000622836180F822B00830FEF7DBFD40467F
:1000A00006F082FA0228074609D126492A48FEF7B7
:1000B0001FFE00243046FEF7C1FD02273AE090B350
:1000C0004A20FEF7AFFD044610B91E492348EEE76B
:1000D0000F2303720369222243F00103036149469F
:1000E00045728572C57280F81CB045778577C577F3
:1000F00080F8205080F8215080F8225080F823505A
:100100002830FEF7A7FD636A4A2243F00E0321461A
:100110004046636201F0D2FC013005D10949104824
:10012000FEF7E6FDC6E704464AF827604046B16997
:10013000FFF796FD002C3FF47FAF2046FEF77EFDD3
:100140007AE700BFB4650200CEBA01000CA301003B
:10015000E6BB010004BC01002EBC01004FBC010045
:1001600075BC01002DE9F041C36807468846164674
:1001700023B128492848FEF7BBFD0AE01268102A7F
:1001800003D8264BD340DB0706D422492448FEF788
:10019000AFFD4FF0FF3539E01146FFF72DFD054665
:1001A0000028F6D13020FEF73DFD044610B919496C
:1001B0001C48E0E7102303720369457243F0010312
:1001C0008572C5720562036108223146C0F81C8041
:1001D0002830FEF73FFD636A302243F003032146D7
:1001E0003846636201F06AFC05462046FEF726FDAC
:1001F00065B9384606F0B7F90446326841463846D4
:1002000006F0B3F954F8283032689A612846BDE800
:10021000F08100BF80650200CEBA01000CA301008E
:10022000E6BB0100C8BB01002DE9F743C5680746DE
:100230000E464DB133493448FEF75AFD4FF0FF35B5
:10024000284603B0BDE8F08306F08DF950F82690FB
:100250008046D9F81820102A03D82C4BD340DB074E
:1002600004D428492A48FEF743FDE7E78EB124204D
:10027000FEF7D8FC044640BB22492648FEF738FD6D
:100280004FF0FF354846FEF7D9FC002348F82630EA
:10029000D6E7022A10D0032A02D0083A012A0BD846
:1002A000082200216846FEF7DBFC02236A46002193
:1002B00038460093FFF756FF00243846D9F8181047
:1002C000FFF7F6FCE4B1002516E011230372036981
:1002D000457243F001038572C57205620146C6612D
:1002E00003612422384601F0E9FB05460028E4D0EA
:1002F00004490948FEF7FCFC2046FEF79FFCC1E7D5
:100300002546BFE79A650200CEBA01000CA30100A2
:10031000E6BB01004FBC0100A0BC01002DE9F84381
:10032000C56806460F46914645B121492148FEF76A
:10033000DFFC4FF0FF352846BDE8F88306F013F9DF
:1003400080462920FEF76EFC044610B918491A4869
:10035000EDE7122303720369457243F001038572CE
:10036000C572C76105620361052249462430FEF764
:1003700071FC58F8277030463D752922214601F05E
:100380009DFB42F2107605463B7D43B9013E0AD102
:100390000A2207490948FEF7ABFC4FF0FF3520461B
:1003A000FEF74CFCC7E70120FEF754FDECE700BF69
:1003B00060650200CEBA0100C8BB0100CBBC0100E1
:1003C0002DE9F04188461746054620B94FF0FF3524
:1003D0002846BDE8F08122B916491748FEF788FC87
:1003E000F4E7C66816B113491448F7E72A20FEF768
:1003F00019FC044610B90F491148EFE73423037282
:100400000369394643F00103036146728672C6727E
:10041000C0F81C80066206222430FEF71BFC2A224C
:100420002146284601F04AFB05462046FEF706FC19
:10043000CEE700BF3E6502008C960100CEBA0100F7
:10044000EEBC01004FF0FF332DE9F04FB5B00C4684
:100450000546049300B149B99A499B48FEF748FC08
:100460004FF0FF36304635B0BDE8F08FC36813B1AA
:1004700094499648F2E7BC22FF21076B05A8FEF7D6
:10048000EFFBA86833AA05A901F068F9064620B178
:100490008C498F48FEF72CFCE4E7A86803A901F01B
:1004A0008DF9064610B187498A48F3E7A86804A980
:1004B00001F0A4F9064610B182498748EAE70146EF
:1004C00004222046049DFEF7CBFB44F245339D42B7
:1004D00000F095806FF003036FF007014FF0330ACF
:1004E00003224FF054094FF0400E4FF0380C3020EB
:1004F0009B46CDE9003122736273A2733422A27449
:10050000E274A2754322A377009B002584F8213072
:10051000FC2322774FF02A08072284F82230019B1F
:1005200084F810E084F811E0207584F815C0E075B7
:10053000627784F8201084F823309E21674AE571A1
:1005400025726572A57225766576A576E57684F8BE
:10055000068084F80BA084F80F90E57704F12A0058
:1005600084F8245084F825B0FEF754FD013084F857
:100570009B5084F89C5084F89D5084F89E5084F8D9
:100580009F5084F8A05084F8A15084F8A25084F8B9
:10059000A35084F8A45084F8A55084F8A65084F899
:1005A000A75084F8A85084F8A95084F8AA5084F879
:1005B000AB5084F8AC5084F8AD5084F8AE5084F859
:1005C000AF5084F8B05084F8B15084F8B25084F839
:1005D000B35084F8B45084F8B55084F8B65084F819
:1005E000B75084F8B85084F8B95084F8BA5084F8F9
:1005F000BB5084F8BC5017D1324939482EE74FF030
:10060000340C6FF013036FF00B054FF0450A052211
:100610004FF044094FF03C0E60466FF003016FF05D
:10062000070BCDE9005366E7339B1B0704D4012277
:100630002AA9A01DFEF70EFBBDF80E3003F00F0334
:1006400003933A7894F90F309342A8BF1346E373AB
:10065000BA7894F910309342A8BF134623747A787D
:1006600094F911309342A8BF134663743A7994F910
:1006700012309342A8BF1346A374BA7994F9133089
:100680009342A8BF1346E3743A7A94F91430934224
:10069000A8BF13462375FA7894F915309342A8BF82
:1006A000134663757A7994F916309342A8BF1346BE
:1006B000A375FA7994F917309342A8BF1346E375EE
:1006C000D0E600BF1E6502006A940100CEBA0100A8
:1006D00010B6010009BD010033BD010057BD010086
:1006E0003ABE01002DE9F04F894692469B460546E9
:1006F000EBB048B955495648FEF7FAFA4FF0FF34C7
:1007000020466BB0BDE8F08FC36813B14F49514824
:10071000F2E70920FEF780FA092276992863FEF7AE
:1007200099FAA86801F08AF8044620B147494A4876
:10073000FEF7DEFAE4E7BC22FF2109A8FEF790FAF3
:10074000A86837AA09A901F009F8044610B13F4981
:100750004248EDE7284638A9FFF774FE044610B179
:100760003A493F48E4E7286805F0FBFE80462868E0
:1007700005F0F7FE0746284605F0F5FE0646786CBC
:10078000C000FEF755FA706300283CD13549364861
:10079000FEF7AEFA4FF0FF340BE032460021284658
:1007A00001F0E8FB044658B132462E492F48FEF7C7
:1007B0009FFA2F492F48FEF79BFA631CA0D141E016
:1007C00001367B6C9E42E8D3002CE3D1789B01225A
:1007D0000693779B28460593759BCDE9009A049371
:1007E0009DF8D03138A9CDE902B308F1200300F01B
:1007F0004BF8044658B11E491F48FEF779FA2846BF
:10080000FFF7AEFAD9E726464FF0FF34D9E7FEF7F7
:1008100031FB0646194FAB7D002B7FF471AF0120F1
:10082000FEF718FB3046FEF72DFBB842F3D9AB7D3F
:10083000002B7FF465AF0E491148FEF759FA2846A0
:10084000FFF78EFA01490F4856E700BFB066020075
:10085000E2BA0100CEBA010075BE010010B6010077
:1008600096BE01007C660200B3BE0100D0BE01004E
:1008700096660200F4BE010007BF01003F4B4C002A
:100880001CBF010034BF01002DE9F04F87B0029377
:10089000109B04460393DDE914930493169B0068B0
:1008A000884616460593DDF844B09DF848A09DF8AB
:1008B0004C5005F056FE4FF4B772019000212046CF
:1008C00001F0E6F80746002800F00E816E210022B4
:1008D00001740121027342738273C2734174827482
:1008E000C27480F8FE6026B1C82241463630FEF759
:1008F000B1F96FF07B023A771C227A776FF07702BA
:1009000087F82020132287F821204E2287F82520FF
:10091000142200264FF00108C7F82CB087F84A21AE
:100920004FF0200B3222039B0199BB6187F84F21C6
:100930002B310C22BE77FE7787F8226087F8236080
:1009400087F824B087F8266087F8276087F8288022
:1009500087F8296087F82A6087F82B6087F83A8142
:1009600087F84B6187F84C6187F84D6187F85061D3
:1009700087F8516187F8526187F8418107F1FF00DC
:10098000FEF768F90B22029907F20B10FEF762F9E5
:100990007B2287F81A21102287F824210C2287F85D
:1009A0002A210E2287F82E21282287F832210822B8
:1009B00087F8168187F8262187F81761042287F8BF
:1009C000186187F8196187F81B6187F81C6187F83F
:1009D0001D6187F81EB187F81F6187F8206187F8CD
:1009E000216187F8226187F8236187F8256187F8FC
:1009F0002B6187F82C6187F82D6187F82F6187F8C4
:100A0000306187F8316187F8336187F8346187F89E
:100A1000356187F8276187F8286187F8296107F130
:100A2000EF00C7F83DA10499FEF714F904224946E6
:100A300007F1EB00FEF70EF91A2209F1040107F1A4
:100A4000D100FEF707F90222059907F23B10FEF7E5
:100A500001F93DB987F8468187F8475187F8485131
:100A600087F849516FF0050187F858110A210022D3
:100A700087F86111012187F84E2187F8592187F8FD
:100A80005A2187F85B2187F85C2187F85D2187F878
:100A90005E2187F85F2187F8602187F8622187F857
:100AA000632187F8642187F8651187F8662187F844
:100AB000672187F8682187F8751187F8762187F80C
:100AC000772187F8782187F8712187F8722187F8D4
:100AD000732187F8742139464FF4BD72A06807B0BE
:100AE000BDE8F04F00F044BC04490548FEF700F9AA
:100AF0004FF0FF3007B0BDE8F08F00BFE5660200A1
:100B000059BF01002DE9F0418D680746022D0C46C2
:100B100009D0032D2DD0002D00F098804FF0FF3527
:100B20002846BDE8F0810028F8D04FF0FF3554F892
:100B30000C6B0C3E002EF3DD384605F014FDD4F8A6
:100B40000080B8F1030F0FD12146384601F0A8FA12
:100B5000054648B142464E494E48FEF7C9F84E494F
:100B60004E48FEF7C5F8DBE763680025F61A1C441B
:100B7000E0E720B94A494B48FEF7BAF812E00068AE
:100B8000D1F8008005F0EDFC0646384605F0EBFC98
:100B900046B138B1A26AD2B2012A05D940494248C9
:100BA000FEF7A6F80025BBE750F8220010B93C4933
:100BB0003E48E1E740F21313626904F10C019A42E6
:100BC0003BD0B2F58A7F0CD2B2F5817F24D040F2BF
:100BD00003139A421ED040F201139A42E2D1736885
:100BE0000BE040F221139A4209D040F223139A42BB
:100BF00018D0B2F58E7FD5D1B36913B907E0F36988
:100C00001BB1424640689847CCE740F22112244984
:100C10002748C5E7B368F0E7F368002BF1D14FF43C
:100C20008172F4E723697469003B18BF0123002C2B
:100C3000EDD042464068A047B4E7226B002A02DAB2
:100C400017491C48ACE701230375ABE700283FF4C4
:100C500065AF05F088FCE268022A08D0032A14D0A8
:100C6000012A10D014491548FEF742F856E73B7D9B
:100C7000002B97D040F28722386904F11401FDF768
:100C8000E9FF3D758EE7BA758CE70123FB7589E7AF
:100C90002A67020073BF01004B6702008DBF01008D
:100CA000126702006A940100B0BF0100D6BF0100C4
:100CB000EABF010012C00100F766020038C001005F
:100CC00013B50023044601A9806E0193FDF7F2FFDE
:100CD00094F8D4303BB9204600F040FC18B10549E7
:100CE0000548FEF705F8A06E01A9FDF7E9FF02B07F
:100CF00010BD00BF9667020053C0010037B5002544
:100D00000446019528B90E490E48FDF7F1FF03B0DE
:100D100030BDD0F8DC0001A9FDF7CCFF23681B6AC9
:100D200043B12A4629466068984718B106490748E2
:100D3000FDF7DEFFD4F8DC0001A9FDF7C1FFE6E70F
:100D4000B867020075C00100A76702008DC00100EE
:100D50002DE9F047DDF820E0044620B100EB830ADE
:100D6000DAF86C6036B924492448FDF7C1FF002346
:100D70009B68FFDE4FEA0E1816F8089006EB0E1778
:100D8000B9F1000F04D01C491D48FDF7B1FF0CE07C
:100D90007960FA60D0F8009009EB8305ED8D9542FB
:100DA0000AD015491748FDF7A3FFB86810B1012311
:100DB00006F80830BDE8F087DAF888300A4605FB07
:100DC0000E3AC36FAAEB030C0CF1304199F82C30AA
:100DD00001F5A041FEF7E6FB23682A4693F82C10A4
:100DE000A0680123514405F0EEFCB8600028DCD176
:100DF00001490548C9E700BF226802006A94010062
:100E0000A5C00100CDC00100F7C00100F8B500EB9E
:100E10008202D26E0F46190102EB0314535C0546A1
:100E200033B914491448FDF763FF00252846F8BD7F
:100E30000123D4E90212806805F0CDFC97B110B906
:100E40000C490E48EFE72B68EE6F93F82CC06168F1
:100E5000C6F1304606F5A04632183B4628466144A6
:100E6000FEF742FB1022002120466568FDF7F8FEE0
:100E7000DCE700BF046802000AC101002CC10100C8
:100E80002DE9F0410E460546006E14469846FDF7E2
:100E900005FF022E1FD10821AF6C069B022E03FB1B
:100EA000017708BF27F07F41224618BF39464346E5
:100EB000284608BF41F04041FEF774FB0446B8B134
:100EC000324612491248FDF713FF286EFDF7ECFE7B
:100ED0002046BDE8F081042E02D19421EF6CDCE7BE
:100EE0000A4932460B48FDF703FF00210F46D4E7BD
:100EF0003B4631462846079A00F0E6F904460028AA
:100F0000E3D002490448FDF7F3FEDEE7E56702009F
:100F100062C1010041C1010089C1010070B50546EF
:100F2000E0200E46FDF77EFE044630B96B496C4862
:100F3000FDF7DEFE0024204670BDC0E900562B7987
:100F40005A1C2A7103734DF6AD63036505F038FB37
:100F5000606538B961496348FDF7CAFE2046FDF770
:100F60006DFEE7E705F02CFBA06538B95B495E48EC
:100F7000FDF7BEFE606D05F025FBEFE7FDF77CFE9B
:100F80000646206628B955495848FDF7B1FEB36DAD
:100F9000FFDEFDF77DFEFDF76FFEA06650B94F49FD
:100FA0005248FDF7A5FE206EFDF76CFEA06D05F022
:100FB00009FBDFE7FDF76CFE0020FDF723FF60660D
:100FC00038B946494A48FDF793FEA06EFDF75AFE30
:100FD000E9E722464749FDF725FF0020FDF712FF0C
:100FE000C4F8D80038B93D494348FDF781FE606E2A
:100FF000FDF710FFE9E722464049FDF713FFFDF733
:101000003BFEC4F8DC0040B934493D48FDF770FEB2
:10101000D4F8D800FDF7FEFEE9E7FDF739FE2046DB
:1010200000F020F940B12D493648FDF761FED4F8B3
:10103000DC00FDF727FEEBE72146286800F03AFCCC
:10104000A06010B925493048EFE7204600F074FD54
:10105000054638B121492D48FDF74AFEA06805F044
:1010600087FBE4E704F16806236803EB8503188E29
:101070000001FDF7D7FD46F8040F28B92A461749A5
:101080002348FDF735FEE9E70135032DECD194F84F
:101090005C20204804F17C01FEF724FC40B11E498D
:1010A0001E48FDF725FE0D491D48FDF721FE42E7CC
:1010B000E36F2268C4F8803003F52A339033C4F814
:1010C0008830118ED08D00FB0133C4F88C30918EA6
:1010D000528E02FB0133C4F890302CE7CC6702003B
:1010E000AFC10100D2C10100F7C101001AC2010065
:1010F0003AC20100C10C01005FC20100FD0C0100F9
:1011000087C20100ACC20100C7C20100E7C20100F2
:1011100005C30100005000B06D670200C9B60100B0
:1011200026C3010000232DE9F34107460D469046F2
:10113000322601932A46384601A9FEF71FFB0446D2
:1011400028B12A46019B0E490E48FDF7D1FD019BAF
:1011500003F00103434508D00A20FDF77BFE013E62
:10116000E8D2204602B0BDE8F0813EB92A460449E3
:101170000548FDF7BDFD4FF0FF34F2E70024F0E72E
:10118000C368020041C3010071C301002DE9F341AE
:10119000044648B92F493048FDF7AAFD4FF0FF3506
:1011A000284602B0BDE8F08190F8BE50002DF7D07F
:1011B00090F8B030012B46D0806805F019FB012370
:1011C00084F89830FDF766FEC4F89C00FDF752FEE7
:1011D00006464FF47A70FDF745FEDFF88080A06880
:1011E00005F00BFB00F00603062B05461CD0FDF7AF
:1011F00041FE07463846FDF745FEB0F57A7FF9D344
:101200003046FDF73FFE4045E9D90623012211494A
:10121000009313482B46FDF76BFDD4F8D800FDF77B
:1012200009FE4FF0FF350FE00123D4F8A00084F849
:10123000B030FDF737FE41F28833984203D9D4F835
:10124000A030C4F8A43000250A21D4F8B400FDF77A
:10125000B1FEA5E7E96902006A9401003F420F0070
:1012600091C3010010B50446FDF706FDC4F8B800AF
:1012700030B911491148FDF73BFD4FF0FF3010BD6B
:10128000FDF706FDFDF77EFEC4F8B40040B90A493B
:101290000B48FDF72DFDD4F8B800FDF7F3FCECE7A3
:1012A00022460849FDF77EFE0020012384F8B000A5
:1012B00084F8BC30E3E700BFD9690200E3C3010052
:1012C000FFC30100D1650100022A70B504460E4635
:1012D000104607D91E491F48FDF70AFD4FF0FF359C
:1012E000284670BD11F0FB0F0CD104F120011A4605
:1012F000204600F00BFE054670B115491648FDF773
:10130000F7FCEDE7022903D1063004EBC001EEE75C
:101310000A4612480E49DFE7022EE1D0226D204630
:1013200042F0FF420E4942F4FE02FEF77BFA064607
:1013300048B10C490C48FDF7DBFC05490B48FDF7AB
:10134000D7FC3546CCE7236D01332365C8E700BFE2
:10135000C86902001CC4010050C4010036C4010069
:10136000800400A4B469020076C401009DC4010099
:101370002DE9F34705461646006E0F46FDF78EFC35
:101380002B685B6A9E4243D9B9464FF0FF34002E6A
:1013900008DC3846FDF752FCBCB94FF0FF34DFF8EB
:1013A000688171E02B68B2465B6AB3423CBF9846E5
:1013B000C2460AF1040028BFB046FDF733FC0446DC
:1013C00030B952495248FDF793FC4FF0FF3410E01A
:1013D000524649460430FDF73DFCC4F800A02146C2
:1013E000686D05F0F1F8044670B148494948FDF7C9
:1013F0007FFC49494948FDF77BFC286EFDF754FC0A
:10140000204602B0BDE8F087A6EB0806D144BEE74F
:10141000301DFDF707FC044610B93C494048D2E7AF
:10142000324639460430FDF715FC26602146686DCA
:1014300005F0CAF804460028ABD034493948D6E74D
:10144000FDF718FD044600230193EA6A284601A926
:10145000FEF794F9019A0746E8B133493348FDF79E
:1014600047FC2046FDF70EFD4045ECD900223049EF
:101470003048FDF73DFC30493048FDF739FC304637
:10148000FDF7DCFB4FF0FF34686D05F09FF8064672
:101490000028D5D1B1E7002AE3D0D6F8009005F1B5
:1014A0002801019001AA284600F040FD0199044658
:1014B00090B10A4622482349FDF71AFC3A462249D0
:1014C00022480197FDF714FC1B492148FDF710FC49
:1014D0003046FDF7B3FBD7E74B462846321DFEF7F3
:1014E00061F8044620B118491A48FDF701FCEBE702
:1014F00002460146019B2846FFF7E6FE0446002807
:10150000E6D011491448F0E73F420F008769020016
:10151000BFC40100E9C40100996902005FC5010070
:101520000AC5010038C5010045690200D6C50100A1
:101530005A6902007EC501006D690200A4C5010060
:1015400007C601001E6902003369020033C60100AC
:101550008BC6010065C601009DC4010070B506463A
:101560000024B06D05F032F8054680B101463368BD
:1015700051F8042BDB6970689847044618B1054997
:101580000548FDF7B5FB2846FDF758FBE9E720467F
:1015900070BD00BF0769020058990100012970B5AC
:1015A00005460E460BD90A461E481F49FDF7A0FB0B
:1015B0004FF0FF34002385F85C30204670BD0122D7
:1015C00080F85C1059B94FF02441FEF72BF904461E
:1015D000A0B1324614491548FDF78AFBEAE71449E1
:1015E000FEF720F904460028F3D1024610492846A8
:1015F000FFF798FD48B901220E490DE002464FF071
:1016000024412846FFF78EFD20B144B232460649F8
:101610000948E1E7012209492846FFF783FD44B262
:10162000C8E700BFADC60100D9680200CFC60100FF
:10163000000100A4180100A406C70100180000A4BE
:101640002DE9FF41002506460C46039571B301299B
:1016500031D00A461C481D49FDF74AFBA8466327BE
:1016600086F85C4004234246304603A9FDF73CFF60
:1016700020B1224615491648FDF73AFB039BAB42C1
:101680001ED00A20FDF7E6FB013FEBD2039B22466A
:1016900000930E492B460F48FDF72AFB4FF0FF3011
:1016A000002386F85C3004B0BDE8F0814FF05A3575
:1016B000DFF82480D3E74FF05A354FF03048CEE7BB
:1016C000002FE3D00020EBE72FC70100AA6802003B
:1016D0004EC701007FC70100500D00B7F7B50746A0
:1016E00048200E461546FDF79DFA044628B91649CE
:1016F0001648FDF7FDFA002412E020223946243076
:10170000FDF7A8FA02224FF03040C4E9076504F162
:101710004401FEF7E7F830B10B490D48FDF7E8FA50
:10172000204603B0F0BD636C0A4901A8019300F0A4
:10173000FDF820600028F3D103490748FDF7D8FAE7
:101740002046FDF77BFAD6E798680200C3C7010080
:10175000C9B6010035660100EBC7010070B5164639
:10176000054600B139B910491048FDF7C1FA4FF0EC
:10177000FF34204670BDB8234FF03042FDF7B4FE71
:10178000044620B108490A48FDF7B2FAF1E70423FC
:1017900031462846074AFDF7A7FE04460028E8D050
:1017A00001490548F0E700BF7E6802006A94010025
:1017B000F6C70100DC4F00B00EC8010010B500B143
:1017C00039B90A490A48FDF793FA4FF0FF34204629
:1017D00010BD0423074AFDF787FE04460028F6D013
:1017E00002490548FDF784FAF1E700BF5D68020091
:1017F0006A940100D84F00B027C8010010B500B1AD
:1018000039B90A490A48FDF773FA4FF0FF34204608
:1018100010BD0423074AFDF767FE04460028F6D0F2
:1018200002490548FDF764FAF1E700BF3E6802008F
:101830006A940100D44F00B049C8010038B50123B3
:10184000054680F8BE30806800F05CF8044628B198
:1018500011491248FDF74CFA204638BD3823284676
:101860000F4A05F11001FDF73FFE044610B10A4989
:101870000C48EFE7042328460B4A05F14801FDF721
:1018800033FE044610B104490848E3E7084B2846F4
:10189000EB6404F040FFDFE7F168020065C8010077
:1018A000240000B086C80100580D00B7A5C801008B
:1018B000B80000B070B5054610200E46FDF7B2F92D
:1018C000044630B90C490D48FDF712FA00242046B1
:1018D00070BDC0E900566B6801469B682868984750
:1018E000A0600028F3D104490548FDF701FA20461D
:1018F000FDF7A4F9EAE700BF216A0200C8C80100A9
:10190000EBC80100012310B50373036880685B68AE
:101910001B699847044618B102490348FDF7E8F9E6
:10192000204610BD0B6A020002C9010070B50546D1
:1019300014200E46FDF776F9044630B90E490F48DB
:10194000FDF7D6F90024204670BD066100F09CF832
:10195000606038B908490A48FDF7CAF92046FDF722
:101960006DF9EFE70368074928469847206000288B
:10197000E9D101490448EFE7F969020016C90100FD
:101980003EC9010069670100EBC7010073B5054658
:1019900014200E46FDF746F9044638B9104911489F
:1019A000FDF7A6F90024204602B070BDC0E900563C
:1019B00001462868FDF78EFAA06038B908490A4840
:1019C000FDF796F92046FDF739F9EBE76946FDF793
:1019D000B1FA009AE260AB6813442361E3E700BF09
:1019E0004D6A020058C901007CC9010070B5064665
:1019F0000C200D46FDF716F9044630B90C490D4888
:101A0000FDF776F90024204670BD042231460830E7
:101A1000FDF720F96560FDF74DFA20600028F2D14E
:101A200003490548FDF764F92046FDF707F9E9E7A2
:101A3000366A02000E990100A6C9010038B50146B8
:101A400005460D4A8068FDF765FA044628B10B4942
:101A50000B48FDF74DF9204638BDA868FDF74AFA56
:101A600004460028F7D005490648FDF741F9A86863
:101A7000FDF758FAEFE700BF05680100676A02004A
:101A8000C9C90100F4C901000048704740020020A4
:101A900070B502F10C0528460E46FDF7C3F8044662
:101AA00028B904490448FDF723F9204670BD866033
:101AB0000560FAE78F6A02001BCA0100F8B5837D52
:101AC00005460F4616463BB98A680F480F49FDF791
:101AD0000FF94FF0FF30F8BD0321FFF7D9FF04469F
:101AE00020B90A490A48FDF703F9F2E732463946B8
:101AF0000C30FDF7AFF82146A86806F10C02BDE8EE
:101B0000F840FFF735BC00BF3BCA0100826A020003
:101B100059BF01000A4610B500F1180100F0F6F9AE
:101B2000044618B102490348FDF7E2F8204610BD0B
:101B3000DF6A020061CA0100002337B5144A01A917
:101B400005460193FDF71AFE044630B111491248CB
:101B5000FDF7CEF8204603B030BD019A284642F486
:101B600000320B490192FDF75DFE044610B10949B0
:101B70000A48EDE74FF00042284609490192FDF777
:101B800051FE04460028E5D002490648E0E700BFC0
:101B9000000400A42E6B020080CA0100B0CA01003C
:101BA000940400A4D3CA01002DE9F04F04468846EE
:101BB0000027A3B000F1100A00235146204601AAD5
:101BC000019300F0B3F9834608B3B649B648FDF770
:101BD0008FF8002502952046B44A02A9FDF7CEFDF4
:101BE000002800F00D81B249B248FDF781F8002FBE
:101BF00000F08A814FF000422046AF49FDF712FE07
